:020000040000FA
:2000000000800010B9020000C1020000C3020000C5020000C7020000C90200006E6FFFEFE7
:20002000000000000000000000000000CB020000CD02000000000000CF020000D102000080
:20004000D3020000D3020000D3020000D3020000D3020000D3020000D3020000D3020000F8
:20006000D3020000D3020000D3020000D3020000D3020000D3020000D3020000D3020000D8
:20008000D3020000D3020000D3020000D3020000D3020000D3020000D3020000D3020000B8
:2000A000D3020000D3020000D3020000D3020000D3020000D3020000D3020000D302000098
:2000C000D302000000F002F800F0C0F80AA090E8000C82448344AAF10107DA4501D100F07A
:2000E000B5F8AFF2090EBAE80F0013F0010F18BFFB1A43F001031847C4430100E443010025
:200100000A444FF0000C10F8013B13F0070408BF10F8014B1D1108BF10F8015B641E05D029
:2001200010F8016B641E01F8016BF9D113F0080F1EBF10F8014BAD1C0C1B09D16D1E58BFE3
:2001400001F801CBFAD505E014F8016B01F8016B6D1EF9D59142D6D3704700000023002476
:2001600000250026103A28BF78C1FBD8520728BF30C148BF0B6070476E2904F0F682702901
:2001800003F02483662908F09887652908F09587672908F09287612908F0918703681B0AB2
:2001A00028BF41F08001692903F09282642903F08F82752903F08C826F2904F0F18378293C
:2001C00003F0F082E92904F08983E42904F08683F52904F08383EF2904F0EE83F82903F0F5
:2001E000EF820368DB0928BF41F08001632904F0F882732904F0FD82E32905F09682F32968
:2002000005F09B82002070471FB508F0D5FE9DE8030004F0C7F904F09DF90400002000214B
:2002200007F0AEFF401C60600020002107F0BEFFE0600020002107F08DFF206104F0F4FE9E
:2002400004F072F91FBD002006F0BCFF06F0DEFF1146FFF7D9FF00F08DFE07F0F1F800003F
:2002600010B506F0D3FD1349016010BD4068C26812F0020FFBD08160704710B50446D4E955
:20028000021206F0B1FD20462169BDE8104006F0B5BD4068C16811F0140F08BF7047C168BD
:2002A00011F0040FFBD08168C16811F0140FF6D170470000C84301000648804706480047F5
:2002C000FEE7FEE7FEE7FEE7FEE7FEE7FEE7FEE7FEE7FEE7116C0000C50000000346084653
:2002E000194604F08BBA0FB4014610B504AA039804F084FA10BC5DF814FB7047FFFFFFFFF9
:2003000010F0030F09D1FE4AA2FB003252096FF018035A4310EB82021AD14FF4C872B0FBD6
:20032000F2F302FB1300002818BF002210D0F548002A084410F8010C18BF0122F24B1A703E
:2003400008BF7047022902BF401CC0B2704770470122ECE70329B4BF01230023C01AE84B0E
:2003600083FB00C34FEA631CACEBE3734FEAE07C00EB9C7C00EBAC0CACEB0303DFF88CC399
:200380000CEB810151F8041C19444FF4C87390FBF3F010440144DE4B08460022C3FB012021
:2003A0008210A2EBE070A0EBC0000844704730B583B04FF6E071D74802F034FDD64C022547
:2003C0008422C4E912522946D24801F0C7FED3A1D04806F0A8FD00218C20C4E912109622AC
:2003E000CC4801F0BBFED1A1CA4806F09CFDE06CA16C00F11602C74801F0B0FECFA1C5489F
:2004000006F091FDE06CA16C00F12202C14801F0A5FECEA1BF4806F086FDE06CA16C00F114
:200420002E02BC4801F09AFECCA1BA4806F07BFDE06CA16C00F13A02B64801F08FFECBA1B4
:20044000B44806F070FDE06CA16C00F14602B14801F084FEC9A1AF4806F065FDE06CA16C2D
:2004600000F15202AB4801F079FEC8A1A94806F05AFDE06CA16C00F15E02A64801F06EFE40
:20048000C6A1A44806F04FFDE06CA16C00F16A02A04801F063FEC5A19E4806F044FD4FF411
:2004A0007844CDE90054782391220A21994801F046FC8220CDE90004024602231A21954808
:2004C00001F03DFC03B030BD70B5934C206D01281ED04FF6FF718F4802F0A4FCE06C00F14F
:2004E0009602A06C00F120018A4801F037FE8648B2A18278874806F016FDE06C60260C304D
:20050000E064206C1B2809D000251C2808D011E04FF61F017F4802F085FCDFE7E66470BDE1
:20052000E564A06CA6A10B30A0647A4806F0FBFC1120A064206C2228F0D0232818BF2928F3
:2005400003D02C281CBF312870BDE564A06C1130A06470BD2DE9F04F9C489AB0416C01F02B
:2005600001026D498A74D0F88820069202EB82029300D0F88420079202EB820203EB420210
:20058000D3B24B72426F0492D0F880C0CDF80CC002EBCC04C26F0292D0F878C0920002EB38
:2005A0004C022244D2B2CDF814C08A721A440A66D0F860C0436DC26D0892846D920003EBCE
:2005C000CC0502EB44022A44D6B20E72C26E099202EB8202D500826E0A9202EB820205EBA3
:2005E0008202456E05EB850702EB4702D2B2CA713244CA65D0F8B0200B929600D0F8AC204F
:200600000C9206EB4206D0F8A8200D9232444A66D0F890200E92D0F89C60019602EBC60781
:20062000D0F898200092D0F89460920002EB46023A44D7B24F73D0F8A4200F9202EB8202BE
:200640004FEA8208D0F8A020109202EB820208EB4202D2B20A733A448A66D0F8C420119247
:2006600002EB82025206170E8F73D0F8B4201292D0F8C0B0CDF84CB002EBCB08D0F8BC20ED
:2006800014924FEA8209D0F8B820159209EB42024244D2B2CA733A44CA66D0F8E420169208
:2006A00002EB82021701D0F8E020179202EB820207EBC207D0F8DC20189202EB820207EB43
:2006C0008202D0F8D87007EB870802EB4802D2B20A74D0F8C8B0CDF864B0D0F8D090D0F8C3
:2006E000D480D0F8CCA04FEA890E0BEBC80B0EEB4A0EF3440BF0FF0B81F811B05A4467E02D
:200700001F85EB51DA01001064010010E801001093244992D4020010C80000102020206D83
:20072000206820642064206D207900002020312069206F20612061206F20650020203220D2
:200740006E207520742079206E20610020203420752072206520202074207200202038203C
:20076000742020202020202068202000203130206520202020202020202020002032302095
:2007800020202020202020202020200020343020202020202020202020202000203830204D
:2007A0002020202020202020202020002020502061726974792020202020200025640000B7
:2007C0002020202020202020202000004C0400100A67089A234462441A4453190A9A134494
:2007E000099A1A44036F13444B70DDE9042C02EB0C04DDE9022C624404EB020C079A944471
:20080000069A6244D0F88CC0944481F802C00E9ADDF84CB09419DDE9002632441444109AE1
:20082000D0F8E80014440F9A14440D9A14440C9A14440B9A1444129A1444159A1444149AFC
:20084000224402EB0B04119ADDF864B022445A4452444A444244D419189A1444179A1444F4
:20086000169A22441044C8700CF001020A7103F001024A7100F0010088711AB0BDE8F08FD3
:2008800000B5FFF767FEFE4908794A7910438A79104318BF012008700A6B0120632AC8BFFA
:2008A0000870CA6A0C2AC8BF0870CA7A1F2A88BF08708A69172AC8BF0870CA693B2AC8BFB9
:2008C000087004DC0878002808BF032000D00420886700BD2DE9F047E94D6869401C0026B8
:2008E000C5F884606861E748A0F11807796909687A68114214BF01220022E249002A496809
:2009000014BFC06800690160686901244FF00409142821D16E61286A401C2862E86F401CA8
:20092000E867D94806F090FAB0F1804FD8BFC5F8806007DDD44806F093FAD34806F098FAFD
:20094000C5F88040286A0228C8BFC5F88860686F012808BFC5F878904FF0020A286C3A2865
:2009600008BFC5F878A003D03B2808BFFFF788FF286A3C2804DBE969491C3C38C5E907109C
:20098000E8693C2804DBA969491C3C38C5E90610A869182807DB1838A861686A401C686290
:2009A000A86A401CA862686A0628C8BF6E622A6BEB6AD0B2D9B210F0030F0CD1DFF8CCC21D
:2009C000ACFB008C4FEA5C1C6FF018080CFB08FC10EB8C0C35D14FF4C87CB0FBFCF80CFBE3
:2009E0001800002818BF4FF0000C2AD0A848DFF8A4820844BCF1000F10F8010C18BF4FF07B
:200A0000010C88F800C003D0022904BF401CC0B2A96A8842BABF581CC5E90A4018460C28A6
:200A2000C6BF501CC5E90B4010466328C8BF2C63686906282FD007DA01280AD003283CD1BB
:200A400010E04FF0010CD1E70A282AD00C2834D12DE0796909687A68114018BF012188F831
:200A600001102AE0796909687A68114018BF012188F80210002901BF98F801100029D5F8CA
:200A80008810002918BFEE6317D1AE65EC63EE672E64AC6311E0796909687A6811420BD1D8
:200AA0000BE0796909687A68114205D105E0796909687A68114200D06C67012827D17869DB
:200AC00000687968084218BF6C630AD1686B401C6863052805DDC5F87890C5F88840C5E901
:200AE0000DA6686F012804BFD5F88000012832D1C5F87890FFF75BFCAE6305206E64C5E93F
:200B000012602E646E67EE67EE63C5F888406869032804BFA86B01281DD15F49286C98F81C
:200B2000022041F82020EA6F012A24D0022808BFAC67286C1538262838BFFFF7C5FC286C2D
:200B40003C2805DD6C67FFF732FC2E64C5E91D69A86D01281BD0A86D002818BFBDE8F08739
:200B600078690068796808421EBF6E61AC65BDE8F087BDE8F0872E64AE64EE64C1F8E86015
:200B80006E65286D01280CBF2E652C65D1E7286C401C2864BDE8F08700B58BB0002007F07E
:200BA000ECF90A900AA803F033FA03463BA22821684603F023FB372204213B4801F0CEFAFC
:200BC0004FF6FF71384802F02DF93849364801F0AAFE6946344806F0A6F95022042132485F
:200BE00001F0BCFA3149304801F09DFE2448816F03291CBF0BB000BD807C48B14FF620514A
:200C0000294802F00FF92AA1274806F08CF908E040F2FF71244802F005F928A1224806F0A5
:200C200082F92949204801F07EFE692296211E4801F094FA4CF218611B4802F0F3F8154877
:200C40002249007800EB800001EB400220A1164806F069F90BB000BD10B58CB04FF6FF7173
:200C6000114802F0DFF8002007F087F90A9019490D4801F058FE024CD4F88C003B282BE00F
:200C8000C800001034040010400500101F85EB51DA010010640100104C04001025612D2567
:200CA000642D256227257900D4020010169B000053756D6D65722054696D650057696E74F6
:200CC00065722054696D6500B2910000C601001025730000DEE0000011D10AA803F098F906
:200CE0000346FEA22821684603F088FA00220621FC4801F033FA6946FA4806F014F90AA84E
:200D000003F086F90346F8A22821684603F076FA0022AC21F34801F021FA6946F14806F010
:200D200002F90AA803F074F90346EFA22821684603F064FA684602F0E1FEC4F88C00EB4989
:200D4000E84801F0F0FD0CB010BD00B5E8488BB0016A0091C169019181690291816A039128
:200D6000C16A491E0491006B64300590684603F070F9A0F5616006F09AFF684603F069F9C6
:200D80000BB000BDDA48016C0162C16DC161016E8161416E4162816E8162C16EC162016F62
:200DA0000163704730B5D24C8BB06069002840D1F0228C21CB4801F0D1F94FF6FF71C94885
:200DC00002F030F8CB49C74801F0ADFDCAA1C548226C06F0A8F8C549C24801F0A4FDA06FE6
:200DE000032804BF206C012823D12062E16DE161226EA261636E6362A36EA362D4F86CC013
:200E0000C4F82CC0256F25638DE80F00ACF10100049005F164000590684603F01AF9A0F520
:200E2000616006F044FF684603F013F93B20C4F88C006069012808BFFFF70EFF60690428B7
:200E400045D1AF4DD4F89410A87888420ED073220621A44801F082F940F2FF71A14801F0B8
:200E6000E1FFAA78A7A19F4806F05DF8A878C4F89400A06B98B9D4F8980040B373223C21E1
:200E8000984801F06BF94FF47841964801F0CAFF9FA1944806F047F8A06BC4F89800A06BCE
:200EA000012814D1D4F89800012810D073223C218C4801F053F94FF4FC618A4801F0B2FFA0
:200EC00096A1884806F02FF8A06BC4F898006069052807D1D4F88C0001281CBF0BB030BDBD
:200EE000FFF75AFE60690A281CBF0BB030BDA06F20B94FF6FF717B4801F094FFA06F01280A
:200F000004D140F2FF71774801F08CFFA06F022803D11F21734801F085FFA06F032804D193
:200F20004FF4FC616F4801F07DFFA06F042804D14FF478416B4801F075FF4FF496723C2121
:200F4000684801F00BF9D4F89010A06F88420CD06649644801F0E7FCA06F734900EBC00026
:200F600001EB40015F4805F0DEFFA06FC4F890000BB030BD00215B4801F056FF594801F02C
:200F800058F90021574800F0EAFA564801F051F96649544801F0C7FC0A220021514801F0BD
:200FA000DDF80F214F4801F03DFF61A14D4805F0BAFF4FF478714B4801F034FF5EA14948B0
:200FC00005F0B1FF40F2EF31464801F02BFF5DA1444805F0A8FF4FF4F041424801F022FF3B
:200FE0005BA1404805F09FFF47F60F013D4801F019FF59A13B4805F096FF47F6E031394829
:2010000001F010FF56A1374805F08DFF4CF21861344801F007FF54A1324805F084FF47F68B
:20102000EF31304801F0FEFE52A12E4805F07BFF4FF478412B4801F0F5FE51A1294805F0A8
:2010400072FF4FF4FC61274801F0ECFE4EA1254805F069FF1F21234801F0E4FE4CA12148A8
:2010600005F061FF4FF6E0711E4801F0DBFE4AA11C4805F058FF4FF61F011A4801F0D2FE32
:2010800047A1184805F04FFF40F2FF71154801F0C9FE46A1134805F046FF4FF62051114883
:2010A00001F0C0FE43A10F4805F03DFF4AF6E5710C4801F0B7FE41A10A4805F034FF42489F
:2010C00007F028F8074801F0B4F80849054801F02AFC3E4807F01EF8024879E025483A2556
:2010E0004D2E0000D402001025530000B2910000C80000107AB600002530326400000000E1
:2011000064010010426974202564202000000000204E6F2053796E632000000020496E20A1
:2011200053796E63200000006C010010169B00006E6176790A0000004461726B47726565F7
:201140006E0A00004461726B4379616E0A0000004D61726F6F6E0A00507572706C650A0008
:201160004F6C6976650A00004C69676874477265790A00004461726B477265790A000000AA
:201180005265642000000000477265656E200000426C75650A00000059656C6C6F770A00EB
:2011A0004D6167656E74610A000000004379616E202000004F72616E67650A0047726565B4
:2011C0006E59656C6C6F770000004040CDCC4C3E01F02FF84C4C01252565FFF7E8F8002626
:2011E0002664A663E6636565C4F89050C4F88850A6673B20C4F89850C4F88C00E1228C2115
:20120000424800F0ABFF4FF6FF71404801F00AFE3F493E4801F087FB3EA13C48226C05F00D
:2012200082FE4FF496720621384800F097FF4FF6FF71364801F0F6FD3549344801F073FB46
:2012400037A1324805F06FFE374805F011FEFFF703FDFFF7A1FC354841690968406801424B
:201260001CBF6661A565324EAFF697114CF2503706F1140005F090FD3946304605F090FE2B
:20128000D4F884000028FBD1FFF78CFDC4F88450F6E700B5284883B026A1CDE90001431EE7
:2012A000421C811C194800F010FB244A244905F071FF2548154A23490090CDE90112431CA7
:2012C000821CC11C214801F061FE18482049002206F049F91F482049012206F044F9124837
:2012E00005F0DFFD124805F031FD1C4940F8141B002105F055FD03B01438104A18495DF85D
:2013000004EB05F047BF0000C8000010D4020010B2910000444346205365636F6E64730026
:201320005374617475733A00400500101C0400104C0500105446540010C009200000000022
:20134000377100004DC0092006C009207803001045C009203404001032C0092064440100FB
:20136000DB6F000010B501F0F7FC04466F482060743060604FF6FF71204601F053FD002118
:20138000204601F051FD204610BDDDF800C08184C28401851944491E418502EB0C01828584
:2013A000491EC185704710B50B460446B0F92620B0F924100068D0F84CC02046E047A08CA8
:2013C000401C00B2A084B4F92A108842D8BF10BD208DA084E08C401C00B2E084B4F92E102C
:2013E0008842C4BFA08DE08410BD30B50446006883B0416D2046884705462068016D2046EE
:201400008847E18B0346CDE90051216800222046D1F860C01146E04703B030BD2DE9F843D8
:201420000646DDE90857009500689846D0F858C03046E047002408FB05F5002DD8BFBDE859
:20144000F88330683946C26D30469047641CA542F7DCBDE8F8832DE9F8430546DDE9086753
:20146000009600689846D0F858C02846E047002408FB06F6002ED8BFBDE8F88357F8241090
:201480002868C26D28469047641CA642F6DCBDE8F8832DE9F8430546DDE90867009600681F
:2014A0009846D0F858C02846E047002408FB06F6002ED8BFBDE8F88307EBE40004F00701FF
:2014C0000078884010F0800F14BFA98BE98B2868C26D28469047641CA642EDDCBDE8F8836D
:2014E000DFF84CC000B50CEBC30383B0F83B4FF0080CCDE900C30368D200C900D3F868C06C
:201500000823E04703B000BD10B50168096D8847C11700EB5170C01010BD10B50168496D91
:201520008847C11700EB5170C01010BDC0420100A232010038B504460068416D2046884761
:2015400005462068016D204688470095216803460022D1F858C011462046E04738BD01636E
:20156000E8E770B504460D0A5430CEB2416800690160722104F1400005F016FC294604F16C
:20158000400005F011FC314604F1400005F00CFC206EA16D016070BD70B5044654300D46F0
:2015A000416800690160702104F1400005F0FCFB002104F1400005F0F7FB294604F1400025
:2015C00005F0F2FB206EA16D016070BD70B505461446FFF7E1FF21462846BDE87040C0E78E
:2015E00070B5044603220821403005F0FDFBFE4904F1400005F002FC00210D462046FFF792
:20160000CBFF29462046FFF7ACFF01210D022046FFF7C2FF29462046FFF7A3FF02214FF469
:20162000E0652046FFF7B8FF29462046FFF799FF032141F230052046FFF7AEFF2946204685
:20164000FFF78FFF042100252046FFF7A5FF29462046FFF786FF082140F202252046FFF78E
:201660009BFF29462046FFF77CFF092100252046FFF792FF29462046FFF773FF0A21204680
:20168000FFF78AFF29462046FFF76BFF0C2101252046FFF781FF29462046FFF762FF0D210D
:2016A00000252046FFF778FF29462046FFF759FF0F212046FFF770FF29462046FFF751FFF9
:2016C000322006F037FD072140F201152046FFF763FF29462046FFF744FF322006F02AFDE3
:2016E00010214FF486552046FFF756FF29462046FFF737FF112107252046FFF74DFF294674
:201700002046FFF72EFF12214FF488752046FFF743FF29462046FFF724FF13214FF4306535
:201720002046FFF739FF29462046FFF71AFF292100252046FFF730FF29462046FFF711FF5C
:201740002B2144F210052046FFF726FF29462046FFF707FF502100252046FFF71DFF294623
:201760002046FFF7FEFE5121EF252046FFF714FF29462046FFF7F5FE522100252046FFF76A
:201780000BFF29462046FFF7ECFE532140F23F152046FFF701FF29462046FFF7E2FE322037
:2017A00006F0C8FC60214FF41C552046FFF7F4FE29462046FFF7D5FE612101252046FFF74A
:2017C000EBFE29462046FFF7CCFE6A2100252046FFF7E2FE29462046FFF7C3FE802120460C
:2017E000FFF7DAFE29462046FFF7BBFE81212046FFF7D2FE29462046FFF7B3FE8221204644
:20180000FFF7CAFE29462046FFF7ABFE83212046FFF7C2FE29462046FFF7A3FE842120465F
:20182000FFF7BAFE29462046FFF79BFE85212046FFF7B2FE29462046FFF793FE90211025A2
:201840002046FFF7A9FE29462046FFF78AFE922100252046FFF7A0FE29462046FFF781FE16
:20186000932101252046FFF797FE29462046FFF778FE95214FF488752046FFF78DFE294610
:201880002046FFF76EFE972100252046FFF784FE29462046FFF765FE98212046FFF77CFE08
:2018A00029462046FFF75DFE072140F233152046FFF772FE29462046FFF753FE642006F0FE
:2018C00039FC2046BDE8704034E62DE9F0410C46DDE9065116461F46FFF744FD4349016063
:2018E000743141603B46324621464030FEF7B8FCA0F1400414300122294605F034FE3C49D2
:2019000021673C494FF47A72002509686563B1FBF2F12046C4F89C10FFF762FE204625638C
:20192000FFF708FE84F83C502046C4F8A050BDE8F081006B002816BF0228F0204FF4A07086
:201940007047006B002816BF02284FF4A070F02070472DE9F0410446006B0D461F46164614
:2019600040B1012819D040F23F1802282AD003285DD148E02021ADB22046FFF70DFE2946C0
:201980002046FFF7EEFD2121B5B22046FFF704FE29462046FFF7E5FD49E0C2F1EF0220213E
:2019A00096B22046FFF7F8FD31462046FFF7D9FD2121ADB22046FFF7EFFD29462046FFF731
:2019C000D0FD34E0C5F1EF0085B220212046FFF7E3FD29462046FFF7C4FDA8EB060085B271
:2019E0002121204608E00000006CDC0244430100F11FFF1F94020010FFF7CEFD294620461B
:201A0000FFF7AFFD13E0202196B22046FFF7C4FD31462046FFF7A5FDA8EB050085B2212105
:201A20002046FFF7B9FD29462046FFF79AFD22212046FFF7B1FDB9B22046BDE8F04190E5C9
:201A40007221403005F0B0B970B5016B89B101291AD0022923D0032918BF70BD044603218A
:201A600041F29805FFF798FD29462046BDE8704077E50446032141F2B005FFF78DFD294640
:201A80002046BDE870406CE50446032141F2A805FFF782FD29462046BDE8704061E50446BD
:201AA00003214FF48455FFF777FD29462046BDE8704056E52DE9F84F8846A2EB0806044607
:201AC0009946002506F1010A0A9FFFF7BDFF01200090206853464A46D0F858C04146204676
:201AE000E04722212046FFF757FD606EA16D0160722104F1400005F057F90322102104F137
:201B0000400005F071F9002E07D9394604F14000FEF7ACFB6D1CAE42F7D804F14000FEF756
:201B2000B8FB0322082104F1400005F05DF9206EA16D0160BDE8F88F2DE9F84F9146A3EB39
:201B4000090604468A46002506F101080A9FFFF77BFFCDF80080206801234A46D0F858C0BD
:201B600051462046E04722212046FFF715FD606EA16D0160722104F1400005F015F9032263
:201B8000102104F1400005F02FF9002E07D9394604F14000FEF76AFB6D1CAE42F7D804F169
:201BA0004000FEF776FB0322082104F1400005F01BF9206EA16D0160BDE8F88F2DE9FF4F66
:201BC00081B00C4607461546032141F23006DDF838B0FFF7E1FC31463846FFF7C2FC384696
:201BE000FFF7A8FC0498ABEB0501001B0028C8BF4FF00108B8BF4FF0FF382CD00029C8BF68
:201C00004FF00109B8BF4FF0FF393AD008FB00F009FB01F14FEA40024FEA410A0092814246
:201C200045DCAAEB00060498844218BFAAEB020B54D038682A462146D0F84CC038460F9B76
:201C4000E0474444002EB2BF56445E444D4404988442EED142E00F98AB45009008DD5B4679
:201C60002A4621463846FFF767FF05B0BDE8F08F2B465A4621463846FFF75EFF05B0BDE837
:201C8000F08F04982B46A0420F98009007DD21463846049AFFF70EFF05B0BDE8F08F2246F4
:201CA00038460499FFF706FF05B0BDE8F08F561A5D4518BFA2EB0A0A10D038682A46214654
:201CC000D0F84CC038460F9BE0474D44002EB9BF00980644564444445D45EED138680F9BFB
:201CE0002A46D0F84CC005B021463846BDE8F04F60472DE9F84301EB0309DDE908541646B4
:201D0000134680460F464A460094FFF7D3FE35442B463246394640460094FFF70DFF2B46F6
:201D20004A46394640460094FFF7C4FE2B463246494640460094FFF7FFFEBDE8F8832DE907
:201D4000F84F0446DDE90A58894692461F1E4FF00006BCBF01EB07095F42002DBCBF02EBF4
:201D6000050A6D42FFF770FE009520683B465246D0F858C049462046E04722212046FFF770
:201D80000BFC606EA16D0160722104F1400005F00BF80322102104F1400005F025F87D43E2
:201DA000002D07D9414604F14000FEF75FFA761CB542F7D804F14000FEF76BFA03220821D7
:201DC00004F1400005F010F8206EA16D0160BDE8F88F2DE9FF4F89B08B468146032141F21C
:201DE0003005169CFFF7D8FB29464846FFF7B9FB4846FFF79FFB0C980C9900FB00FA01EB44
:201E0000D17222F00102891A4FEAEA7204FB04F00AEB927201EBA20101444942039104EB64
:201E2000D471009021F00101C217611A00EB927001EBA00000EB0A0149424042CDE9041020
:201E4000CAF1000000FB04F600980025400000270AFB04F1019049004FEA4A00C1F100089D
:201E6000029055E00B980BEB05010219CDE90621D9F80000179BD0F84CC04846E04755EAB9
:201E800004000AD00B98ABEB0501021BD9F80000179BD0F84CC04846E047002D18BF002CCC
:201EA00013D00B98179B021BD9F800000799D0F84CC04846E047D9F80000ABEB0501179BB4
:201EC000D0F84CC04846069AE047009800FB05610398814204DD0AFB04610598814204DCF7
:201EE00001986D1C07443E4412E00AFB14610498814204DD0298641E8044464408E001985C
:201F000002990744F0196D1C8844641E00EB0806002CA4BF0C98A842A4DA0DB0BDE8F08F86
:201F20002DE9FF4F8FB00120DDE91C89924605460290129A129802EBD273404323F001039B
:201F4000D21A44460490C31708FB04F100EB937002EBA000084440420B9004EBD4700A91F3
:201F600020F00100CA17201A01EB927100EBA10104980026084440420C9048420D900498CA
:201F80000A99404200FB08F700204900089004985FEA080400FB04F04FEA4000C0F1000017
:201FA000099106900498B3464FEA400007904FF0010066D1CDE900091299524600EB4103A4
:201FC0001098411A0F98FFF7BAFE13B0BDE8F08F0A9800FB0B710B98814205DD049800FBCA
:201FE00008710D9881423EDC012D30D06800811E012000EB440088421BD9681ECDE900095E
:202000001098AAEB0402801B05900146029B0F98FFF795FEC5F10100CDE900090AEB0400CA
:20202000421C029B05990F98FFF789FE601B441C0CE06000401CCDE900091098AAEB04025E
:20204000811B029B0F98FFF77AFE00240125DDE908010844074408900298761C801C0BF126
:20206000010B02900DE0049800FB18710C98814228DDDDE906010844A8F1010807446D1CBA
:202080000690B8F1000FA4BF12985845A0DAAC4255D9CDE900591098AAEB0402861B314648
:2020A000029B0F98FFF74BFE6842CDE900090AEB0400421C3146029B0F98FFF740FE13B02B
:2020C000BDE8F08F012000EB4400B0EB450F15D9CDE900591098AAEB0402801B03900146E8
:2020E000029B0F98FFF72BFE6842CDE900090AEB0400DDE90231421C0F9809E06000401C78
:20210000CDE900091098AAEB0402811B029B0F98FFF715FEDDE908010844DDE90612089043
:202120003844114447180298761C801C641B0BF1010BA8F10108069101250290A1E7600047
:20214000401CCDE900091098AAEB0402811B029B0F98FFF7F4FD13B0BDE8F08FC0E90D12AB
:2021600070472DE9F8430646DDE908940D4690461F46FFF769FCCDF8009030683B464246CA
:20218000D0F858C029463046E04722213046FFF703FA706EB16D0160722106F1400004F08C
:2021A00003FE0322102106F1400004F01DFEA9F10100784304EB40044FF00008B9F1000FF9
:2021C00011D90025002F08D9218806F14000FEF74DF8A41C6D1CAF42F6D808F10108A4EB2D
:2021E0008704C845EDD306F14000FEF752F80322082106F1400004F0F7FD306EB16D016087
:20220000BDE8F88370B50D46164604462021FFF7C3F929462046FFF7A4F9254621213446FE
:202220002846FFF7B9F921462846BDE87040FFF798B9F0B5044690F83C0083B000B3256BEE
:20224000D4F8A01020462163FFF774F92068416D2046884706462068016D20468847FE498C
:2022600003460022496E2046CDE900611146FFF778FF256303B02046BDE8F040FFF75AB97C
:202280000025032141F230062046FFF785F931462046FFF766F92046FFF74CF900273E4634
:2022A00020212046FFF778F939462046FFF759F921212046FFF770F931462046FFF751F9BF
:2022C00022212046FFF768F9606EA16D0160722104F1400004F068FD0322102104F1400015
:2022E00004F082FD2068016D2046884706462068416D204688474643002E07D9E18B04F191
:202300004000FDF7B3FF6D1CAE42F7D804F14000FDF7BFFF0322082104F1400004F064FDD0
:20232000206EA16D016003B0F0BD70B504465430416800690160702104F1400004F034FDEF
:20234000002104F1400004F02FFD002104F1400004F02AFD206EA16D0160C04904F140005B
:2023600004F04CFD606EA16D0160732104F1400004F01AFD002104F1400004F015FD002192
:2023800004F1400004F010FD0502002104F1400004F00AFD284385B2206EA16D0160B04917
:2023A00004F1400004F02AFD284670BD10B504460068016D20468847E16E497890FBF1F09C
:2023C00010BD10B504460068416D20468847E16E897890FBF1F010BD70B504460068A26B69
:2023E0000D460A2907D0D0F82CC0616B2B462046E047284670BD00266663E16E89781144D3
:20240000A163416D20468847E16E8978401AA16B884298BFA663ECE72DE9FF4F0446A3F1E0
:202420001F0087B088461D46612824BF0BB0BDE8F08FE06E06784178019181780491C078ED
:2024400003902068016D20468847626B01991144884210D200276763A16B04980844A0636E
:202460002068416D20468847E16E8978401AA16B814228BFA7632046FFF7E6FAE06EA5F167
:20248000200101FB0600001D029000780590049800902068D4E90D12D0F858C02046019BEB
:2024A000E04722212046FFF777F8606EA16D0160722104F1400004F077FC0322102104F130
:2024C000400004F091FC04984FF00009002827D90198002600281ED9C9F3C400401C0090E5
:2024E00009F00700012101FA00F00690099800EB0907DDE9020101FB06010098095C069836
:2025000001422BD0A18B04F14000FDF7AFFE0198761C8642EDD3049809F101098145D7D3B8
:2025200004F14000FDF7B5FE0322082104F1400004F05AFC206EA16D016005980199801C22
:202540008842616B3FBF084460630BB0BDE8F08F0198084460630BB0BDE8F08F94F83C00AA
:2025600078B13D48D4F8A010456E206B401A10F003000CD001281AD0022831D0032841D040
:202580004AE0E18B04F14000FDF770FEBFE72068016D2046884782462068416D204688470A
:2025A000C01B401E08EB06010AFB001032E02068416D2046884782462068416D2046884723
:2025C00083462068016D2046884708EB0601401A401E0BFB00A0C01B05EB4000851E1BE006
:2025E0002068016D2046884782462068016D2046884700FB07A008EB0601401A05EB400097
:20260000851E09E02068416D2046884708EB060100FB017005EB400504F140002988FDF74E
:2026200025FE74E72DE9F04F054688468FB010464FF0010A0BA101F090FB040014D0034676
:2026400036220121684603F088FA9DF800004FF0FF3B422812D015E01802001080969800B6
:20266000006CDC02726200000021C5F8108085E8C202C5E905510FB0BDE8F08F9DF8010020
:202680004D280ED0204601F099FB2846C5F800B0C0E90554C0E90167C5E903980FB0BDE861
:2026A000F08F9DF81C009DF81D1000EB0120102808BF102712D0182808BF18270ED020467A
:2026C00001F07CFB2846C5F81080C0E905546FF00101A0E8C2020FB0BDE8F08F9DF816009A
:2026E0009DF817109DF8192000EB01209DF81810090401EB026100EB01099DF812009DF8FA
:2027000013109DF8152000EB01209DF81410090401EB02614618D8F80000416D404688477A
:20272000484506DBD8F80000016D40468847B04210DA204601F042FB2846C5F80890C0E9BC
:2027400005546FF00201C0E90016C5E903780FB0BDE8F08F9DF80A009DF80B109DF80D20E2
:2027600000EB01209DF80C10090401EB0261014406FB07F0C21700EB52700BF1010B0BEB7F
:20278000E00212F0030FF8D1C5F800A0C5E90514C5E90169C5E9037B0FB0BDE8F08F2DE919
:2027A000F04788B08A4690461D460446FFF74CF92A46214601A8FFF735FF019801281CBFD5
:2027C00008B0BDE8F0870498C11700EB51700299C010484300F0E6FE07462068416D204652
:2027E000884703994044884207D32068016D2046884702995044814204D908B06FF0020033
:20280000BDE8F087002F02BF6FF0030008B0BDE8F0870398461E002EA8BF4FF0010975DB49
:20282000049902984843C21700EB52700599002201EBE000069906FB0011079801F09EF9EC
:2028400004990298079B4843C11700EB5170C2100121384603F081F90498182816D1029953
:202860000020002912DD00EB4001CA19795C93785278DB08DB02920843EA421343EAD1028B
:2028800027F810200299401C8142ECDCDDE902304044801BCDF80090421E20685146D0F8B4
:2028A00058C02046E04722212046FEF775FE606EA16D0160722104F1400004F075FA0322D5
:2028C000102104F1400004F08FFA04F14000FDF7D4FC02980025002809DD37F8151004F106
:2028E0004000FDF7C3FC02986D1CA842F5DC04F14000FDF7CEFC0322082104F1400004F09D
:2029000073FA206EA16D0160761E89D5384600F078FE079801F052FA2046FEF70BFE08B07F
:202920000120BDE8F087C166704780F83C1070472DE9F04F87B00C460646FFF785F82246FC
:2029400031466846FFF76EFE009801281CBF07B0BDE8F08F0398C11700EB51700199C010F0
:20296000484300F01FFE80464FF4807000F01AFE82463068416D304688470299884206D12F
:202980003068016D304688470199884204D007B06FF00200BDE8F08FB8F1000F0DD0BAF138
:2029A000000F0AD0002425461D22192106F1700000F092FA082805D010E007B06FF0030035
:2029C000BDE8F08F1D22192106F1700000F0A0FA1D22192106F1700000F08BFA02984FF03B
:2029E00000090028C8BFDFF848B376DD039901984843C21700EB52700499002201EBE00029
:202A0000059909FB0011069801F0B8F803990198069B4843C11700EB5170C2100121404665
:202A200003F09BF80398182818D101990020002914DD00EB400101EB080218F8011093782A
:202A40005278DB08DB02920843EA421343EAD10228F810200199401C8142EADC0198002741
:202A600000281FDD38F817002AF81400641C802C14D11D22192106F1700000F049FADBF8BE
:202A80006400630000EB0522514606F1700000F04CFA00246D1CB5F57A7F2ED001987F1CA7
:202AA000B842DFDC029809F1010948459EDCA4B11D22192106F1700000F02AFADBF864003C
:202AC0004FF4807300EB0522514606F1700000F02CFA681CB0F57A7F0FD0404600F091FD95
:202AE000069801F06BF9012086F83C00306BC6F8A00007B00120BDE8F08F8EA19348FDF715
:202B0000F2FB012004F09CFC2DE9F04704460D460898194410444F1EA0F10108164620213C
:202B20001FFA85F92046FEF737FD49462046FEF718FD21211FFA86F92046FEF72DFD494682
:202B40002046FEF70EFD206B002835D001285AD040F23F1902287DD0032818BFBDE8F087E5
:202B60005021B6B22046FEF717FD31462046FEF7F8FC51211FFA88F62046FEF70DFD314662
:202B80002046FEF7EEFCA9EB070086B252212046FEF702FD31462046FEF7E3FC2646A9EB9F
:202BA0000502532194B23046FEF7F6FC21463046BDE8F047FEF7D5BC5021ADB22046FEF78D
:202BC000EBFC29462046FEF7CCFC5121BDB22046FEF7E2FC29462046FEF7C3FC5221B5B2FF
:202BE0002046FEF7D9FC29462046FEF7BAFC53211FFA88F52046FEF7CFFC29462046BDE87B
:202C0000F047FEF7AEBCC8F1EF001FFA80F850212046FEF7C1FC41462046FEF7A2FCC6F125
:202C2000EF02512196B22046FEF7B6FC31462046FEF797FC5221ADB22046FEF7ADFC294632
:202C40002046FEF78EFC5321BDB22046FEF7A4FC294600E004E02046BDE8F047FEF781BC0A
:202C6000C7F1EF0087B250212046FEF795FC39462046FEF776FCC5F1EF0085B25121204617
:202C8000FEF78AFC29462046FEF76BFCA9EB080085B252212046FEF77FFC29462046FEF7A2
:202CA00060FCA9EB0602532195B22046FEF774FC29462046BDE8F047FEF753BC70B5044672
:202CC0005430416800690160214904F1400004F095F8732104F1400004F066F8002104F1AC
:202CE000400004F061F8002104F1400004F05CF8002104F1400004F057F80502002104F1F3
:202D0000400004F051F8284385B2206EA16D0160104904F1400004F071F8284670BD10B54C
:202D20000446FEF739FC2046BDE81040C6E7000018020010546F6F206D616E7920666C6193
:202D40007368777269746573000000005C06001080969800006CDC0270B50D4604F0F2F83A
:202D600004464C48206054300023606063832383002D08BF23620AD0284601F045F8801C77
:202D800004F0DBF92A4644A1206200F061FC204670BD10B50446006A98B10A463FA100F0D2
:202DA0008DFF002808BF10BD2068416B2046884703464FF400720021394800F05BFF012057
:202DC00010BD38493848FDF78EFA002010BD70B50446006800221146036C20469847206830
:202DE0000025416B2046884706462068016B2046884770430028D8BF70BD2021204604F01E
:202E000058F820686D1C416B2046884706462068016B204688477043A842EEDC70BD0183E3
:202E20004283704781837047C183704770B5044600680025628B0E460A291DD0D0F82CC04F
:202E4000218B33462046E047208B401C20832068426B20469047218B88420BDC2583608BB4
:202E6000401C60832068016B20468847618B884200DC6583304670BD2583511C6183026B67
:202E800020469047618B8842F4DCF2E74FF0FF30704700005C4201002F2573007700000094
:202EA0000C060010AC3501005C06001010B5044636206060226804F11801201D9047E06982
:202EC00010BD10B504463A206060226804F11801201D9047E06910BD10B504463520E26094
:202EE000C4E90101226804F11801201D9047A06910BD10B504463420E260C4E90101E06A03
:202F00002061226804F11801201D9047A06910BD10B504463220E260C4E90101226804F1DD
:202F20001801201D9047A06910BD10B504463320C4E90102C4E90313E06A6061226804F12F
:202F40001801201D9047A06910BD10B504463820C4E90102C4E90313226804F11801201DBF
:202F60009047A06910BD10B50446372060600020E061226804F11801201D9047E06910BD5B
:202F80004FF4B02070474FF42030704770B5DDE90465DDF818C0C0F810C0143003F036FF28
:202FA000A0F1140414300122314604F0DCFA04F140000022294604F0D6FA2D206067A0671B
:202FC0004FF48772BE21E067C4E92021C4E92210C4F89000C4F89400C4E92621C4F8A010C6
:202FE000606BE16A0160FE4904F1140003F006FF0022082104F1140003F0F6FE204670BD44
:203000002DE9F04104460D4616461F46006941F230020321FEF7DAFA2069FEF78BFA2069C4
:203020003B4632460168D1F84CC02946E04720693B4632460168D1F84CC0691CE0472069CE
:203040003B46721C0168D1F84CC02946E0472069721C3B460168D1F84CC0691CBDE8F0415C
:20306000604770B5044628300D46426800690260012005F064F8294604F1140003F094FEAB
:20308000012005F05CF8002104F1140003F08CFEC5B2012005F053F8002104F1140003F02A
:2030A00083FEC1B2606BE26A026041EA0520C0F3CB00800870BD2DE9F0410C4616460746DE
:2030C000D021FFF7CEFF0546012005F038F890213846FFF7C6FF25603060BDE8F0812DE980
:2030E000F04192B006460D4600244821684600F027FF002D08BF06F10805E846D0213046E0
:20310000FFF7AFFF0746012005F019F890213046FFF7A7FF08EB840148F824704862601C62
:20312000C4B2706D0068716C084201D1092CE5D3092C03D012B00020BDE8F081DDE9000127
:2031400008440299A74E084486FB0010DDE903121144059AA0EBE070114486FB0121A1EB88
:20316000E172DDE906131944089B194486FB0131A1EBE171831A541AA1EB000C002BD8BFCA
:203180005B42002CD8BF6442BCF1000FD8BFCCF1000C022BC4BF022CBCF1020FCADC9C42ED
:2031A00007DD9C4507DB104400EBD070401028600CE0644505DD084400EBD070401028604B
:2031C00004E0501800EBD07040102860DDE9090108440B99084486FB0010DDE90C121144CA
:2031E0000E9AA0EBE070114486FB0121A1EBE172DDE90F131944119B194486FB0131A1EBE8
:20320000E171831A541AA1EB000C002BD8BF5B42002CD8BF6442BCF1000FD8BFCCF1000CD5
:20322000022BC4BF022CBCF1020F83DC9C4207DD9C4507DB104400EBD070401068600CE08B
:20324000644505DD084400EBD0704010686004E0501800EBD0704010686012B00120BDE83D
:20326000F0812DE9F003D2F810C01468D668A4EB0C0554690020361B75439668ACEB060C53
:203280005668341B0CFB045CC3F818C0BCF1000F02BF0120BDE8F0037047D1F810C00C682D
:2032A000D668A4EB0C055469361B75438E68ACEB060C5668341B0CFB045CC3F800C0D2F812
:2032C00010C014688E68A4EB0C050C69361B75430E68A41B9668A6EB0C0C04FB0C5CC3F890
:2032E00004C0D2F810C08C6895680E690CFB04F705FB1677D2F8048007FB08F8176807FBA8
:2033000006F90E680CFB169C7543D2F80C9007FB14540CFB098C556904FB05CCC3F808C04A
:20332000D1F814C04C68D668A4EB0C055469361B7543CE68ACEB060C5668341B0CFB045C45
:20334000C3F80CC0D2F810C01468CE68A4EB0C054C69361B75434E68A41B9668A6EB0C0C20
:2033600004FB0C5CC3F810C0D2F810C0CC6895684E690CFB04F705FB1677D2F8048049684B
:2033800007FB08F817687E430CFB116CD66869430CFB068C07FB1411526901FB02C1596189
:2033A000BDE8F00370472DE9F04383B04FF6FF78CDE9002806460C468B1E154600690F3955
:2033C000FEF7FCFBCDE9005804F10F032A46A11C3069FEF7F3FBA81ECDE90008234603E073
:2033E00020A1070056555555A5F10F0219463069FEF7E4FB05F10F07CDE900782346AA1CD4
:2034000019463069FEF7DAFB47F6EF38CDE90078E31F3A46A4F10F013069FEF7CFFBCDE923
:203420000078A4F10F03EA1D19463069FEF7C6FBA5F10F09CDE90098E31F4A46A4F10F0185
:203440003069FEF7BBFBCDE90098A4F10F03EA1F19463069FEF7B2FBCDE9007804F10F035B
:203460003A46E11D3069FEF7A9FBCDE9007804F10F03EA1D19463069FEF7A0FBCDE900988A
:2034800004F10F034A46E11D3069FEF797FBE81FCDE9000804F10F034A4619463069FEF72E
:2034A0008DFB03B0BDE8F08370B582B0044600F1580300F18C0200F17401FFF7D2FE3049A8
:2034C0002069FFF730FA002520690168C96B884720690A2201680B6C1146984729A120690B
:2034E00003F021FD4FF4FA7004F024FE04EBC5062046D6E91D12FFF756FF69462046FFF794
:20350000EEFD0028F9D00098C6F88C000198C6F89000681CC5B2032DD6D304F1580304F1ED
:203520008C0204F174012046FFF79BFE20690168C96B884702B070BD30B4016F4FF0000C2B
:20354000002908BF4FF0010C16D0836D8268C56D03FB02F4C36805FB0344056E2C4494FB65
:20356000F1F40460446E6243846E04FB0322C36E1A4492FBF1F1416030BC604670470000AD
:2035800002360100546F7563682063726F73736861697220746F2063616C69627261746537
:2035A0000000000070B5064600F0D0FF056806F10B0020F00704B4429CBF002070BD2B4642
:2035C0006A68BAB11068A04210D304F1080188423CBF5068586007D3516810194160116868
:2035E000091B016058601460101D70BD13465268002AE7D12146284600F0C0FF0028DED170
:2036000070BD70B50446051F00F0A0FF0068002C14BF446870BD002C18BFA54284BF204688
:203620006468F8D801680A18AA4218BF456003D12A6805461144016028684119A1421CBFEC
:203640006C6070BD6168696021680844286070BD0FB41CB5084B06AA7B4469460090059823
:2036600001F09DF804460020694601F0ABF820461CBC5DF814FB00006911000070B505468B
:203680000C46012A05D02868800600D5EA69002302E0012305E05B1C934202D2E05C002808
:2036A000F9D1A869E618C01AA861286A18442862284600F0C3FF04E0D5E9012114F8010BDA
:2036C0009047B442F8D3284600F0CFFF70BD00002DE9F0410746002510687529394616A4F1
:2036E00011D000F0D4FF002803DAC0F1000013A407E039688A0701D511A402E0490704D50A
:2037000010A4012501E000F0CBFF00210A2307F1240607E0B0FBF3F203FB12003030705419
:203720001046491C0028F5D12B4622463846BDE8F04100F0BEBF0000000000002D00000019
:203740002B00000020000000F0B40F460168090502D5234C7C4402E0214C7C440E34002136
:2037600000F124050BE002F00F064FEA1212A65D42EA03724FEA13136E5401F1010152EAEB
:203780000306F0D1224604680023240704D5702F05D009B111320223F0BC00F08ABF1032A7
:2037A0000123F9E770B504460D462146106800F077FF024629462046BDE870400023C3E7BF
:2037C000D21D22F00703D3E90023BDE70368126843F0200303600823C3610023B4E70000B0
:2037E000F00901002DE9F05F044689464FF0000ADFF878B1FB44C0F820A02046E1688847D3
:20380000002875D0252806D0D4E901219047206A401C2062F1E700265F462046E1688847D9
:203820002028054608DB312D06D207EB050010F8200C08B10643F0E7B00701D526F004062B
:20384000C4F81CA00027C4F818A02A2D09D0284603F0E4FC38B304EB8708303DC8F81850E6
:2038600019E059F8041B204604EB87029161E1688847012F054618D1E069002820DA26F012
:2038800020061DE0D8F8180000EB800005EB40003038C8F818002046E1688847054603F086
:2038A000BDFC0028EED1012F0AD02E2D08D12046E16888477F1C0546022F46F02006C4DB9A
:2038C000A069002803DA404246F00106A061F00701D026F010066C2D0BD0682D09D04C2DCB
:2038E00039D06A2D35D0742D35D07A2D33D016E038E0E1682F4620468847B842054609D1B3
:203900006C2F26D04FF48060E168064320468847054604E06C2F1AD04FF4807006430DB33C
:20392000A5F14100192802D8203546F400664A462946204626604E46FCF71EFC80B10128BA
:203940000BD0F61D26F0070000F1080955E74020E4E78020D8E70020D6E706F104094CE780
:20396000284651E7206ABDE8F09F0000780901000FB400B58DB010A9099000910B904FF0EF
:20398000FF300A9000200C90064878440690064878446A4607900F9909A801F02BF80DB087
:2039A0005DF814FB8B100000A31000002DE9FF5F1D464FF0FF3B91464FF000085F46D5E984
:2039C0000146A96901987F1C8847296A824688470028F6D11AF101000CD0002E24F4C06420
:2039E00019DD600614D5BAF12B0F09D0BAF12D0F0ED103E0584604B0BDE8F09F44F4806479
:203A0000A96901987F1C8847761E8246002E02DDBAF1300F03D0B9F1000F26D032E0A96998
:203A2000761E01987F1C44F400748847002E824605DDBAF1780F06D0BAF1580F03D0B9F1D4
:203A4000000F10D01EE0B9F1000F02D0B9F1100F18D1A969761E01987F1C24F40074884707
:203A60008246102002E0082000E00A20814609E0A96908FB0908761E01987F1C44F40074F0
:203A800088478246002E05DD4946504600F09EFF0028EDDAE96901988847A00502D46FF04A
:203AA0000100A8E7E00727D1600614D5600502D5C8F1000000E04046296801F104022A60DA
:203AC0000968220501D5087016E0220701D5088012E0086010E0286800F1040129600068C2
:203AE000210502D580F8008006E0210702D5A0F8008001E0C0F8008038467CE770B5064669
:203B000000F034FD0468054630460A22002100F0A3FF2C6070BD000070B50446C0688107A0
:203B200013D0800601D5A56A04E0A169606808442169451A204601F033FA002206462946EB
:203B4000204600F01BF8304670BD002070BD70B510B1BDE87040DFE70025074C6E1E07E020
:203B60002046FFF7D9FF00B13546E06C20F00104002CF5D1284670BDBC0500102DE9F041DF
:203B800004460D4616464769C06880072ED0384603F072FB50BB3EB3012E02D0022E25D1CE
:203BA00004E0204601F0A5F905441DE0384603F051FBE168002841F01001E16005DA2046F0
:203BC00001F0BAF90120BDE8F081C9030BD5E26A61688A4200D91146A26911442269891ABF
:203BE000814200DD08460544002D01DA0220EAE7E16A6068E268814206D29103E06203D5ED
:203C000022F4003141F010024FF0000CA669AE4211DCE16A814201D90B4600E003469F19C9
:203C20002369FF1AAF4206DD814201D90F4600E007469F4207D1C4F808C0C4F800C042F001
:203C40002000A5620DE0AD1BE669AE1B8142A66000D90846C01A281A20605819606022F0A1
:203C6000200003490840E060002084F844C0AAE7BFCFD7FF70B5C468A50713D0650211D48F
:203C8000B2F5807F09D0B2F5007F06D0B2F5806F08D1012300F1240106E05D1E6FF07F467B
:203CA000B54201D3012070BD0161C361416024F470611143C160002070BD00002DE9F041D2
:203CC00007460C461646104600F078F82078611C61280AD0722802D077283CD102E001259B
:203CE000002405E00225042402E0082448F2020511F8010B2B2806D0622809D011F8010C66
:203D000074280AD00BE045F0030544F00204EFE745F0040544F00104EAE744F010043846E7
:203D2000214603F0BBFA411C15D00021316171604FF40071F560F1617061200704D530460C
:203D400002220021FFF71AFFF06C40F00100F0643046BDE8F0810020FBE72DE9F04105460E
:203D60000E46104CE06CC10704D0410804D020F00104F7E722460EE05020FFF713FC0700C9
:203D80000ED0E06C47F0010108435021E064384600F0D6F83A4631462846BDE8F0418DE7D5
:203DA0000020D6E7BC05001011B14FF4807201E04FF480624FF40073FFF75CBF2DE9F04744
:203DC00004464FF000094FF0FF37C568D4E90486A80707D0204601F0E3F8304603F026FA27
:203DE000002802DA3846BDE8F087280502D54046FFF707FC4821204600F0A2F8E06C20F0ED
:203E00000100E0644846EEE710B5431C02E010F8011B71B18107FAD14FF0013202C88C1A79
:203E20008C4314EAC211F9D0C01A0A0603D0C01E10BDC01A10BD0A0401D0801E10BD0902B5
:203E4000FCD0401E10BD40EA010370B59B072ED14FF00136042A2AD308C810C9121F9D1B44
:203E60009D4315EAC61517D0D8B2E1B2401A50EA056110D198B2A1B2401A50EA05410AD157
:203E800023F07F4024F07F41401A50EA052102D1180EA0EB146070BDA342DBD018BA21BA60
:203EA000884201D9012070BD4FF0FF3070BD0AB9002070BD10F8013B11F8014B63B1A342D3
:203EC0000AD1521E08D010F8013B11F8014B1BB1A34201D1521EEDD1181B70BD10B5203AF6
:203EE000C0F00B80B1E81850203AA0E81850B1E81850A0E81850BFF4F5AF5FEA027C24BF4A
:203F0000B1E81850A0E8185044BF18C918C0BDE810405FEA827C24BF51F8043B40F8043BD6
:203F200008BF7047D20728BF31F8023B48BF11F8012B28BF20F8023B48BF00F8012B704783
:203F40004FF0000200B5134694469646203922BFA0E80C50A0E80C50B1F12001BFF4F7AF3E
:203F6000090728BFA0E80C5048BF0CC05DF804EB890028BF40F8042B08BF704748BF20F8DB
:203F8000022B11F0804F18BF00F8012B704700004FF0013C50F8042B51F8043B9A4221D129
:203FA000A2EB0C03934313EACC1317D150F8042B51F8043B9A4215D1A2EB0C03934313EA9B
:203FC000CC130BD150F8042B51F8043B9A4209D1A2EB0C03934313EACC13DBD04FF0000039
:203FE000704700BFD01A01BAB1FA81F101F0180122FA01F0CB40C1F12001DBB2C0B2C01ABB
:204000002CFA01F3D11A914311EAC311E6D17047014901F0ADB80000AC06001030B50368D8
:204020001C1404EB21459BB289B2194495FBF2F402FB145301EB034191FBF2F302FB13117A
:2040400001E05B1E11440029FBDB016003EB044030BD2DE9F04704464FF0FF3A86B0006885
:20406000029060680390A0680490E0680190206900906569B5F1804F7DDCB5F1404F7ADB9F
:204080003C22002102A8FFF7C9FF3C22014603A8FFF7C4FF1822014604A8FFF7BFFF411EF0
:2040A00040F2B55201A8FFF7B9FF0C22064668460021FFF7B3FF00EB860028443D4D0026F2
:2040C0007D440FE0511A5B1CCDE90031022B02D00C2B07D104E0820704D0491C019101E040
:2040E000401C0096009B019AE95C9142EADD012B06D11C2A04D1810702D00221CDE9001652
:20410000A0F146018B293FD20199009B00228C4602E0AE5C521C31449A42FADB012B02DD4E
:20412000820700D0491E40F2B55540F26D16C21700EB927292106A4300F0030505FB062297
:2041400085070A4400D1521E049D02EB4206DDF80C80A94605EBC605174EC5EB0515029F93
:2041600008EB850535442E14ADB2C6EB0616C5EB0515B60000E007E007EB850506EB1546CC
:2041800066F31F45360C03D0504606B0BDE8F087C4E90430521C072092FBF0F304F11806EC
:2041A00000FB13200CF1010CA6E803042846A4E88013EAE7C8000100A039CEFD70B50546F7
:2041C00001B90721541A241DB4F5B67F09DD286800F062F9A04204DC2868401C2860012058
:2041E00070BD002C05DA2868401E286000F054F90444072094FBF0F0401C70BD2DE9F04F18
:2042000082468B4615461F46002689B000F0A2F9D0F810800024BBF1000F6FD015F8010BCC
:2042200020B125280FD00AF8060018E124B1641E06A850F82450F1E7002130460AF8061038
:2042400009B0BDE8F08FE94615F8010B59286ED023DC49286CD014DC44286ED008DC252803
:2042600068D041283ED0422849D043282CD157E04528E9D0462869D0472877D0482823D186
:204280007DE04D380C281FD2DFE800F08A1E061E1EA0A6AAB5B7C3D2D6E75A38212813D208
:2042A000DFE800F0111212121212121A26374351125A2D127712127B801282128B129CA4FB
:2042C00012B5BFCD1100A9E725200AF80600761C5E4513D26D1EA1E7D8F80010BA69D8F89D
:2042E000240011E0D8F80410BA69D8F828000BE0D8F808103A69D8F82C0005E0B8E0D8F8EB
:204300000C103A69D8F8300002FB001101EB0809B0E006A840F82450D8F81810641C52E03F
:204320007969642091FBF0F28FE0FA688DE08EE027E002E090E048461EE006A840F82450BE
:20434000641C66A56AE7FA6867A1F4E706A840F82450641C65A561E7384600F0B2F8642173
:2043600090FBF1F201FB120259E0FFE7384600F0A8F8024660A1684600F04AF97AE0BA68EC
:2043800063E0B8680B300C2190FBF1F201FB120204E0FA6959A1521CCDE73A69521C54E02C
:2043A0007A6852E00A2158E0B8680C2802DAD8F81010ABE7D8F81410A8E706A840F82450F7
:2043C000D8F83410641C01EB080527E706A840F82450641C4BA521E73A6836E009213CE072
:2043E00006A840F82450641C48A517E7BA6902B9072249A19FE700210CE0786900F26C70C5
:204400000890D7E9061208A8FFF7D8FE06E0BA69EFE70121D7E9062000F031F8024640A187
:20442000A9E706A840F82450D8F81C10641CCAE706A840F82450D8F82010641CC3E77969FF
:20444000642091FBF0F200FB121235A173E77A6929A102F26C726EE725210AF80610761C57
:204460005E45B2D304E00AF80600761C5E4501D30020E5E619F8010B0028A6D0F3E7511A34
:2044800001D501F10701401A01D500207047072190FBF1F0401C704781070CD1642190FB29
:2044A000F1F201FB120151B94FF4C87190FBF1F201FB120018B1002000F26D1070470120D8
:2044C000FAE708B5416901F26C710091D0E906126846FFF773FE009808BD0000256D2F250A
:2044E000642F2579000000002532640025592D256D2D25640000000025640000252E33646A
:204500000000000025483A254D00000025483A254D3A255300000000252E316400000000CF
:20452000252E32640000000070B5064C7C44064D7D4403E0206820448047241DAC42F9D1B8
:2045400070BD0000500201005002010000487047D806001000487047DC06001000487047AB
:20456000F006001000487047F406001000487047F8060010704770477047704738B504460C
:204580000A460020694601F0E7FB002808BF38BD02460099204600F047FE012038BD012092
:2045A00001F0B0BBF8B501F0CDFB054600200C46102000BF0646A819A0420DD93246694691
:2045C000002001F0C9FB070008BF01F09BFB0098A04218BF0546C419FFF7B8FF05600746D9
:2045E000F01D20F007004619284600F00AF8B44208BFF8BDA21B31463868BDE8F84000F0C5
:2046000013BE00210160C0E901107047102070470FB41CB5084B06AA7B44694600900598BD
:2046200000F0BDF804460020694600F0CBF820461CBC5DF814FB0000A901000070B504464E
:2046400085690068C10601D5302600E02026C00708D070BDD4E9012130469047206A00F178
:20466000010020626D1EF5D570BD70B5044685690068C00708D170BDD4E9012120209047AD
:20468000206A00F1010020626D1EF5D570BD09684A0501D540B27047C905FCD500B2704753
:2046A00009684A0501D5C0B27047C905FCD580B270472DE9F0470D4604469246994600F121
:2046C00024080168880604D5E06921F01001216000E00120A84202DDA0EB050700E000278A
:2046E000A16907EB050202EB0300A1EB0000A0612068C00602D42046FFF7A0FF002608E00D
:20470000D4E901211AF806009047206A401C761C20624E45F4DB2068C0060AD52046FFF7E6
:204720008DFF06E0D4E9012130209047206A401C2062381EA7F10107F4DC07E0D4E901210D
:2047400018F805009047206A401C2062281EA5F10105F3DC2046FFF788FF2068000602D50C
:204760000220BDE8F0870120FBE711680268006A530501D508700BE0D30501D5088007E0FD
:20478000130603D5C217C1E9000201E0520608600120704701694A1C02610878704700B50B
:2047A0008FB0CDE901310021059105497944CDE9031011466846FFF715F80FB000BD0000C3
:2047C000E5FFFFFF0A6802F8010B0A60704710B5436913B1AFF3008001E0FEF74FFF0120C2
:2047E00010BD126800F124010A7000224A700122EDE711684FF0FF32E9E70000074B70B5DF
:204800000C467B44FFF7CBFF0546204600F05CF910B14FF0FF3070BD284670BD2B2D000082
:204820002DE9FF5F04468A461546DFF8AC80F8440027D8E900103E46CDE9001011E03AF8EB
:2048400016106A4602A801F031FA411C07D02168890603D5E269391891420ED8074406F101
:2048600001062068800602D5E069B84205DDAE42E5DB3AF816000028E1D1A069C01BA06170
:204880002046FFF7DBFED8E90010CDE90010002016E03AF818106A4602A801F007FA8146C9
:2048A000401C0BD000250DF1080B05E0D4E901211BF8050090476D1C4D45F7D308F10100F9
:2048C000B0428046E5DB206A384420622046FFF7CCFEBDE8FF9F000052F900002DE9F041DD
:2048E0008046D21D22F007020026D2E90002F52914A512D0002A06DA0023D0EB030063EB13
:20490000020211A508E0D8F800108B0701D50FA502E0490701D50EA501261146002408F1A3
:20492000240704E000F09AFC30323A55641C50EA0102F7D133462A4621464046BDE8F041C0
:20494000FFF7B7BE000000002D0000002B0000002000000030B4002100F124040CE002F078
:20496000070505F130054FEAD20242EA4372655401F101014FEAD30352EA0305EFD10468E6
:20498000002310A2250708D504F020040C4304D0C46901230CA2641EC46130BCFFF789BE2F
:2049A00010B5044621461068FFF77AFE02462046BDE810400023CDE7D21D22F00701D1E95E
:2049C0000023C7E700000000300000003A2800D2303820F02002412A01D3A2F13700884235
:2049E00001D34FF0FF3070470268114413780160184670470B461146054A7A444A61054A4F
:204A00007A440A620022C1E9033200F09BBE0000EBFFFFFFE3080000426842B1016811F840
:204A2000013B23B1521EC0E90012184670470121C160881E7047416859B1C368026843B942
:204A40008368934205D0521E491CC0E90021002070474FF0FF3070472DE9F0470F469146AD
:204A600080460446002614F8015B2DB100F0D4FB0068405DC007F6D12B2D02D02D2D18D0FC
:204A8000641E4A463946204601F018F827B13968A14201D1C7F800804FF0020471050BD516
:204AA0004042002803DDFFF761FD0460A007BDE8F08746F48066E4E70028F8DAFFF756FDC3
:204AC00004606FF00040F2E7C06800F08000704770B5064614460D46D36850690A463146D2
:204AE00002F052FC002807DA411C07D0E16820F0004041F48041E160281A70BD204600F0A4
:204B00001BFA4FF0FF3070BDC1680022026021F4805141F0400111F4C06FC16001D08260D8
:204B2000704702694168891AC269891A816070472DE9F0470446C06840F48000E0600103EA
:204B400013D520F40020E060810607D4E26A61688A4200D80A46A2EB0101216040F400103A
:204B6000E06094F82500BDE8F08720F40010E060800602D5204600F036FAE06842F28101E3
:204B80004FF0FF390140012903D0204600F0D4F9B8E02168002600290ADAC94340F48050D9
:204BA0002160C4E902606068411C61600078DAE744F2400108420ED020F4A04040F0400043
:204BC0002660E06021696068A0EB0100E169A0EB0100A06096E0216991B9C00310D4E06921
:204BE000FEF7E0FC2061B0B1E06840F4006010F4407FE06002D140F48070E06020696060A3
:204C0000E068D4F814A0C1061AD5C0030ED5204600F0C6F914E004F1240020610120E0616B
:204C2000E06820F4407040F48060E6E721696068401AA1690144504602F0C4FB0028A4DB9E
:204C4000E068C0032AD56168E06A884200D808462169451AE069471B1BD02046D4F81880FE
:204C600000F09EF908EB05015046C4F8188002F0A9FB002889DBE06840F40030E0600002BA
:204C800002D5A0692844A061E1692069C91B45180DE0204600F084F9E769F5E72569616870
:204CA000D4E90607491BE56208446560A061E06820F0100010F4C06FE06002D0204600F06A
:204CC000DBFFE06840F48050C4E90260000205D52069E06260606FF0010044E722463946C6
:204CE0002846FFF7F5FE411C0CD02918E16258B1401E2060681C6060E06840F40030E06089
:204D0000287830E748462EE765602046FFF7FCFEF8E72DE9F04705460C46C86820F42010E1
:204D200040F48000C860800602D5084600F05BF9E06841F282014FF0FF390140022903D0F4
:204D4000204600F0F9F8B9E000F42041B1F5004F0FD1C00306D56168E06A884200D80846A8
:204D6000606006E02069E0626060606902F072FAA061A0680022EEB200280FDAE1688B0526
:204D80000CD4C043A06041F490302260E060304661684A1C62600E70BDE8F087E06890465A
:204DA000226040F40050E060206968BB606902F063FA012704F12405A0B1E06810F4407F47
:204DC00008D0E069FEF7EEFB206118B1E06840F4006016E0E7612561E06820F4407040F4AA
:204DE00080600EE0E069FEF7DDFB00282061F1D0E06840F4006010F4407FE06002D140F47F
:204E00008070E06020696060E06825696FF0010AC10520D56168E06A884200D80846411BBF
:204E200004D02246284600F091F8E8BBE068010203D5E562C4E9015857E005F10101E162CA
:204E40006160E16940F48030A1F10101C4E9021030462E70A0E7010202D500F480320AE00B
:204E60006068411C61600670E0680A2E40F48030E06006D00022E16A6068814203D90B4637
:204E800002E00122F7E70346E768A3EB05037F0503D4E7699F4200DDEAB1814200D801461B
:204EA0000F1A002BE56200E008E0C4E9015807DD22461946284600F049F808B148466BE7A6
:204EC0004FB1A069E5626560A0EB0700A061E06840F01000E060E068000208D56168A06969
:204EE000E562491B08446560A061504654E7304652E710B50146C268900703D0900607D563
:204F0000886A0BE0FFF732FB01210160881E10BD8B69486818440B69A0EB030091F844309C
:204F200023B191F84510A0EB010010BD1103FCD50028FADD401E10BDC16821F4001141F0D7
:204F40008001C16000218160016070472DE9F04781460E4614464FF0FF383248D5685769E6
:204F6000054209D03846A16902F02CFA002811DB2C48C0430540E5602B4632464946384666
:204F800002F034FAA16920F00042B21A11440028A16103D02046FFF7CFFF4046BDE8F087AB
:204FA00070B504460569C06A6168884200D80846E16821F42011E160C90312D5A84208D0EC
:204FC0002246411B2846FFF7C1FF10B14FF0FF3070BD0020E562C4E90150E06820F480301C
:204FE000E060002070BD10B50446C06820F02000E060A16AA06988420DD02046FFF7D0FF97
:20500000E06820F4405040F01000E060A06AA0612069E062606044F24001E0688843E060C4
:2050200010BD00001000020010B542485021FEF787FF41485021FEF783FF40485021FEF7F7
:205040007FFF3F483B493C4B3F4A01603D4803603A4810605A1CCA64411CD9640121C164F7
:205060003B48344A39A17844FEF728FE20B9384878440A3800F03FFE37482F4A35A1784470
:20508000FEF71CFE20B9344878440A3800F033FE32482A4A2FA17844FEF710FE20B92F48C0
:2050A00078440A3800F027FE40232248DC0000212246FEF7DFFD20B125487844543800F064
:2050C0001AFE1D48224640230021FEF7D3FD20B121487844543800F00EFE18482246102329
:2050E0000021FEF7C7FD002806D01C487844BDE81040563800F0FFBD10BD104870B5C06C13
:2051000020F001040B48FEF759FE0B48FEF756FE0A48FEF753FE09E0E06C20F001052046F6
:20512000FEF74CFE2046FEF76CFA2C46002CF3D170BD0000BC0500100C0600105C0600107B
:20514000C4020010C8020010CC02001072000000FCEE000077000000EBEE0000DBEE00004C
:2051600010B500F0D7FDBDE8104000F0BFBD000070B50C46016800204A1C34D040F2B5559F
:205180003C23B1FBF3F203FB12112160B2FBF3F103FB112218236260B1FBF3F203FB12110C
:2051A000A16046F2E0310A440721B2FBF1F301FB1321B2FBF5F305FB1322A1619900B2F562
:2051C000B77F06D3521EAD10B2FBF5F3194405FB13220F4BE261616189077B440CD03B2A7D
:2051E0000AD3521C08E02C212046FEF7A9FE0120E0600AE0521A401C195C9142FAD9521C91
:20520000C4E903204FF0FF302062204670BD0000AEEF000000F0BCBD10B5FFF79BF9001DC9
:2052200010BD00BF5D2F0000034640688C46002818BF814284BF03464068F8D818681844F1
:20524000884207D00CF1030020F00700001D411A521A0146081D0A60FEF7D3B930B5B0F1D5
:205260000A024FEA900E71F100034EEA817EB0EB0E0061EB91014FEA101E4EEA017E10EB0F
:205280000E0041EB11114FEA102E4EEA016E10EB0E0041EB11214FEA104E4EEA014E10EB14
:2052A0000E0041EB1141401841F100014FEAD00040EA41704FEAD10110EB80054FEA8104AA
:2052C00044EA907444EB01046D1944EB0404521BA3414FF0000348BF0A3200D530BD401CB7
:2052E00041F1000130BD10B50446FFF795FF0068005D00F0010010BD70472DE9FF4F0C4605
:205300001E464FF0FF378BB0D2E90001DDF860800A908A46C1F30A5505B93D4600210846DB
:205320004FF00000BAF1000F00F4400005DA00EB80004FF4400101EA50004FEA9059B9F16B
:20534000010F00DDB9460A9850EA4A000ED044F61050A5F2FF3545432F14B8F1000F1ED087
:205360007542291E1EDDC9F100021CE0B8F1010F4FF0000001D1F24307E0302101E02154EF
:20538000401CB042FBDB30460022002121540B99C1F80880C1E900200FB0BDE8F08FBD1B51
:2053A0006D1CDEE74A4600DA694206A800F0C8FE06AB07CB03AB07C350460A9901F052F8B7
:2053C0008DE80700A0F500501F3800900398002D09DD42F21F014A46084403A903906846BA
:2053E00001F0B1FA08E0A0F500504A461F3803A90390684601F0BBFA8DE807000004000C3E
:2054000003D04FF0FF30410800E01046B8F1000F03D00022009215461FE0751E06D4FFF7D0
:205420001DFF02F1300262556D1EF8D5B3460122084302D000227F1C04E02078302801D180
:2054400000227F1E002A099787D01DE0112D07DAFFF704FF303262556D1C50EA0102F5D1B2
:2054600008430FD10021681E05E0235C625C6354491C2254401E8142F7DBAB46A81B401EA1
:20548000099001E0009848B1002004F80B000B98099AC0F80880C0E9002B7DE711264FF0A6
:2054A00000085AE72DE9F04F88460446D21D22F0070191B0D1E90001CDE90A0101F056FE2B
:2054C00002460B98C00F01D02D2007E02068810701D52B2002E0202101EAC000032A099048
:2054E00001D0072A05DB03464146204600F0E8FD0EE12068800601D5E06900E00620B8F1F4
:20550000650F814606D0B8F1660F18D0B8F1670F72D132E00020B9F1110F0090484601DB1C
:20552000112300E0431C0AAA01A90CA8FFF7E5FEDDE90C70002609F10105834648E0012093
:205540004B4600904FF000470AAA01A90CA8FFF7D4FEDDE90C050E990026AB4619B909F169
:20556000010100EB0105B9EB050003D4C0F1FF3609F10105A5EB09002BE0B9F1010F01DA99
:205580004FF001090020B9F1110F0090484601DD112300E003460AAA01A90CA8FFF7ADFECC
:2055A000DDE90C704D4600268346206800070AD4AB4500DA5D4601A8012D04DD411911F832
:2055C000011C302907D04F4502DA17F1040F04DA0120824610E06D1EEEE7002F02DCED1BC7
:2055E0003E4403E0781CA84200DD0546A7EB060000F1010A4FF000472068000703D4AA4531
:2056000001DB4FF0FF3A0021B7F1004F0DF143088DF8431022D002202B23002F01DA7F42D0
:205620002D230A22011EA0F1010000DC4FB197FBF2F102FB117C0F460CF1300C08F801CD06
:20564000F0E7A8F1010003702168090501D5452100E06521A0F1010800F8011C09980FA925
:20566000A1EB080707F1070700B1012000EB050101EBEA70A1693844A1EB0000A0F10100DC
:20568000A0612068C00602D42046FEF7D7FF099830B1D4E901219047206A00F1010020627E
:2056A0002068C00620D52046FEF7C8FF1CE0002E04DBB34502DD01A8805D00E03020D4E932
:2056C00001219047206A761C401CBAF1010A20620AD1FEF73FFFC0680168405CD4E9012107
:2056E0009047206A401C2062281EA5F10105DEDC07E0D4E9012118F8010B9047206A401C30
:205700002062381EA7F10107F3DC2046FEF7ADFF022011B041E610B5436913B1AFF30080DA
:2057200001E0FFF77DF8012010BD126800F1240182840022C2840122EDE711684FF0FF3251
:20574000E9E700002DE9F34F4FF0000A0C4656468FB001200DF1100B0D9001F10C00039043
:20576000626903980121904705002DD0252D2CD0216A8847C0B16269039801219047216AC5
:2057800088470028F7D16269411E0398904700E0761CA1690F988847216A88470028F7D172
:2057A000E1690F988847DBE7A1690F988847A842074601D1761CD3E7E1690F9888477F1C37
:2057C00002D1BAF1000F6FD06BE16269039800273D46394690472A2804D16269039801219C
:2057E00090470125DFF8D0826269039801219047A0F130010A290AD24745E5DC07EB87018C
:2058000000EB4107303FDFD445F01005ECE7E90601D46FF000476C280AD04C2814D0682856
:2058200015D06A280DD074281CD07A281AD01DE062690398012190476C2802D045F0040500
:2058400014E045F002050DE045F020050AE06269039801219047682802D045F0080505E0FF
:2058600045F400656269039801219047C4E9015765283DD019DC582879D00CDC452837D072
:2058800004DC252826D041289ED131E046282FD0472899D12CE05B287FD0612828D06328CC
:2058A0007BD0642823D159E0F6E06F2847D008DC66281DD067281BD0692821D06E2816D188
:2058C00027E0702844D0732867D0752846D078280DD14CE0A1690F988847252805463FF49B
:2058E00069AFE1690F9888476D1C3FF46AAFD8E00F9923466A466FF00100AFF30080C5E05B
:2059000045F0400023464FF000026060A80735D43DE0206800F1040121600068290501D568
:2059200006701DE7290701D5068019E7A90704D54FEAE671C0E9006112E7066010E745F0B3
:20594000400023464FF008026060A80716D41EE040F60E0125EA0100606016E045F040007E
:2059600023464FF00A026060A80707D40FE045F040006060A80708D5234610220F996FF0D7
:205980000100AFF3008081E007E0102223460F996FF00100FEF70AF878E04FF000096328D7
:2059A0004F46C8464B46CDF8309002D05B2806D02FE0E80601D40120A060012729E0626914
:2059C0000398012190475E2805D14FF001094946626903989047216979B3E168891E0C917F
:2059E00060B3216959B308F1010862690398012190475D28F4D1B9F1000F09D05946002002
:205A000051F82020D24341F82020401C0828F7DB04AB2069002860684FEA407027D02246A1
:205A2000CDF80080CDE901970C9B0F9900286FF0010029DAAFF3008028E001E031E007E0F6
:205A400000235A4642F82130491C0829FADBC7E7C11700EBD1635A1123F01F030BEB8201CF
:205A6000C31A0A680120984002430A60BDE7009722460F9900286FF0010002DAAFF300805E
:205A800004E0AFF3008001E0AFF3008000280ADA401C06D10D9820B14FF0FF3011B0BDE874
:205AA000F08F5046FAE7E90701D10AF1010A064400200D9054E60000CCCCCC0C2DE9F05F12
:205AC000824604468B461546641C0027B9460078302801D09DB113E014F8010B0127782820
:205AE00003D0582801D045B10AE00DB1102D07D1002714F8010B102502E0082500E00A253D
:205B00000026B0460EE005FB080005FB06F101271FFA80F801EB1046B6F5803F00D3B94645
:205B200014F8010B2946FEF751FF0028EBDABBF1000F05D00FB1641E00E05446CBF800405D
:205B4000B9F1000F06D0FEF711FD02210160C81EBDE8F09F48EA0640FAE72DE9FF5F0646FC
:205B60008B461C46080068D000250299284627680BFB01F965E0002F65DCE069484541DA4F
:205B8000BAF1000F3ED0E068800601D5A06A04E0A169606808442169401A2246A9EB0501A7
:205BA00080463046FEF794FF002814DD4FF000078044A8F101010644A161226916F8011C61
:205BC00005441170216901F10101E1626160E16841F40031E160411C03D010B1E06840060A
:205BE00044D52046FEF790FFC4F8188020696060E062E068276020F40030E060E0694042A5
:205C0000A06018E0484503DAE06840F40000E0602046FEF78DFFE16821F40001E160411C82
:205C200008D0811C0CD02768002809DB6D1C06F8010B1BE02760B5FBFBF004B0BDE8F09FE0
:205C40000120824612E0A9EB0500B846B84200DA804630464246616800F048FB6168A7EBE3
:205C60000807464401EB0800454460604D4582DB27600298E1E7000070B5054640F20226AC
:205C8000094C0EE0E06CC00708D0AC4206D0E06836EA000002D12046FDF73EFFE06C20F0E4
:205CA0000104002CEED170BDBC05001070B505460C461646FFF7B0FA036893F80101012817
:205CC00006D0FF2C0FD8185D68B101202C7070BDD3F807013246214603442846BDE87040A8
:205CE00003F2071318474FF0FF3070BD002801D000F05CB8704710B500F0B6FABDE810408D
:205D0000FFF7F4BF10B500F0C9FABDE81040FFF7EDBF000010B5002102A000F08BFA0120AD
:205D200010BD00005349475056464E3A2050757265207669727475616C20666E2063616C18
:205D40006C656400114B00F580528A421A6001D8114670471960704730B50C4D6B46A3F507
:205D600080532C6822449A420FD89B1A02F5805003EBD37302EB6303984200D91846C01DA2
:205D800020F007020C60101B2A6030BDD002001010B500F0F3FA016919B1002202618847D0
:205DA00001E08068804700F03DFA000001491820ABBEFEE7260002002DE9F04F04460D4642
:205DC000D21D22F0070089B0D0E9009248461746394601F0CBF90246F80F01D02D2307E0C1
:205DE0002068810701D52B2302E0202101EAC0038DF820300BB1012000E00020032A8246F7
:205E000001D0072A04DB2946204600F059F943E12068800601D40D2500E0E569C7F30A5609
:205E20000D2D4CDA00214FEA175B08464FF00000002F00F4400007DA00EB80004FF4400176
:205E400000EBD07001EA60004FEAA05CBCF1010F01DD4FF0FF3CAB000021182B06D30A464A
:205E6000A3F118004FF08051C14002E04FF48012DA400C33202B03D3203B09FA03F001E002
:205E800007FA03F0BCF1000F4FF0004801DD18B915E014D1404512D319EB01035741994659
:205EA000BCF1000F06D1404504D1184613469F4320EA0109BBEB175F01D006F101062068D5
:205EC000000502D57C48784402E07B487844193808AB302203F80A20027C0AF10101002EE1
:205EE0000AF1020A5A54694602DC4FF0300201E04FF031024FF001088DF8002002D0A6F245
:205F0000FF3603E059EA470200D06C4E002D02DC2268120704D54FF002082E228DF801208D
:205F2000C44600230BE0C7F303423F01825C5B1C6D1E01F80820052B08F1010801DA002DCF
:205F4000F1DC00220CE000EB1973521C1B786D1E082A01F8083008F101084FEA091901DAC8
:205F6000002DF0DC2268920602D514E0A8F10108E04505DD01EB080212F8012C302AF5D046
:205F8000B8F1000F07DD01EB080212F8012C2E2A01D1A8F10108002D05DD3E2201F80820DC
:205FA0006D1E08F10108407C002E01F8080008F1010806DA2D2001F80800764208F101087F
:205FC00004E02B2001F8080008F101080A274FF47A739E420ADB96FBF3F000F1300203FBD4
:205FE000106601F8082008F1010801E0642E0BDB642396FBF3F000F1300203FB106601F824
:20600000082008F1010801E00A2E07DB96FBF7F000F1300001F8080008F1010896FBF7F047
:2060200007FB106000F1300001F80800A16908F1010808EB050202EB0A00A1EB0000A06142
:206040002068C00602D42046FEF7F8FA216A08AE01EB0A00206204E0D4E9012116F8010B39
:206060009047BAF1010AF7D22068C00602D52046FEF7E4FA6E4609E016F8010B3E280FD070
:20608000D4E901219047206A401C2062B8F10108F2D22046FEF7E9FA09B00220BDE8F08F2F
:2060A000206A2844206203E0D4E90121302090476D1EEBD3F8E70000E1E2000002FCFFFF98
:2060C0002DE9F04104461F4603260168072A01F4006004DB08B116A505E016A503E008B123
:2060E00015A500E015A521F010002060A069C01EA0610FB1401EA0612046FEF79FFA4FB1B0
:20610000D4E9012138469047206A401C2062C01C206206E0206AFAE7D4E9012115F8010B3C
:206120009047761EF8D22046FEF79FFABDE8F0814E414E006E616E00494E4600696E6600EC
:206140002DE9F047814616468AB035487844D0E9002380680092CDE90130314878440C38A6
:20616000D0E90223006903924FF03702CDE9043041F69B30014491FBF2F0A0F1800502FB19
:2061800010141B3C02D56442012000E00020DFF890A080460027FA44AAF1C60A0DE0E00775
:2061A00009D03246684607EB47010AEB810100F0DEFB8DE8070064107F1C002CEFD1184F88
:2061C0007F44B43F17E0E80713D007EB04100DF1180A90E80E00AAE80E00C068F04201D1C8
:2061E00098190890324606A903A800F0C0FB03AB07C36D10641C002DE5D132466946B8F1B1
:20620000000F03A802D000F09EFB01E000F0AFFBC9E90001C9F808200AB0BDE8F08700007C
:20622000ECE00000002000F0DBF8AFF300800120FFF7BCFD70B505460C460A2000E06D1C68
:2062400000F0C2F835B128780028F8D102E0641C00F0BAF814B120780028F8D1BDE8704076
:206260000A2000F0B1B8000010B5014602A0FFF7E1FF012010BD00005349475254524544C5
:206280003A2052656469726563743A2063616E2774206F70656E3A200000000010B5012831
:2062A00005D0002103A0FFF7C5FF012010BD09A1F8E7000053494752544D454D3A204F758E
:2062C00074206F662068656170206D656D6F7279000000003A2048656170206D656D6F72C6
:2062E0007920636F7272757074656400032A40F2308010F0030C00F0158011F8013BBCF198
:20630000020F624498BF11F801CB00F8013B38BF11F8013BA2F1040298BF00F801CB38BF7F
:2063200000F8013B11F003033DF4D8AD083AC0F0088051F8043B083A51F804CBA0E8081070
:20634000F5E7121D5CBF51F8043B40F8043BAFF30080D20724BF11F8013B11F801CB48BF19
:2063600011F8012B24BF00F8013B00F801CB48BF00F8012B70470000FFF754FF70B500F0CD
:206380002BF804680546A4B92020FDF70BF9040011D00A4900202C60C4E900010849A160AA
:2063A0002073206160610749A06109B100F01FF8E061204670BDFFF735FF000000000000F8
:2063C000796300000000000008B569468DF800000320ABBE08BD000000487047FC0600108E
:2063E00010B500F027F8BDE81040FFF77FBC10B58820FDF7D7F8002801D00021017010BD1B
:20640000802902D808B1017809B100207047012100F8081B704718B100F10802914201D0DA
:20642000002070470021017070470000004870470007001010B5002102A0FFF7FBFE01208E
:2064400010BD0000534947414252543A2041626E6F726D616C207465726D696E6174696F81
:206460006E0000005FEA400C08BF91F0000F4FEA8C234FEAC12243EA51514FEA1C5018BF73
:2064800000F5F0404FEA300018BF41F000415FEA6C5C00F02980BCF1FF3F08BF40F08040D9
:2064A0007047130C06BF12044FF0100C4FF0000C130E04BF12020CF1080C130F04BF120184
:2064C0000CF1040C930F04BF92000CF1020CD30F04BF52000CF1010C11464FF00002A0F183
:2064E0001F00A0EB0C00704711F0004F08BF704731F000413FF4D5AF0B0C06BF09044FF020
:20650000100C4FF0000C0B0E04BF09020CF1080C0B0F04BF09010CF1040C8B0F04BF890042
:206520000CF1020CCB0F04BF49000CF1010CCCF12003A0EB0C0022FA03F302FA0CF241EAB2
:20654000030100F10100704720F07F4C80EA030023F07F47ACEB070303F57C5300F00040D5
:2065600003F1FF032DE980494FEA154B09B44FEA144325EA0B4E24EA03480FF2042606EB83
:20658000132749083E785FEA320203FB0667C7F5000707FB06F64FEA54374FEAD64606F101
:2065A000020607FB066CCCF1005C4FEA1C472CEA074C07FB06F40CFB06F504EB15464FEAC0
:2065C000961634BF00204FF000404FEAD13706FB07FC4FEA1C4C0CFB0BF7D21B03FB0CF7A0
:2065E00061EB07010CFB0EF7B0EB074072EB17420CFB08F734BFA2EB0742B2EB074261EBA2
:2066000017414FEA0C444FEA910706FB07FC4FEA1C4C0CFB0BF7B0EBC74072EB573203FB94
:206620000CF734BFA2EBC742B2EBC74261EB57310CFB0EF7B0EBC70072EB57720CFB08F7BA
:2066400034BFA2EBC702B2EBC70261EB5771039F4FEA816141EA921104EBCC044FEAD137EC
:206660004FEA826206FB07FC42EA90124FEA80604FEA1C4C0CFB0BF7D21B03FB0CF761EB2E
:2066800007010CFB0EF7B0EB074072EB17420CFB08F734BFA2EB0742B2EB074261EB1741F5
:2066A0004FEA8C554FEA910704EB9C2406FB07FC4FEA1C4C0CFB0BF7B0EBC74072EB57320A
:2066C00003FB0CF734BFA2EBC742B2EBC74261EB57310CFB0EF7B0EBC70072EB57720CFB1B
:2066E00008F734BFA2EBC702B2EBC70261EB577115EB4C254FEA816141EA92114FEA826261
:206700004FEAD13742EA901206FB07FC44F100044FEA80604FEA1C4C0CFB0BF7D21B03FB7F
:206720000CF761EB07010CFB0EF7B0EB074072EB17420CFB08F734BFA2EB0742B2EB0742A9
:2067400061EB174115EB1C154FEA813141EA92414FEA823242EA90424FEA80304FEA0C76EC
:2067600044F1000448EA03434EEA0B484FF0000EB2EB080C71EB030724BF624639464EEB36
:206780000E0E4FF0000B0018524149414BEB0B0BB2EB080C71EB03077BF1000B24BF6246F9
:2067A00039464EEB0E0E4FF0000B0018524149414BEB0B0BB2EB080C71EB03077BF1000BAC
:2067C00024BF624639464EEB0E0E51EA020718BF46F0010616EB0E7655F1000254F10001EF
:2067E00003D5BDE88901BDE80088BDE88901BDE80048B619524141EB0101A3F1010370476A
:2068000080807F7E7D7C7B7A7978777676757473727171706F6E6E6D6C6C6B6A6A69686811
:20682000676666656464636362616160605F5F5E5E5D5D5C5C5B5B5A5A5959585857575692
:20684000565555555454535352525251515050504F4F4F4E4E4D4D4D4C4C4C4B4B4B4A4A44
:206860004A4949494848484747474746464645454544444444434343434242424241414177
:20688000002B26D4770021D01CB54FEA370703B44FF010004FF010014FF000000FBCBDE81E
:2068A00010400BF1010BBBF1010F08BF5FEA170722BF12F1010211F101014FF0004143F1F7
:2068C000000300F0004043EA00007047F9D35708DAE746EA064613F1400F4FEA16461FDD55
:2068E00013F1200FDFBF16430A46002120335B42C8D0C3F1200746EA064602FA07F74FEAEB
:20690000164646EA0706C3F1200722FA03F201FA07F721FA03F14FF0000342EA0702B1E7DB
:2069200046EA020646EA06464FEA164646EA0106BCBF46EA0646360C4FF000034FF000021B
:206940004FF000019EE72DE9C048934630B491E8380007C831EA400C48BF34EA430C03D564
:20696000FFF7F2FDFFF78CFFF0BCBDE800882DE9C048934630B491E8380007C810F0804FAE
:2069800008BF13F0804F03D100F005F8FFF778FFF0BCBDE8008820F07F4780EA030023F001
:2069A0007F4C07EB0C03A3F57C5300F00040A3F1FE0392F0000F00F0B38095F0000F00F0A7
:2069C00077802DE901494FEA11404FEA144621EA004800FB06FC24EA064708FB06F607FB97
:2069E00008F800FB07F718EB06484CEB164C4FEA124B18EB07484FEA15464CEB174022EA9E
:206A00000B4E0BFB06FC25EA06470EFB06F607FB0EFE0BFB07F71EEB064E4CEB164C4FF06D
:206A200000061EEB074E4CEB174B18EB0B0840F1000018EB0E0B58EB000840F100008F1AD1
:206A40004FF000013CBFC943661B14BFB5EB040C00213CBFC943F61B4FEA17444EEA8E0E4A
:206A600027EA04454FEA1C4704FB07622CEA074C05FB07F70CFB05F604FB0CFC16EB0746FA
:206A800042EB174216EB0C4642EB1C421BEB060658EB0202414146EA9E0601D5BDE80189DE
:206AA000B619524141EB0101A3F10103BDE801894FEA14454FEA114724EA054621EA074CA5
:206AC00005FB07F406FB07F70CFB06F105FB0CFC11EB074144EB17444FEA124711EB0C410D
:206AE00044EB1C4422EA074C05FB07F206FB07F70CFB06F605FB0CFC16EB074642EB1742D1
:206B000016EB0C4642EB1C456A1854F1000148BF7047B619524141EB0101A3F1010370472F
:206B200095F0000F37D04FEA11424FEA144721EA024624EA074C02FB07F106FB07F70CFBEB
:206B400006F402FB0CFC14EB074441EB17414FEA154714EB0C4441EB1C4125EA074C02FB9C
:206B600007F506FB07F70CFB06F602FB0CFC16EB074645EB174516EB0C4645EB1C4212192C
:206B800051F1000148BF7047B619524141EB0101A3F1010370474FEA14454FEA114724EAE4
:206BA000054621EA074C05FB07F106FB07F70CFB06F24FF0000605FB0CFC12EB074241EB77
:206BC000174112EB0C4251EB1C4148BF7047921841EB0101A3F101037047000070B50A4D18
:206BE0002C680A4AB4F1805F136809D02C68002254F8226043F82260521C312AF8DB2B606D
:206C000003EB8000016470BD08ED00E09002001030B525482021C0F8A011D0F8A0118906F9
:206C200003D5D0F8A0114906FBD500F180000221C0F884104FF00002C0F82821C0F82C21BD
:206C40004FF00103C0F88C304FF00B0141604FF0AA04C4604FF05501C1600360C460C16022
:206C6000A0F18000D0F888506D01FBD5032540F8805FC460C160A0F18000D0F8881011F02F
:206C8000407FFAD00521C0F808110849C0F8C410C0F8C821016843F23A0221F47041114302
:206CA00001600348036030BD00C00F40DE872804A002001004480068002804D1034A04483C
:206CC000511E00F04DBF7047A402001003C00920AC02001070B505460068012200210369AA
:206CE000284698470446401C0ED02868022200210369284698470646286800222146036964
:206D000028469847304670BD4FF0FF3070BD000010B5074901600021064A0B4652F8214005
:206D2000844201D142F82130491C1029F6D310BDD44301007C050010016889680847024662
:206D4000001D01F06DB9001D01F0B6B910B5044603482060034801F0C9F9204610BD000077
:206D600000440100396D000010B5044603482060201D01F0A1F9204610BD0000004401000E
:206D8000016801B108474268002A04D000F1080183691046184770470160002141607047B5
:206DA000016000214160704770B50D46044600F007F82946201DBDE8704001F0D1B80000CD
:206DC00070B5084D04462868A0420AD0D4E902120023201D00F074FF201D216900F0B4FFA5
:206DE0002C6070BD9C020010C0E90212024A00211160FFF7E5BF00009C020010024A01619B
:206E000000211160FFF7DCBF9C02001038B504460B4820604FF0FF300090201D01F014F85F
:206E2000082100220748A160C4E903201346201D00F046FF201D216900F086FF204638BD85
:206E40001444010040420F0010B500F019F802F00DF8BDE81040014901F046BF0024744975
:206E600010B5044601F01AF960600020A06010BD10B5044601F012F960600120206010BD19
:206E800010B5044600F003F8A168084410BD10B504460068002803D001F000F96168401A57
:206EA00010BD10B50446FFF7DBFF204610BD0020704770B504460D464069FCF748FE28460A
:206EC0006169BDE8704000F033BB2DE9F04107460E460C468D1807E03868816A3846884717
:206EE000411C03D004F8010BAC42F5D1A01BBDE8F08100207047002070472DE9F041074693
:206F00000E460C468D1807E0386814F8011B426A38469047401C01D0AC42F5D1A01BBDE835
:206F2000F081002070470FB470B5054606AC4069FCF70DFE224668690599F9F7CFF970BCC2
:206F40005DF814FB3EB500F093F804460948206034306060224608A16846FCF779FB07A152
:206F60006846FCF7FAFE00216061FCF71DFF20463EBD0000204401003A257000772B000050
:206F800010B5044605482060343060606069FCF715FF2046BDE8104000F07AB8204401003F
:206FA00070B50D460446FFF7CEFE256101F076F8216901442046BDE87040FFF7C0BE10B5A5
:206FC00004464068216901442046FFF7B8FE04F11400BDE81040FFF7D3BEFFF7C5BE007B65
:206FE0007047000070B506460B480D4604680EE0A06858B12A463146FCF725FF30B9A06869
:20700000FCF702FFA84201D1204670BD6468002CEED1002070BD0000C0020010064B0360A3
:207020008160027321B105490A68426008607047002141607047000078440100C00200109F
:20704000094901608168002905D0084A1168814203D141681160704711464A688242FBD1CA
:2070600042684A607047000078440100C002001010B5054A04C00022FFF7D0FF034940F833
:20708000041D2C31416010BDD44301008844010010B5001DFFF7D4FFBDE81040001FFFF76A
:2070A00037BE10B5044600F004F8002800D0606810BD10B54068FFF792FF012800D0002046
:2070C00010BD10B5044600F007F8002803D06068002800D0001F10BD10B54068FFF77FFF5D
:2070E00008B1002010BD012010BD0068704770B5044600202060606008782F280DD1487899
:2071000058B14E1C00253146266008782F2806D038B16D1C491C2160F7E7204670BD481C00
:20712000206029463046FFF75DFF29463046FFF759FF6060F1E7FFF723BF10B500F002F846
:2071400010BD000010B5040007D1012405E0FDF705FA006800B9044880472046FCF722FA1B
:207160000028F4D010BD000015520000490050EAC12018BF04204A0D18BF40F0010040F2FF
:20718000FF72B2EB515F08BF40F00200012808BF052070472DE9F04106460F469046002589
:2071A0001020FCF7FFF904000AD0201DA0E8C001FDF7D8F90168216004602846BDE8F081B9
:2071C0000125FAE72DE9F0410646FDF7CBF9804613E026B1E068B04201D025460EE02068E1
:2071E0002860D4E90101D8F8007088472046FCF708FAD8F80000B84200D045462C68002CF9
:20720000E7D1BDE8F0810020FDF7AABF02486A4620F00700704700000B07001030380A289F
:2072200001D201207047002070470000032801DA002070470649002201EB800151F80C0DAF
:207240000A6010B10168496808474FF0FF3070477C050010032801DA00207047054901EBCD
:20726000800050F80C0C10B10168896908474FF0FF3070477C050010032801DA012070472F
:20728000054901EB800050F80C0C10B10168C96808474FF0FF3070477C0500102DE9FC471B
:2072A0000E4605463549FCF773FEB0B133492846C91DFCF76DFEA8B1304928460F31FCF74B
:2072C00067FE98B12E4F00244FF0FF3957F8240080B1641C102CF9D34EE0FFF7EBFC002091
:2072E000BDE8FC87FFF7E6FC0120F9E7FFF7E2FC0220F5E7102C3FD228783A280CD0294621
:207300006846FFF7F4FE6846FFF7E6FE0028684609D0FFF7D6FE2AE06A461AA12846FCF700
:2073200027FB009823E0FFF7BCFE28B3B10701D5022508E0710701D5012504E0310701D502
:20734000092500E0002516F00C0F01D045F40075710701D545F4806580466846FFF7C5FEC1
:207360000146D8F800002A4683684046984718B147F82400E01CB3E74846B1E7663F0100A8
:207380007C0500103A25700070B50D461446032805DA0A4800F0DCFB2870012009E00849A5
:2073A00001EB800050F80C0C28B101688B6829469847201A70BD4FF0FF3070BDAC020010BE
:2073C0007C050010032801DA00207047064A02EB800050F80C0C18B10268136900221847F2
:2073E0004FF0FF30704700007C05001070B50E46154603280FDA0F48006808B9FFF75AFC23
:20740000002404E0315D0C4800F04AFC641CAC42F8D3284609E0094901EB800050F80C0C9E
:2074200028B101680B6831469847281A70BD4FF0FF3070BDA4020010AC0200107C05001032
:20744000044600F011F908B100F020FA0CB100F0C9F8FEE72DE9F041C1F30A52A2F2FF36B2
:207460002F4A304B0D460446142E2FDA002E12DA00F0E4FE0022134601F070FA4CD2002D23
:20748000A4BF0024254647DA25F00040204318BF254D41D018E0DFF894C02CFA06F705EA92
:2074A000070C5CEA040C08BFBDE8F08100F0C6FE0022134601F052FA2ED2002D03DA4FF4CD
:2074C0008010F0400544BD43002425E0332EC8BFBDE8F081A6F1140C4FF0FF3727FA0CF72C
:2074E0003C4208BFBDE8F08101F06EFA0022134601F034FA10D2002D0DDA142E08BF6D1CB6
:2075000009D0C6F13400012101FA00F02044A04238BF6D1C0446BC4329462046BDE8F081A0
:207520009C7500883CE4377E0000F0BFFFFF0F008A68002A01DCFDF7ECBB521E8A604A6881
:20754000C0B2531C4B601070704739B1012904D181680A68406802430A60704781680A68BB
:2075600040688243F8E770B504460D461646481C1DD02846256000F01BF8606025F01F0066
:2075800000F11801E160091D216108396161A06031462046FFF7D9FF1EB1012E07D1022151
:2075A00000E003212846BDE8704000F079B870BD70B5074A054600211068012400B914600A
:2075C000284600F053F805F01F0004FA00F070BD98020010426809B1C06800E000690260F2
:2075E0007047000098B001221E496846FFF7BBFF1C490122891C06A8FFF7B5FF194901229A
:20760000C91C0CA8FFF7AFFF16490122491D12A8FFF7A9FF01216846FFF7DCFF002106A87D
:20762000FFF7D8FF00210CA8FFF7D4FF012112A8FFF7D0FF962000F07DFD00216846FFF759
:20764000C9FF012106A8FFF7C5FF01210CA8FFF7C1FF002112A8FFF7BDFF962000F06AFDB2
:20766000D8E7000032C0092000F008B910B5421C10D0094A104403090007C20E074800EBB8
:207680008300036803249440A3430360036891400B43036010BD00000040F6DF00C00240E7
:2076A000F0B5421C21D0114A114F1044420907EB820200F01F05966EC1F3800303FA05F4C1
:2076C000A6439666956E25439566002B0DD103090007C20E07EB8300036C03249440A343AE
:2076E0000364036C91400B430364F0BD0040F6DF00C0024088420BD0421C08D0491C07D053
:2077000004A10948F8F7EFFD0120FFF799FE08467047000070696E6D6170206D69732D6D5D
:2077200061746368000000005C060010421C06D1501E7047824201D1486870470C310A6831
:20774000531CF7D103A10B48F8F7CDFD0120FFF777FE000070696E6D6170206E6F7420663A
:207760006F756E6420666F72207065726970686572616C005C06001010B50446401C17D0DC
:207780000CE0A24209D189682046FFF76FFF2046BDE810400221FFF783BF0C310A68501CB3
:2077A000EFD104A10848F8F79EFD0120FFF748FE10BD0000636F756C64206E6F74207069DF
:2077C0006E6F7574000000005C0600100648016841F40071016005484FF000010172017A38
:2077E00041F0010101727047C4C00F40004002400248007AC0F30000704700000040024027
:207800000B4800B501788BB0009101790191017A0291017B0391017EA1F101010491808B3E
:20782000A0F26C7005906846FCF713FC0BB000BD2040024001B56846FCF7EAFB0E490A7866
:2078400042F002020A7002680A7642680A77826881F82020C26881F82420026902F1010278
:2078600081F83020406900F26C708886087820F00200087008BD00000840024002480068AF
:20788000C0F3000070470000F0ED00E01FB569461820ABBE04B010BD2DE9F04F83460846B0
:2078A000684ADBF80010684B87B08A180FD0B2F5804F16D0B2F50C2F3CD0B2F5102F43D085
:2078C00062A16548F8F70FFD0120FFF7B9FD03F5D473196821F0C0011960196841F0400132
:2078E00008E003F5D473196821F440711960196841F48071196059494FEA00134FF0000A4A
:2079000009680591B1FBF3F24FF0000100914FF00101019105991FFA82F803FB12110029B0
:207920006FD001F0A3FA03904FEA5806CDF81080029060E003F5D673196821F44031196068
:20794000196841F48031D5E703F5D673196821F440211960196841F48021CBE701240125FF
:2079600041E0204601F09AFA0746284601F096FA394601F0B9F94FF07E5101F047F901F06D
:2079800019F907468946304600F09BFE042201F0CAFB3A464B4600F0E3FE07468946059843
:2079A00001F07CFA01F006F93A464B4600F002FD00F012FC0146039801F00AFB039901F00D
:2079C00093F920F000473846029901F07BFA08D200952348CDE90147B046874201DA4FF094
:2079E000010A6D1CEDB2A542BBD3641CE4B20F2CB5D9761CB6B20498864202D8BAF1000F0E
:207A0000ACD0DBF80000017B41F080010173DBF800004FEA18210171DBF8001081F80080E2
:207A2000DDE9000140EA0110DBF8001081F82800DBF80000017B21F08001017307B0BDE80F
:207A4000F08F00000040FFBF00C00F4073657269616C5F62617564005C0600109402001007
:207A60006F12833A70B5012B03D0022B01D018A128E05B1E4C1F042C05D30A461BA12B487A
:207A8000F8F731FC21E0491F052A1AD2DFE802F00305080B0E00002400E00124002507E02F
:207AA0000124254604E00124022501E00124032541EA8301006841EAC40141EA051101731C
:207AC00070BD1BA11948F8F70EFC0120FFF7B8FC496E76616C69642073746F70206269748C
:207AE000732073706563696669656400496E76616C6964206E756D626572206F66206269F7
:207B00007473202825642920696E2073657269616C20666F726D61742C2073686F756C6469
:207B200020626520352E2E38000000005C060010496E76616C69642073657269616C20700C
:207B400061726974792073657474696E670000000068017D11F0010FFBD0007870470000ED
:207B60002DE9F74F044641490198FFF7DFFD3F4905466C310298FFF7D9FD01462846FFF7E9
:207B8000B9FD0646401C15D039482660351839484FF480494FF40C2A4FF4102B11D04D4557
:207BA00014D055454AD05D4515D150F8C41F41F000710FE030A13848F8F795FB0120FFF702
:207BC0003FFC50F8C41F41F0080103E050F8C41F41F01001016020680127077221684FF063
:207BE0000008C1F804804FF416512046FFF754FE0123002208212046FFF734FF1B490198ED
:207C0000FFF7BAFD194902986C31FFF7B5FD00210198FFF745FD00210298FFF741FD95B14F
:207C20004D4513D0554513D05D4501D1032060600F48404286420DD101200CE050F8C41F44
:207C400041F08071C6E7C4F80480F1E76760EFE70220ECE70020002805D010480760D4E912
:207C60000012C0E90212BDE8FE8F0000803F01000040FFBF00C00F4053657269616C207046
:207C8000696E6F7574206D617070696E67206661696C6564000000005C060010A4020010FC
:207CA0000068027D12F0200FFBD00170704710B50446FFF78BFD2046BDE81040FFF7BABD64
:207CC00070B50468656825F0020565600C1F0D2C01D2042A06D316A11A48F8F704FB0120FF
:207CE000FFF7AEFBC2F3400502F00104491E0DB1012200E0002204B1012405682E6841EAA2
:207D000082116FF30F0641EAC4113143296001684A6822F00D040BB1012200E0002244EA0F
:207D200082024A600068416841F00201416070BD53504920666F726D6174206572726F7223
:207D4000000000005C0600102DE9F04105460068426822F0020242602B4A286880182B4A43
:207D60000CD0B0F5B02F13D102F5D672106820F440601060106840F4806008E002F5D47233
:207D8000106820F440101060106840F4801010601F480224DFF87C800668084601F066F880
:207DA0000746B6FBF4F001F061F8394600F09CFF00F000FF0022434600F040FAFFF74AFB8E
:207DC00000F050FCFF2814DC29680C6129680A68114B1A400A6029680A681B1403EB0020EF
:207DE00002430A602868416841F002014160BDE8F081A41CFE2CD4DD08A11248F8F773FAB6
:207E00000120FFF71DFB00000000FDBF00C00F40940200100000E03FFF0000FF436F756C12
:207E2000646E27742073657475702072657175657374656420535049206672657175656E70
:207E4000637900005C0600102DE9FF5F8A4605469346374950460E9CFFF768FC344980460F
:207E60003C315846FFF762FC314906463C390398FFF75CFC2E49814678312046FFF756FCEA
:207E8000074631464046FFF735FC064639464846FFF730FC01463046FFF72CFC2860411C36
:207EA00007D02449401824490FD0B0F5B02F11D106E022A12848F8F716FA0120FFF7C0FA8B
:207EC00051F8C40F40F4001003E051F8C40F40F480600860601C26D0012300220821284678
:207EE000FFF7EEFE1D492846FFF72EFF2868416841F0020141600E495046FFF73DFC0C492A
:207F000058463C31FFF738FC094903983C39FFF733FC601C09D004B02046BDE8F05F0449F5
:207F20007831FFF729BC0023D7E7BDE8FF9F0000944001000000FDBF00C00F4053504920ED
:207F400070696E6F7574206D617070696E67206661696C65640000005C06001040420F00EE
:207F60000268D36813F0020FFBD091600068C16811F0040FFBD08068704710B50446FFF778
:207F800037FC10B90020FFF792FEFFF739FC002C00D0206010BD0000014901200860704741
:207FA000004009400248416921F001014161704700400940144810B50168002922D1012286
:207FC00002601248016841F40001016010484FF0000101670F494FF00203096843604FEAFC
:207FE00091010D4BB1FBF3F1A1F10101C16042600A494FF00400FEF7F1FD4FF0E0201021C7
:20800000C0F8001110BD0000B4020010C4C00F40004009409402001040420F005D80000094
:2080200070B5054672B60020C5E900120A4A146806E02368A1EB0303002B03DD2046A46878
:20804000002CF6D118B18560AC6062B670BD0846156000F055F8F7E7B802001010B5FFF7CB
:208060009BFF0D4C206870B100F018F821680A68101A00280BDC886820606268002AF1D00B
:2080800048689047EEE7BDE81040FFF78BBF0868BDE8104000F034B8B8020010044810B533
:2080A000006808B9FFF786FF0248806810BD0000B40200100040094010B572B60A4A116814
:2080C00081420DD18168116061B1086800F018F808E08A68824202D18068886002E01146A9
:2080E0000029F6D162B610BDB802001010B50446FFF760FF0148446010BD0000B8020010F9
:2081000003498861486940F001004861704700000040094010B500F04DFD0022044B00F0FF
:208120001FFB00F09FFABDE8104000F008B8000080842E414FF47A714843AFF3008070B584
:208140000446FFF7ABFF0546FFF7A8FF401BA042FAD370BD10B500290AD00878002807D0CF
:2081600005487844FBF714FF002801D0002010BD0248784410BD00007AC3000072C30000C6
:2081800010B500290AD00878002807D005487844FBF7FEFE002801D0002010BD02487844B5
:2081A00010BD0000C6C40000BEC4000010B500290AD00878002807D005487844FBF7E8FEBE
:2081C000002801D0002010BD0248784410BD0000AAC50000A2C5000021F00042A2F1605278
:2081E000B2F5801F01F0004328BFD2F17F6C0BD95FEA001C43EAC20242EB507018BF7047BB
:2082000028BF20F001007047B2F5801FBCBF184670474FEA410C1CF5001F02D2084600F011
:20822000D2BE70B500F046FB00000089FFF7F6BF4FF00040A0F580007047000010B591EA99
:20824000030F48BF83F0004300F1D283841A71EB030C05D2121943EB0C03001B61EB0C014D
:20826000DFF824E14FEA1154A4EB135C1EEA430F18BF9EEA445F73D023EA0E03DCF1200ECE
:2082800021EA045143F4801332D322FA0CFE10EB0E0023FA0CFE41EB0E01CCF1200E03FA36
:2082A0000EFE10EB0E0051F10001B1F5801FCCF1200E32D201EB045112FA0EF2BDE81040F0
:2082C00058BF7047401C38BF5FEA420218BF7047002814BF20F0010041F100014FEA4103A6
:2082E00013F5001F38BF7047A1F1C04100F030BB012A43EB0302ACF1200CDCF11F0E32BF29
:208300004FF0000E23FA0CF310EB030041EB0451B4EB115FD0D0A1EB045101F5801149080D
:208320005FEA300001EB04510ED350F1000038BF12FA0EFE08D1BDE81040C9E7401C38BF81
:208340005FEA4202CAD1C3E7BDE810404FEA410313F5001F38BF7047A1F1C04100F0F8BACF
:208360009EEA445F08D011EA5E0FBDE8104004BF01F0004100207047BDE8104070B500F0C7
:2083800099FA00BF64FBBE3E0000E0FF02494FF0000000F096BE00BF0000F87F491058BFDD
:2083A000C1F140415B1058BFC3F140438B42EFF3008070472DE9C04130B4DFF8A0C23CEA91
:2083C000111418BF3CEA131400F0EC8081EA03051CEA111444EAD57418BF1CEA131500F0EE
:2083E000C780A4EB05044FF0004545EAC12145EAC32341EA505143EA525304F17F74994293
:2084000004F500344FEAC0204FEAC22208BF904200F09C804FEA13650FF24016765D4FEA40
:20842000134506FB05F7C7F1807706FB07F74FEAD737A7FB03687642C8F58038A7FB06CE42
:2084400038BFA8F1010807FB08E64FF0000EA6FB028CE6FB03CEDCF1000CCEF1004E38BF88
:20846000AEF1010EA6FB0C584FF000074FF00005E6FB0E87A1FB08C6A0FB07CE16EB0E065A
:2084800045F10005E1FB076515F1E04E7EBFA4F580345FEA46066D4116F1800745F100058F
:2084A0004FEA17274FEA066647EA0567A6F1DE46B6F1805F4FEA15251FD9384624F0010CB8
:2084C00005EBC471BCF1FE6F01EB0C1102D8F0BCBDE8008124425CBF01F5801E9EEAC47FC8
:2084E00002D4F0BCBDE80081244238D4F0BCA1F1C041BDE8004100F02BBA4FEAD22242EA0F
:2085000043524FEAD323A7FB02864FEAD02040EA415007FB03661EEA0E0F4FEAD12105FBCE
:20852000026658BFA6EB0056B6EB00564FEA520E4EEAC37E18EB0E0E56EB530EBDD518EB76
:2085400002085E417F1C55F10005B6E74FF480154FF000074FF000064FF00008ADE7F0BC05
:208560004FF0000001F1C04101F00041BDE8008111EA0C1F0CEA131500D00CE013EA0C1F49
:2085800000F025804FF00000F0BC81EA030101F00041BDE80081F0BCBDE8004181EA030193
:2085A00000F0D6B9F0BCBDE8004170B500F082F9097EFC3E00F007B881EA03014FF00000FC
:2085C00001F00041704781EA030100F0C1B9F0BCBDE800414FF0000021497047FFFDFBF9F7
:2085E000F7F5F4F2F0EEEDEBE9E8E6E4E3E1E0DEDDDBDAD8D7D5D4D3D1D0CFCDCCCBCAC8B3
:20860000C7C6C5C4C2C1C0BFBEBDBCBBBAB9B8B7B6B5B4B3B2B1B0AFAEADACABAAA9A8A885
:20862000A7A6A5A4A3A3A2A1A09F9F9E9D9C9C9B9A999998979796959594939392919190DF
:208640008F8F8E8E8D8C8C8B8B8A8989888887878685858484838382828181800000FF0741
:208660000000F87F4FEA41034FEA5353A3F58063D3F11E03C8BFD3F1210C0CDD4FF00042E5
:2086800042EAC12242EA505232FA03FC8CEAE17CACEBE1707047102BC4BF0020704703F5D3
:2086A000787CBCF1FF3F04D06FF0004282EA2100704770B500F0FEF84992248000207047C1
:2086C000F2E7B0FA80F310FA03F10AD0C3F11D0303F580634FEA41504FEA035202EBD121E6
:2086E00070474FF00000704751EA030C17D41CF5801F58BFBCF5801F00F10680994218BF58
:20870000704708BF9042704707D711F5801F58BF13F5801F19D499427047894270471CF5FF
:20872000801F08D5BCF5801FF7D58B4218BF704708BF824270474FF4001C1CEB410F38BF57
:208740001CEB430F01D28B42704770B500F0B2F8922449004FF000514FF08053FFF71EBE37
:20876000DFF848C170B51CEA111E1EBF1CEA13159EEA0C0F95EA0C0F00F06F8081EA030426
:2087800023EA4C134EEAD47E21EA4C1141F4801143F48013AE44A1FB024CA0FB0365AEF16D
:2087A0007F7E361955EB0C05A1FB034C4CF10003A0FB021C16EB0C06654153F100030942ED
:2087C00018BF46F0010613F4007F0BD14FEA03314FEA0530340341EA155140EA16506FF091
:2087E00003020AE04FEAC3214FEAC520F40241EA555140EA56506FF0020202EB2E4201EB0C
:20880000025585EACE710AD05FEA440C18BF24F0004450F1000041F1000120EAD47040F2BD
:20882000FE7C624500D270BDA84214BF4FF080444FF04044002E08BF0024BEF1806FA8BF77
:20884000A1F1C041BDE8704080F282804FF0000001F1C04101F0004170479EEA0C0F0CEA08
:20886000131518BF95EA0C0F06D04FF0000081EA030E0EF0004170BD00F01CF88900013E96
:2088800000F007B800F009B84FEA430C5FEA5C5C08D081EA030100F05BB84FEA410C5FEAD6
:2088A0005C5CF6D14FF00000014970470000FF070000F87F0EF1020E2EF0030E5EF8046B79
:2088C000364205D4012A43EB030515F5001F12D8012841EB010C1CF5001F0CD80ED14FEA45
:2088E000D17C15F5001F0CEB4C0C0CF1020C08BF4CEBD37C04E04FF0080C01E04FEAD37CBB
:208900000CEB4C0526FA05F606F00706B6F1040C06D20EEB860CBDE870404CF0010C604792
:20892000DFE80CF0090B02024FF000414FF00000A1F5002170BD19461046012851EB01049A
:2089400018BFD4F5001484BF002001F0004170BD0808A0F500114FEA3101704753EA010C7F
:2089600017D41CF5801F58BFBCF5801F00F106808B4218BF704708BF8242704707D713F5FB
:20898000801F58BF11F5801F19D48B4270479B4270471CF5801F08D5BCF5801FF7D59942F3
:2089A00018BF704708BF904270474FF4001C1CEB430F38BF1CEB410F01D2994270470FB4AB
:2089C0000CBC03BCFFF7C1BE91EA030F10B581F000413FF53BAC83F0004300F009B8000015
:2089E00010B591EA030F48BF83F000433FF52EAC841A71EB030C07D212198CF0004C43EB57
:208A00000C03001B61EB0C01DFF8A4E14FEA1154A4EB135C1EEA430F18BF9EEA445F00F08F
:208A2000B08023EA6E03524221EA0451C3EB6E0338BF5B1EDCF1200E25D322FA0CFE10EBF1
:208A40000E0043FA0CFE41EB0E01CCF1200E03FA0EFE10EB0E0051F10001CCF1200E29D45E
:208A600012FA0EF201EB0451BDE8104058BF7047401C1CBFB2F1004F704700280CBF491CAE
:208A800020F00100704712EB020E43EB030218BF4FF0010E4EEA4202ACF1200CDCF11E0E6B
:208AA00054D943FA0CFE10EB0E0051F1FF31CCF11E0ED5D50EF1010E12FA0EFE404141EB61
:208AC000010101EB445C5FEA5C5C10D910EBDE7001EB045138BFBEF1004FBDE8104018BFD3
:208AE000704700280CBF491C20F00100704730D24FEAD42C11F5001124F400641BD0B1FA3B
:208B000081F20B3AA41AA41ED2F12003914030FA03F31943904001EBCC71002C01EB045184
:208B2000BDE81040A8BF704701F1C0414FF0000001F000417047B0FA80F310FA03F100D11B
:208B400010BDE41A173C4805C90AE4E701EB045110BD491001EB0451BDE810404FEA300006
:208B600002E04FF0000170474A0008BF0042F8D0B2F5001F28BF704701F000414FF000002C
:208B800070479EEA445F07D011EA5E0FBDE8104004BF002100207047BDE8104070B5FFF7F4
:208BA00089FE00BF40DFF63E83F00041104670470000E0FF43004FEAD30C4FEA3C0C43401D
:208BC0001FBF40070CF1605113F0FE4F70471CF0006F03D100200CF0004170470CF0004319
:208BE00043EA507010B540EACC0000F09FF900BF000000924FEA0001FFF7AABE4FF00041DC
:208C00004FF00000A1F500217047000090EA010F48BF81F0004100F1E281421A3CBF801A1F
:208C200089184FEAD0524FF07F4C1CEA410FA2EBD15318BF9CEA026F00F03B804FF0004C23
:208C40004CEA00204CEA012121FA03FC10EB0C0C1ED202F1FF325FEA1C2040EBC25038BF6C
:208C600070471CF07F0F4FEA400C18BFBCF17F4F38BF7047C3F12003994008BF20F0010096
:208C8000BCF17F4F38BF7047A0F1C04000F09BB94FEA3C00000A40EBC25028BF1CF0FF0F19
:208CA0004FEA400CE6D018BFBCF17F4F38BF7047EAE79CEA026F05D010EA5C0F08BF00F0C0
:208CC0000040704710B500F031F900BF64FBBE3E401058BFC0F14040491058BFC1F1404169
:208CE0008142EFF3008070474FF47F0C1CEAD0121EBF1CEAD11392EA0C0F93EA0C0F00F0FC
:208D0000858090EA010F48BF42F4807240F4000C41F400002CF07F4120F07F4000B58142FD
:208D2000A2EB03020FF2081CACEB504EC0F100009EF800E04FEA4E0E00FB0EFC38BF490046
:208D40004FEA2C1C02F5FA020CFB0EF34FEACE1E4FEA112C4FEAC1210EEB635E42EB224296
:208D60000EFB0CFC4FEA1C5300FB03114FEA112C4FEA01310EFB0CFC4FEADC4C00FB0C11C0
:208D8000C14228BF09184CEB03335DF804EB10EB410143EBC250B2F57C0F38BF704729D5BC
:208DA00012F0F00F1CBF00F1C04000F000407047008182838485868788898B8C8D8E8F9100
:208DC0009293959697999A9C9D9FA0A2A3A5A7A8AAACAEB0B2B3B5B7B9BCBEC0C2C5C7C939
:208DE000CCCED1D4D7D9DCDFE2E6E9ECF0F3F7FAFE0000004FEA400C0CF1807CBCF17E4F62
:208E000028BF7047B0F1C04000F0DDB890EA010F0CEAD11348BF42F48072624538BF6345B5
:208E200007D213F47F0F16D080EA010000F00040704710B500F07AF8097EFC3E00F005B8F7
:208E400080EA010000F00040704780EA010000F0004000F0B8B812F47F0F04BF024870476D
:208E600080EA010000F0AFB80000C07F10F0004148BF4042B0FA80F310FA03F2C3F19D03B7
:208E80000BD051EAC35101EB1220530638BF704700F1010008BF20F001007047B0FA80F3E5
:208EA00010FA03F2C3F19D030AD0D90501EB1220530638BF704700F1010008BF20F00100B8
:208EC0007047000050EA010C00F113801CF5000F58BFBCF5000F01D48842704707D710F5E0
:208EE000000F58BF11F5000F15D488427047894270471CF5000F04D5BCF5000FF7D5814203
:208F000070474FF0807C1CEB400F38BF1CEB410F01D28142704710B500F008F892244900BA
:208F20004FF000504FF08051FFF7D2BE0EF1020E2EF0030E5EF8044B244204D44FEA41026F
:208F4000B2F17F4F11D84FEA4003B3F17F4F0CD80ED14FEAD07CB2F17F4F0CEB4C0C0CF1C4
:208F6000020C08BF4CEBD17C04E04FF0080C01E04FEAD17C0CEB4C0324FA03F404F00704A0
:208F8000B4F1040C06D20EEB840CBDE810404CF0010C6047DFE80CF0070802024FF0004081
:208FA000A0F5800010BD0846420018BFD2F1807288BF00F0004010BD10B5FDF737FA4FF046
:208FC0000001016010BDFF2141EAD050C005704790EA010F48BF81F000413FF51EAE421ADC
:208FE00004D882F00042A0EB020011444FEAD0524FF07F4C1CEA410FA2EBD15318BF9CEA36
:20900000026F4AD04FF0004C4CEA00204CEA012121FA03FCB0EB0C0C0FD412F0FE0F36D0C7
:209020005FEA4C001DD5001240EBC25038BF70471CF03F0F18BF70470BE0A2F101025FEAFA
:209040001C2040EBC25038BF70471CF07F0F18BF7047C3F12003994014BF401E20F00100CF
:20906000704780084FEA122308BF7047B0FA80FCA2EB0C02CCF1280C60FA0CF093EA122FFF
:2090800004BF00EBC25070474FEAC3707047130A5FEADC1008BF7047F6E79CEA026F04D0BE
:2090A00010EA5C0F08BF0020704710B5FFF73EFF40DFF63E81F000407047FCF7F3B9FCF768
:2090C0007BBE0CF00F03092B08BF082000F059800A2B0BD0082B18BF704708BF1CF0400F6A
:2090E0000AD04FF000004FF0000170471CF0400F18BF4FF0004070471CF0100F08D020F0E5
:20910000704300F07F4242EAD3014FEA4370704700F0604021F07F4242EA000201F07F4008
:2091200040EA727070474FF0FF0C4CF4E06C1CEA11531CBF9CEA030C9445C2BFDA4201EB5A
:2091400002517047002B0DD0BCF1000F0FD0002A01F00041A4BF41F0E04141F07F614FF001
:209160000000704701F000414FF00000704750EA01334FF09B0C18BF4CF0806C7FF406A99B
:2091800070471CF4801F11D01CF4E02F03D06FEACC31490070474FF04050EFF3008222F0FB
:2091A000704242EA000282F3008870474FF000007047190C0C0207000000000000000000EB
:2091C0000000000000000000000000000000000200007F010000000000000000000000000D
:2091E00000000000000000000307000000070000000000000000000000000000000000005E
:2092000000072400A4017C00A7017C002700240000000000000000000000060000CE0011AE
:2092200001FF031101E2000000000000000000000000000A00000E0011001101CE003800F6
:20924000E60011011001E00000000000080000E0001E0111012901C600A00000010000007B
:209260000000000000020000070000000000000000000000000000000000000000000400E1
:2092800000F80006030104000000000000000000000000000000000301040603F8000000BF
:2092A000000000000000000000000000000000000502000A0007000A00020000000000008A
:2092C000000000000000000000060000100010007C001000100000000000000000000000CC
:2092E000000002000000070000000000000000000000000000000000000000032000200022
:2093000020000000000000000000000000000000000000000200000001000000000000002A
:20932000000000000000000000000000000380017C0003000000000000000000000000002A
:20934000000000000000060000FE00010101010101FE0000000000000000000000000006FF
:20936000000004000200FF010000000000000000000000000000000006000002018101411B
:209380000131010E010000000000000000000000000600008200010111011101EE000000EF
:2093A00000000000000000000000060000600058004600FF01400000000000000000000069
:2093C0000000000600009C000B0109010901F100000000000000000000000000060000FED6
:2093E00000110109010901F2000000000000000000000000000600000100C101390007004C
:209400000100000000000000000000000000060000EE00110111011101EE00000000000033
:20942000000000000000000600009E00210121011101FE0000000000000000000000000034
:209440000200000401000000000000000000000000000000000000000002000040070000BC
:209460000000000000000000000000000000000000000600001000280028004400440000FE
:20948000000000000000000000000006480048004800480048004800000000000000000016
:2094A0000000000006000044004400280028001000000000000000000000000000060000B8
:2094C00006000100610111000E000000000000000000000000000C0000F0010C02E2041201
:2094E0000909090909F109190902058604780207800170002E0021002E00700080010000B2
:209500000000000000000000070000FF011101110111011101FE00000000000000000000FE
:20952000000800007C008200010101010101820044000000000000000000080000FF010150
:209540000101010101010182007C000000000000000000070000FF011101110111011101B7
:20956000110100000000000000000000060000FF011100110011000100000000000000009F
:2095800000000000000800007C0082000101010111019200740000000000000000000800A1
:2095A00000FF0110001000100010001000FF010000000000000000020000FF010000000059
:2095C0000000000000000000000000000000000005C000000100010001FF000000000000C4
:2095E000000000000000000000080000FF0120001000280044008200010100000000000043
:209600000000070000FF010001000100010001000100000000000000000000080000FF0136
:2096200006007800800178000600FF010000000000000000080000FF0102000C0010006027
:20964000008000FF0100000000000000000800007C00820001010101010182007C00000080
:20966000000000000000070000FF0111001100110011000E00000000000000000000000889
:2096800000007C00820001014101410182007C010000000000000000080000FF011100111D
:2096A0000011003100D1000E010000000000000000070000CE001101110111011101E60085
:2096C0000000000000000000000007010001000100FF01010001000100000000000000007D
:2096E0000000000800007F00800000010001000180007F0000000000000000000703001C3B
:20970000006000800160001C000300000000000000000000000B07007800800170000E0060
:2097200001000E00700080017C0003000000070101C600280010002800C6000101000000B3
:209740000000000000000007010006000800F00108000600010000000000000000000000F3
:209760000700018101610111010D010301010100000000000000000000030000FF070104C9
:209780000000000000000000000000000000000000000303007C00800100000000000000C6
:2097A0000000000000000000000000020104FF07000000000000000000000000000000009C
:2097C00000000000051800060001000600180000000000000000000000000000000700043C
:2097E00000040004000400040004000400000000000000000000030000010002000000004B
:20980000000000000000000000000000000000060000C80024012401A400F8010000000093
:209820000000000000000000060000FF01880004010401F800000000000000000000000098
:2098400000050000F8000401040188000000000000000000000000000000060000F8000477
:209860000104010801FF01000000000000000000000000060000F800240124012401B800B4
:20988000000000000000000000000000040400FE01050001000000000000000000000000BB
:2098A0000000000000060000F804040504058804FC03000000000000000000000000060003
:2098C00000FF01080004000400F801000000000000000000000000020000FD01000000007F
:2098E00000000000000000000000000000000000020004FD03000000000000000000000062
:20990000000000000000000000060000FF0120003000C80004010000000000000000000024
:209920000000020000FF0100000000000000000000000000000000000000000A0000FC011E
:20994000080004000400F801080004000400F80100000000060000FC01080004000400F8EA
:2099600001000000000000000000000000060000F800040104010401F800000000000000E1
:20998000000000000000060000FC07880004010401F800000000000000000000000000062E
:2099A0000000F800040104018800FC07000000000000000000000000040000FC010800040D
:2099C00000000000000000000000000000000000000600009800240124012401C8000000B2
:2099E00000000000000000000000030400FF0104010000000000000000000000000000005B
:209A0000000000060000FC00000100010001FC01000000000000000000000000050C0070C3
:209A200000800170000C000000000000000000000000000000090C007000800170000C00A7
:209A40007000800170000C00000000000000050401D8002000D800040100000000000000BA
:209A600000000000000000050C007004800370000C00000000000000000000000000000062
:209A8000050401C40124011C0104010000000000000000000000000000032000DE030104A7
:209AA000000000000000000000000000000000000000020000FF070000000000000000009E
:209AC00000000000000000000000000400000104DE0320000000000000000000000000007C
:209AE0000000000007000020001000100020002000100000000000000000000000080000C7
:209B0000FE0102010201020102010201FE010000000000000000491817030D0000000000B0
:209B2000000000000000000000000000000000000000000000000000000000000000000025
:209B4000000000000000000000000000000000000000000000000000000000000000000005
:209B60000000000A000000000000000002000003003001000F00E003007C00001E00000217
:209B80000000000000000000000000000000000000000000000000000000000000000000C5
:209BA0000000000000000000000000000D0000000000000000000000000000004000007CDC
:209BC00000000E00000200004000007C00000E0000020000000000000000000000000000A9
:209BE000000000000000000000000000000000000000000000110000000000020098038037
:209C0000F801C07800C01E00C01F02E09903F8F801DE7800C61E00C21F00E01900F81800C3
:209C2000DE0000C6000002000000000000000000000000000000000000000000000010006E
:209C4000000000000000000000F00100F003E0800BF801079CC3030C3B03068701E687010D
:209C60001EC600077E000E3C003E00003C00000000000000000000000000000000000000B7
:209C80000000000000000016000000000000000000000000000004000004E00106F8830341
:209CA0001CC201066200823100E218007E0C001CC60380F307C03904600C0430040318E427
:209CC000010CFC000610000200000000000000001100000000000000C00000F00100F803A6
:209CE000000C03000603600203F80303DC87018C8F01C6FC00C6F0006EF0033E98011C0C91
:209D0000010004000000000000000000000000000000000000000000000900000000000035
:209D20000000000000000000004000007C00000E0000020000000000000000000000000057
:209D4000000000000000000000000000000000000000000000000000000000000000000003
:209D60000000170000000000000000000000000000000000000000000000000000000000CC
:209D80000000000000000000000000000000F81F001F3C800310E000003000001800000C8A
:209DA00000000600000300000000000900001800000C00000600000300C00102F0000F3E64
:209DC00000FE0F006000000000000000000000000000000000000000000000000000000016
:209DE00000000000000000000000000000000000000000000E000000000000000000000055
:209E000000000000900000D800005800003000003C0000FE000052000018000008000000A6
:209E2000000000000000000000000000000000000000000000000000000000000010000012
:209E40000000000000000000040000060000060000060000C60000FE00003F00E00700F012
:209E60000600100600000600000600000600000000000000000000000000000000000000B4
:209E80000000000000000500000000001000000A000007000001000000000000000000009B
:209EA0000000000000000000000000000000000000000000000000000000000000000000A2
:209EC000000000000000000000000000000000090000000000000000000018000018000049
:209EE000180000180000180000180000000000000000000000000000000000000000000002
:209F000000000000000000000000000000000000000000000000000005000000000000003C
:209F200000020000030000010000000000000000000000000000000000000000000000001B
:209F4000000000000000000000000000000000000000000000000000000000000000000001
:209F6000000D00000200000300C00100F000003800000E00000700C00100E00000380000F8
:209F80001E000006000002000000000000000000000000000000000000000000000000009B
:209FA000000000000000000000001100000000000000000000F80100FF03C08703F0000358
:209FC0003800030C00030C800106C00106E0000638008E1F00FC0700780000000000000097
:209FE000000000000000000000000000000000000000001100000000000000000000000050
:20A0000000000000000000000060000220C00330F801103F00E80700FC00001E0000020078
:20A0200000000000000000000000000000000000000000000000000000000000110000000F
:20A0400000000200000300800300C0032060033030031830030C1803040C03060C03060629
:20A0600003060301860100FE00007C000000000000000000000000000000000000000000D2
:20A0800000000000001100000000000000400000E00100E0032000033000031800030C032B
:20A0A0000306030106830186E700867E00FE1C007C000010000000000000000000000000F2
:20A0C000000000000000000000000000000011000000002000003000003800003C00003675
:20A0E00000003300803100C0300260F00330F801183F00EC3700FC30001E00000200000048
:20A100000000000000000000000000000000000000000000000000110000000000000040EE
:20A120000000E00100E103C00103F00103BE0003CE0003C68001C6C001C6E100C67F0086D0
:20A140001F00060200060000020000000000000000000000000000000000000000000000D0
:20A160001100000000000000000000F80100FF01C08703F002033803039C01038C81018624
:20A18000810186E300867F00061F001E00001C000018000000000000000000000000000058
:20A1A0000000000000000000001100000000000000000000000200800300E00104700006AE
:20A1C0003C00060E00060700860100C600006600003600001E00000E000006000002000005
:20A1E0000000000000000000000000000000000000001100000000000000C00000F8010095
:20A20000FC03000C03E00603F803039C03030C830106830106E700867F00FE3C007C0000E5
:20A22000080000000000000000000000000000000000000000000000000000110000000005
:20A24000000000C00100C001008103E00703F00F03180C030C0C030C8C0106C400066600FB
:20A26000063A008E1F00FC0700F800000000000000000000000000000000000000000000F6
:20A28000000000000A000000000000000002000003000001800000C00000C00000000000AE
:20A2A00000000000000000000000000000000000000000000000000000000000000000009E
:20A2C000000000000000000000000000000800000000001000000A000007000001800000D4
:20A2E000C00000C000000000000000000000000000000000000000000000000000000000DE
:20A3000000000000000000000000000000000000000000000000110000000000000000002C
:20A32000000000000000000700000F00000D00801D00801900C03800C030004070006020AC
:20A3400000600000300000100000000000000000000000000000000000000000000000104D
:20A36000000000000000000000000000001800801800C01800C01800C01800C01800C018F5
:20A3800000C01800C01800C01800C00000C0000000000000000000000000000000000000B5
:20A3A00000000000000000000F000000000000000000004000002000003000203000701826
:20A3C00000601800E01800C00C00C00D008005008007000007000000000000000000000061
:20A3E00000000000000000000000000000000000001000000000000000000000000000004D
:20A40000002000023020031838010C3C00040C00060600060300060100860100FE00007C01
:20A4200000000000000000000000000000000000000000000000000000001700C00300F84A
:20A440000F003E1E000738800130C0C07060F87130BC631806631803638C01618C8161C47A
:20A460008060C6C063C6E063C67933861F33868711C68118CEC0080C700CFC3F04F00F00E7
:20A480000000000F00000200000300C00100E000003800001C00001E00801B00C0190060C1
:20A4A00018003818001C1800061800FEFF03FEFF03000000000000000000000000000000E2
:20A4C0000000000000000000000000001000000000000200C00300F803003F03E00703FC84
:20A4E00003031E030306030306030306030106830106C700867E00FE3C003C00000000003F
:20A500000000000000000000000000000000000000000000001100000000780000FF01C0F2
:20A52000C701E080033000031800030C00030C000306800106800106C00006E00006300094
:20A540001E10007C00007800000000000000000000000000000000000000000000001200C7
:20A56000000000000200C00300F803003F03E00703FC00031E000306000306000306800136
:20A5800006800106C0000660000E38009E1F00FC0700700000000000000000000000000092
:20A5A000000000000000001400000000000000000200C00300F803003F03E00703FC030399
:20A5C0001E03030603030603030603030603030603030603010603000600000600000600F6
:20A5E000000200000000000000000000000000001300000000000000000200C00300F80188
:20A60000003F00E00700FC03001E03000603000603000603000603000603000603000600B8
:20A620000006000006000002000000000000000000000000000000000014000000000000F8
:20A6400000380000FF00C0E701E080013080031800031800030C00030C000306040306861A
:20A660000106860106860106C6000EFE001E3E007C06007800000000000000000000000091
:20A6800000001400000000000000000200C00300F801003F00E00700FC03001E030002039D
:20A6A0000000030000030000030200C30300FB01003F00E00700FC00001E0000020000008B
:20A6C00000000000000000000000000A00000000000000000200C00300F801003F00E0078C
:20A6E00000FC00001E0000020000000000000000000000000000000000000000000000003E
:20A7000000000000000000000000000000000000000000000F00000000000000C00100E089
:20A720000300A00300000300000300800100C001007800001F00E00700FC00001E00000291
:20A740000000000000000000000000000000000000000000000000000000000000150000E4
:20A760000000000000000200C00300F801003F00E00F00FC0C001E0600020300800F0080AD
:20A780001D00C0780060E0013080031000021800000C000006000002000002000000000030
:20A7A0000000000000000D00000000000000000200C00300F803003F03E00703FC00031E83
:20A7C00000030200030000030000030000010000000000000000000000000000000000006A
:20A7E0000000000000000000000000000000001700000000000000000200C00300F8010084
:20A800003F00E00700FC00001EF003FEFF03FE8F0300C001007000003800000E0080070275
:20A82000C0C10370F801383F00EE0700FE00001E000002000000000014000000000000008D
:20A84000000200C00300F801003F00E00700FC00001E0000FE0000F80F0000FF0100F00302
:20A8600000C00300F801003F00E00700FC00001E00000200000000000000000000000000DA
:20A88000001400000000000000380000FF00C0C301E080033000031800030C00030C00031A
:20A8A00004000306800106800106C00006C0000670000E38003C0E00F80700E00100000011
:20A8C000000000000000000000001200000000000000000200C00300F801003F00E0070082
:20A8E000FC06001E0600060600060600060600060600060600060300860300FE01007C00E9
:20A90000000000000000000000000000000000000000001400000000000000380000FF00EC
:20A92000C0E701E080033000031800030C00030C400304600306C00106C00106C00306603C
:20A94000070670020E38003C0E00F80700E0010000000000000000000000000013000000F5
:20A9600000000000000200C00300F801003F00E00700FC03001E03000603000603000603B8
:20A9800000060F00067F0006FB03868103860100FE00007C0000000000000000000000000E
:20A9A00000000000001000000000000000F00100F001008003E00003F801039C03030C0392
:20A9C0000306030306830106870106C600067E003E3C003C0000000000000000000000004A
:20A9E00000000000000000000000000000001100000000000004000006000206C00306F873
:20AA000001063F00E60700FE00001E000006000006000006000006000006000006000002C1
:20AA200000000000000000000000000000000000000000000000001200000000000000F80C
:20AA40000100FF03E00703FC00031E000302000300000300000300800100E0000078000005
:20AA60001F00E00700FC00001E0000020000000000000000000000000000000000000000B4
:20AA800011000000000000FEFF03FEFF0300000300C00100E000003800001C000007008026
:20AAA0000300C001007000003800000E000006000002000000000000000000000000000014
:20AAC0000000000000000000001800000000000000E003F0FF03FEFF030EC001007000004A
:20AAE0003800000E00000700C00100E000003800001CC003FEFF03FEBF031EC00100700042
:20AB0000003800000E00800700E001007800001E0000160000020000020000030080010053
:20AB2000C0000060000030000638001E1800FC0C00E00700801F00807D00C0F00160C003F2
:20AB40003000023000001800000C0000060000020000020000000000000000120000000053
:20AB600000000600003E0002F8C003E0FB01803F00000600000300800100C000006000008F
:20AB80003000001800000C0000060000020000020000000000000000000000000000000057
:20ABA000000000001400000200800300C003006003006003003003041803060C03060C03F7
:20ABC000060603060303860103860103C600036600013600003600001E00000E000002007C
:20ABE000000000000000000000000000000C00007800007E00C06700F861003F20E007008D
:20AC0000FC00001E0000060000060000060000020000000000000000000000000000000006
:20AC200000000000000000000000000000000000000000000000080000000000000000000C
:20AC400000000000000080FF03FEFF037E00000000000000000000000000000000000000F4
:20AC6000000000000000000000000000000000000000000000000000000000000000000BC9
:20AC800000006000006000007800003E00C00704F801063F00E60700FE00001E000002002A
:20ACA000000000000000000000000000000000000000000000000000000000000000000094
:20ACC00000000000000000000D000000000000000000000000000200800300C001006000C1
:20ACE000003800001C00000E0000FE0300FC030000000000000000000000000000000000F2
:20AD000000000000000000000000000000000000001500006000006000006000006000009E
:20AD20006000006000006000006000006000006000006000006000006000006000006000F3
:20AD400000600000600000600000600000600000200000000000000000000A0000000000E9
:20AD6000000000000000000000000000000000000600000E00000E000000000000000000B1
:20AD80000000000000000000000000000000000000000000000000000000000000000000B3
:20ADA0000000000E00000000000000C00100F003003203001B03801903C01801C09801C0F0
:20ADC0008C00C0EC03C0FC03C03F00800700000000000000000000000000000000000000F3
:20ADE0000000000000000000000000000D00000000000200C00300F80100BF01E00703FCE2
:20AE000001039E0103C20001C08001C0C000C07900801F0000000000000000000000000030
:20AE20000000000000000000000000000000000000000000000C00000000000000F801000D
:20AE4000FE03000703800103800003C08001C0C001C04100C00300800300000000000000D7
:20AE60000000000000000000000000000000000000000000000000000000000000001000C2
:20AE8000000000000000F80100DE03000303800103800003C08001C08002C0E003C0FF01E5
:20AEA000003F00E00700FC00001E0000020000000000000000000000000000000000000050
:20AEC000000000000000000D00000000000000F80100FE03000F03800D03800C03C00C036B
:20AEE000C08C01C0CC00C04D00800F000003000000000000000000000000000000000000DA
:20AF0000000000000000000000000000000000000E00000000000000000280C003C0F80125
:20AF2000C03F00E00700F80000DC0000C60000C600000600000600000200000000000000BD
:20AF4000000000000000000000000000000000000000000000000000000F0000100000389A
:20AF600000007800F86100FE63000763800163800133C00039C0801EC0E00780FD01003FE2
:20AF800000C00700C00000000000000000000000000000000000000000000000000000002A
:20AFA00000000E00000000000200C00300F801003F00E00700FC01009E0100C20000C00081
:20AFC00002C0C003C0F901C03F0080070000000000000000000000000000000000000000AC
:20AFE00000000000000000000000000900000000000200C00300F801003F00C00700C400C0
:20B00000000600000200000000000000000000000000000000000000000000000000000028
:20B0200000000000000000000000000000000000000000000900003800001E00C00700F8F2
:20B0400001003F00C00700C40000060000020000000000000000000000000000000000001D
:20B0600000000000000000000000000000000000000000000000000000000000000F0000C1
:20B080000000000200C00300F801003F00E01F00FC18001E3C0002E60100C2030003028013
:20B0A0000100C000004000004000000000000000000000000000000000000000000000004F
:20B0C0000000000000000900000000000200C00300F801003F00E00700FC00001E00000267
:20B0E000000000000000000000000000000000000000000000000000000000000000000050
:20B100000000000000000000000000000000001400000000000200C00300F801003F00C05E
:20B120000700C00100800000C00002C0C003C0F801C03F00800700800100800000C0000280
:20B14000C0C003C0F801C03F008007000000000000000000000000000E000000000002001D
:20B16000C00300F801003F00C00700C00100800100C00000C00002C0C003C0F901C03F000D
:20B18000800700000000000000000000000000000000000000000000000000000000000028
:20B1A000000E00000000000000000000F80100DE03000303800103800003C00001C0800198
:20B1C000C0C000C07900801F00000700000000000000000000000000000000000000000010
:20B1E000000000000000000000000E00007800003E00C00700F80100FF03C00703C001033B
:20B20000800003C00001C08001C0E000C07F00801F00000300000000000000000000000028
:20B22000000000000000000000000000000000000000000E00000000000000F80100FE0306
:20B24000000703800103800043C00071C0803EC0E00780FF01003F00C00700C00000000001
:20B26000000000000000000000000000000000000000000000000000000000000C000000C2
:20B2800000000200C00300F801003F00C00700C00100800000C00000C00000C00000400029
:20B2A00000000000000000000000000000000000000000000000000000000000000000008E
:20B2C00000000000000D00000000000000C00100C003008F03800F03801D03C01803C098E6
:20B2E00001C0F801C0F100C00300800300000000000000000000000000000000000000009D
:20B3000000000000000000000000000000000A00000000000080C003C0F803C03F03E0073C
:20B3200003F80000DC0000C00000C0000000000000000000000000000000000000000000B6
:20B3400000000000000000000000000000000000000000000000000F00000000000000C01E
:20B360000100F80300BF03C00703C0000300000100800100800200E00300F801003F00C0A3
:20B380000700C00000000000000000000000000000000000000000000000000000000000E6
:20B3A0000D000000000000C0FF03C0FF0300800300C001007000003800001C00000700806D
:20B3C0000300C000004000000000000000000000000000000000000000000000000000006A
:20B3E0000000000000000000001400000000000000F003C0FF03C09F0300C00100700000F1
:20B400003800000E00800700C0FD03C0FF03C09F0300C001007000003C00000E008003007D
:20B42000C00100400000000000000000000000000000100000020000020000030080014033
:20B44000C000C06100C03700001F0000780000EC03008603000302800100C000004000007F
:20B460004000000000000000000000000000000000000000000000000000000F000060001D
:20B480000060000060000038C0FF1FC0FF0700F80300C001007000003800000E0000070097
:20B4A000800300C00000400000000000000000000000000000000000000000000000000009
:20B4C000000000000F00000200000300800380C003C06003C02003C03003C01803C00C03EF
:20B4E000C00403C00603C00301C00100C00000C000000000000000000000000000000000B7
:20B50000000000000000000000000000001800000000000000000000000000000000000013
:20B5200000000000000000000000000000000000000000000000000000081E00FC3F00FEAC
:20B5400010000300E001007800000C00000600000300000200000A00004000007800003E68
:20B5600000C00700F801003F00E00700FC00001E00000200000000000000000000000000C9
:20B580000000000000000000000000000000000000000000000000000000000000000008A3
:20B5A00000001000000800000F00C003007000821B00F70F003E040000000000000000004C
:20B5C00000000000000000000000000000000000000000000000000000000000000000006B
:20B5E00000000000000000000F00000000000000000000000000040000060000030000032C
:20B60000000003000007000007000006000006000006000003000000000000000000000004
:20B62000000000000000000000000000000000000001000000000000000000000000000009
:20B640000000000000000000000000000000000000000000000000000000000000000000EA
:20B660000000000000000000000000000000000000000000000000000000711C1C040F000E
:20B680000000000000000000000000000000000000000000000000000000000000000000AA
:20B6A00000000000000000000000000000000000000000000000000000000000000000008A
:20B6C00000000000000000000000000000000000000000000000000000000000000000006A
:20B6E000000000000000000000000000000000050000000000000000FE3F3800FE7F38001B
:20B70000FE3F380000000000000000000000000000000000000000000000000000000000B4
:20B72000000000000000000000000000000000000000000000000000000000000000000009
:20B740000000000000000000000000000000000000000000000000000000000000000000E9
:20B7600009000000007E000000FE0000007E00000000000000000000007E000000FE00004A
:20B78000007E0000000000000000000000000000000000000000000000000000000000002B
:20B7A000000000000000000000000000000000000000000000000000000000000000000089
:20B7C00000000000000000000000000000000000000F80C1000080C1380080C13F0080FFA1
:20B7E0000700F8FF0000FEC100008EC1000080C1000080C1380080C13F0080FF0700F8FF86
:20B800000000FEC100008EC1000080C10000000000000000000000000000000000000000D9
:20B82000000000000000000000000000000000000000000000000000000000000000000008
:20B8400000000F00000000F0810300F8830F00FC871F000C071E00060E3800060E3000FF79
:20B86000FFFF01FFFFFF01061C30000E1C38001C381C007CF81F0078F00F0060C00300007A
:20B880000000000000000000000000000000000000000000000000000000000000000000A8
:20B8A00000000000000000000000000000000000000000180000000000000000F00100007F
:20B8C000FC0700000E0E0000060C0000060C4000060C70000E063C00FC070F00F08103008D
:20B8E00000E0010000780000001E000080070000C0810F00F0E03F003C7070000E30600031
:20B9000002306000003060000070700000E03F0000800F0000000000000000000000000077
:20B9200000000000130000000000C0030000F00F0070F81F00FC391C00FC0F38000E0F30CA
:20B9400000060E3000061E30000E3B3800FE731800FCE11C0078C00F0000C0070000F00747
:20B960000000F00F0000301C00000038000000100000000000000000000000000000000034
:20B9800000000000000000000000000000000000000000000004000000007E000000FE0027
:20B9A00000007E000000000000000000000000000000000000000000000000000000000009
:20B9C000000000000000000000000000000000000000000000000000000000000000000067
:20B9E000000000000000000000000000000000000000000000000000000000000000000047
:20BA0000000000000000140000000000000000000000000000000000000000000000000012
:20BA200000000000000000000000000000000000000000000000000000000000FC03008087
:20BA4000FF1F00E0037C007800E0011C0080030E0000070400000200000000000000000056
:20BA60000000000000000000000000000000000000000000000000051C0080037800E001C9
:20BA8000E0037C0080FF1F0000FC03000000000000000000000000000000000000000000AA
:20BAA000000000000000000000000000000000000000000000000000000000000000000086
:20BAC000000000000000000000000000000000000000000000000000000000000000000066
:20BAE00000000000000000000A1000000018010000B0030000F0010000FE000000FE000073
:20BB000000F0010000B0030000180100001000000000000000000000000000000000000058
:20BB2000000000000000000000000000000000000000000000000000000000000000000005
:20BB4000000000000000000000000000000000000000000000000000000F000000000018BE
:20BB600000000018000000180000001800000018000000180000E0FF0700E0FF0700001869
:20BB800000000018000000180000001800000018000000180000000000000000000000002D
:20BBA000000000000000000000000000000000000000000000000000000000000000000085
:20BBC0000000000000000000000005000000000000000000003802000038030000F80000F3
:20BBE000000000000000000000000000000000000000000000000000000000000000000045
:20BC0000000000000000000000000000000000000000000000000000000000000000000024
:20BC20000000000000000000000000000000000000000000000000000000000900000000FB
:20BC400000E0000000E0000000E0000000E0000000E0000000E0000000E0000000E00000E4
:20BC60000000000000000000000000000000000000000000000000000000000000000000C4
:20BC80000000000000000000000000000000000000000000000000000000000000000000A4
:20BCA0000000000000000000000000000500000000000000000000380000003800000038D7
:20BCC000000000000000000000000000000000000000000000000000000000000000000064
:20BCE000000000000000000000000000000000000000000000000000000000000000000044
:20BD000000000000000000000000000000000000000000000000000000000000000800001B
:20BD2000300000003E0000E00F0000FC0100C01F0000F80300003E0000000600000000008B
:20BD40000000000000000000000000000000000000000000000000000000000000000000E3
:20BD60000000000000000000000000000000000000000000000000000000000000000000C3
:20BD800000000000000000000000000000000F0000000080FF0100F0FF0700F8FF0F007C9C
:20BDA000001F001E003C000E0038000E0038000E0038001E003C007C001F00F8FF0F00F04D
:20BDC000FF0700C0FF0100000000000000000000000000000000000000000000000000009D
:20BDE000000000000000000000000000000000000000000000000000000000000000000F34
:20BE00000000000000000000C0010000E0000000E00000007000000038000000FCFF3F00BF
:20BE2000FEFF3F00FEFF3F000000000000000000000000000000000000000000000000008A
:20BE40000000000000000000000000000000000000000000000000000000000000000000E2
:20BE6000000000000000000000000000000000000F000000006000300078003C007C003EB5
:20BE8000001C003F000E803B000EC039000EE038000E7038000E3C38001E1E3800FC0F3862
:20BEA00000F8033800F0013800000000000000000000000000000000000000000000000026
:20BEC000000000000000000000000000000000000000000000000000000000000000000062
:20BEE000000F000000006000030078000F007C001F001C001E000E003C000E1C38000E1C9E
:20BF000038000E1C38001E1E3C00FC3F1C00F8F31F00F0F10F0000C00300000000000000FB
:20BF2000000000000000000000000000000000000000000000000000000000000000000001
:20BF40000000000000000000000000000000000000000F00E0010000F0010000F801000007
:20BF6000CE010000C70100C0C30100E0C0010070C001001CC00100FEFF3F00FEFF3F00FE81
:20BF8000FF3F0000C0010000C0010000C00100000000000000000000000000000000000020
:20BFA000000000000000000000000000000000000000000000000000000000000000000081
:20BFC0000000000F00000000001C0300F01F0F00FE1F1F00FE0E1E000E0638000E07380016
:20BFE0000E0738000E0738000E0F3C000E1E1E000EFE1F000EFC070000F0030000000000D5
:20C00000000000000000000000000000000000000000000000000000000000000000000020
:20C0200000000000000000000000000000000000000000000F0000000080FF0100F0FF077B
:20C0400000F8FF0F007C381E001C1C3C000E0E38000E0E38000E0E38000E1E3C001E3E1EB6
:20C06000003CFC1F0038F80F0030E003000000000000000000000000000000000000000017
:20C080000000000000000000000000000000000000000000000000000000000000000000A0
:20C0A00000000000000F000000000E0000000E0000000E0000000E003C000EC03F000EF8EA
:20C0C0003F000EFE03008E3F0000CE070000FE0100007E0000001E0000000E0000000000C7
:20C0E000000000000000000000000000000000000000000000000000000000000000000040
:20C10000000000000000000000000000000000000000000000000F0000000000C00700F059
:20C12000E10F00F8F71F00FC371C001E1E3C000E1C38000E1C38000E1C38001E3E3800FC84
:20C14000371C00F8F71F00F0E10F0000C007000000000000000000000000000000000000D7
:20C160000000000000000000000000000000000000000000000000000000000000000000BF
:20C18000000000000000000F00000000E0030600F80F0E00FC1F1E003C3E3C001E3C380011
:20C1A0000E3838000E3838000E3838001E1C1C003C0E1F00F8FF0F00F0FF0700C0FF00008B
:20C1C00000000000000000000000000000000000000000000000000000000000000000005F
:20C1E00000000000000000000000000000000000000000000000000005000000000000003A
:20C200000080033800800338008003380000000000000000000000000000000000000000ED
:20C220000000000000000000000000000000000000000000000000000000000000000000FE
:20C240000000000000000000000000000000000000000000000000000000000000000000DE
:20C2600000000000000000000005000000000000000080033802800338038003F8000000C3
:20C2800000000000000000000000000000000000000000000000000000000000000000009E
:20C2A00000000000000000000000000000000000000000000000000000000000000000007E
:20C2C00000000000000000000000000000000000000000000000000000000F00000000004F
:20C2E000080000001C0000001C00000036000000360000006300000063000080C10000800B
:20C30000C10000C0800100C0800100600003006000030030000600000000000000000000DE
:20C320000000000000000000000000000000000000000000000000000000000000000000FD
:20C3400000000000000000000000000F0000000080C1000080C1000080C1000080C10000CA
:20C3600080C1000080C1000080C1000080C1000080C1000080C1000080C1000080C10000B5
:20C3800080C1000080C100000000000000000000000000000000000000000000000000001B
:20C3A000000000000000000000000000000000000000000000000000000000000F0000006E
:20C3C00000300003006080010060800100C0800100C0C0000080C100008061000000630022
:20C3E00000006300000036000000360000001C0000001C000000180000000000000000001E
:20C4000000000000000000000000000000000000000000000000000000000000000000001C
:20C42000000000000000000000000000000E0000000060000000780000007C0000001C007E
:20C4400000000E00000006C0390006F03900067838000E3C00001C0E0000FC070000F80378
:20C460000000F00100000000000000000000000000000000000000000000000000000000CB
:20C480000000000000000000000000000000000000000000000000000000000000001C0080
:20C4A0000000000000000000F8070000FE3F0080077800E001E0007000C00138E087031895
:20C4C000F80F071CFE1F060C1F3C060E07300E8603300C8601300C8601180C86010C0C0677
:20C4E000031F0C06FF3F0C86FF3F0C8CFF310C8C0730041C0018063800180670000E03E06E
:20C50000810703C0FF8101007EC00000004000130000300000003C0000803F0000E00F00A4
:20C5200000FC030000FF0000E0FF0000F8E300007EE000000EE000007EE00000F8E30000BE
:20C54000E0FF000000FF000000FC030000E00F0000803F0000003C000000300000000000E4
:20C560000000000000000000000000000000000000000000000000000000000000000000BB
:20C58000110000000000000000FEFF3F00FEFF3F00FEFF3F000E1C38000E1C38000E1C38B0
:20C5A000000E1C38000E1C38000E1C38000E1C38001E1E3800FC3F1C00F8F31F00F0E10F3E
:20C5C0000000C0070000000000000000000000000000000000000000000000000000000094
:20C5E00000000000000000000000000000000000001300000000007F0000E0FF0300F0FFD8
:20C600000700F8800F003C001E001C001C001E003C000E0038000E0038000E0038000E00C0
:20C6200038000E0038001E003C001C001E007C000F00F8C00F00F0C0030040800000000023
:20C640000000000000000000000000000000000000000000000000000000000000000000DA
:20C660000000130000000000000000FEFF3F00FEFF3F00FEFF3F000E0038000E0038000E59
:20C680000038000E0038000E0038000E0038000E0038000E0038001E001C003C001E00F878
:20C6A000800F00F0FF0700E0FF0300807F0000000000000000000000000000000000000014
:20C6C00000000000000000000000000000000000000000110000000000000000FEFF3F000D
:20C6E000FEFF3F00FEFF3F000E1C38000E1C38000E1C38000E1C38000E1C38000E1C380076
:20C700000E1C38000E1C38000E1C38000E1C38000E1C38000E0038000000000000000000E9
:20C720000000000000000000000000000000000000000000000000000000000000000000F9
:20C7400000000000100000000000000000FEFF3F00FEFF3F00FEFF3F000E1C00000E1C00C1
:20C76000000E1C00000E1C00000E1C00000E1C00000E1C00000E1C00000E1C00000E000085
:20C78000000E0000000000000000000000000000000000000000000000000000000000008B
:20C7A0000000000000000000000000000000000000000000001500000000007F0000C0FF26
:20C7C0000100F0FF0700F8800F0078000F003C001E001C001C000E003C000E0038000E0024
:20C7E00038000E0038000E3838000E3838000E3838001E383C001C381C007C381C00F8F87F
:20C800000F00F0F80F0040F8070000000000000000000000000000000000000000000000D3
:20C82000000000000000120000000000000000FEFF3F00FEFF3F00FEFF3F00001C00000016
:20C840001C0000001C0000001C0000001C0000001C0000001C0000001C0000001C000000F8
:20C860001C0000FEFF3F00FEFF3F00FEFF3F000000000000000000000000000000000000E8
:20C88000000000000000000000000000000000000000000000000005000000000000000093
:20C8A000FEFF3F00FEFF3F00FEFF3F000000000000000000000000000000000000000000C4
:20C8C000000000000000000000000000000000000000000000000000000000000000000058
:20C8E000000000000000000000000000000000000000000000000000000000000000000038
:20C9000000000000000000000C000000000000070000001F0000001F0000003C0000003852
:20C9200000000038000000380000003C00FEFF1F00FEFF0F00FEFF0700000000000000001F
:20C940000000000000000000000000000000000000000000000000000000000000000000D7
:20C960000000000000000000000000000000000000000000000000000013000000000000A4
:20C980000000FEFF3F00FEFF3F00FEFF3F0000380000001C0000000E0000000F0000803FB3
:20C9A0000000C0790000E0F0000070C00100388007001C000F000E001E00060038000200E7
:20C9C000300002002000000000000000000000000000000000000000000000000000000005
:20C9E000000000000000000000000F0000000000000000FEFF3F00FEFF3F00FEFF3F000074
:20CA0000003800000038000000380000003800000038000000380000003800000038000056
:20CA2000003800000038000000000000000000000000000000000000000000000000000086
:20CA40000000000000000000000000000000000000000000000000000000001500000000C1
:20CA600000000000FEFF3F00FEFF3F00FEFF3F003E000000FE030000F03F000080FF07000E
:20CA800000F83F0000803F000000380000803F0000F83F0000FF0300F03F0000FE03000040
:20CAA0003E000000FEFF3F00FEFF3F00FEFF3F000000000000000000000000000000000084
:20CAC000000000000000000000000000120000000000000000FEFF3F00FEFF3F00FEFF3F90
:20CAE000007C000000F8000000E003000080070000001F0000007C000000F0000000E003EA
:20CB0000000080070000001E00FEFF3F00FEFF3F00FEFF3F000000000000000000000000BC
:20CB20000000000000000000000000000000000000000000000000000000000000150000E0
:20CB40000000007F0000C0FF0100F0FF0700F8800F003C000F001C001C001C001C000E0050
:20CB600038000E0038000E0038000E0038000E0038000E0038001C001C001C001C003C0073
:20CB80001E00F8800F00F0FF0700C0FF0100007F00000000000000000000000000000000BB
:20CBA0000000000000000000000000000000110000000000000000FEFF3F00FEFF3F00FEEE
:20CBC000FF3F000E1C00000E1C00000E1C00000E1C00000E1C00000E1C00000E1C00000EE3
:20CBE0001E00001E0E0000FC0F0000F8070000F003000000000000000000000000000000EE
:20CC00000000000000000000000000000000000000000000000000000000000000000015FF
:20CC200000000000007F0000C0FF0100F0FF0700F8800F003C000E001C001C001C001C007E
:20CC40000E0038000E0038000E0038000E003A000E003B000E003E001C001E001C001C00B3
:20CC60003C001F00F8803F00F0FF7700C0FF7100007F20000000000000000000000000006D
:20CC800000000000000000000000000000000000150000000000000000FEFF3F00FEFF3F07
:20CCA00000FEFF3F000E1C00000E1C00000E1C00000E1C00000E1C00000E1C00000E3C00F2
:20CCC000000E7C00000EFC00001EDE01001ECE0300FC8F0F00F8071E00F0033C00000038B6
:20CCE000000000200000000000000000000000000000000000000000000000000000000014
:20CD000000110000000000800300F0810700F8830F00FC071E001C071C000E0E3C000E0EA9
:20CD200038000E0E38000E1C38000E1C38001E1C38001C383C007C781C0078F81F0060F0B2
:20CD40000F0000C00300000000000000000000000000000000000000000000000000000001
:20CD6000000000000000000000000000000000000000110E0000000E0000000E0000000E6A
:20CD80000000000E0000000E0000000E000000FEFF3F00FEFF3F00FEFF3F000E0000000E99
:20CDA0000000000E0000000E0000000E0000000E0000000E0000000000000000000000002D
:20CDC000000000000000000000000000000000000000000000000000000000000000000053
:20CDE000000000120000000000000000FEFF0100FEFF0700FEFF0F0000001F0000003C00B8
:20CE000000003800000038000000380000003800000038000000380000001C0000001E0088
:20CE2000FEFF0F00FEFF0700FEFF01000000000000000000000000000000000000000000E4
:20CE4000000000000000000000000000000000000000000013020000001E000000FE0000A1
:20CE600000FC070000E03F000000FF010000F80F0000C03F0000003F000000300000003EDD
:20CE80000000C03F0000F80F0000FF0100E03F0000FC070000FE0000001E0000000200004C
:20CEA000000000000000000000000000000000000000000000000000000000000000000072
:20CEC00000000000001B0E000000FE010000FE3F0000E0FF070000FE3F0000C03F000000CB
:20CEE000380000803F0000F83F0080FF0700F07F0000FE0700007E0000000E000000FE017F
:20CF00000000FE3F0000F0FF070000FF3F0000E03F000000380000803F0000F83F0080FFD4
:20CF20000700F87F0000FE0700007E0000000600000000000000130000200002003000067F
:20CF4000003C001E001E003C000F0078C00700F0E10100C0FB0000803F0000001E000080E5
:20CF60003F0000C0FB0000F0E1010078C007003C000F001E001E0006003C000200300000AB
:20CF8000002000000000000000000000000000000000000000000000000000000000000071
:20CFA0000000000000000013020000000E0000001E0000003C000000F8000000E00100001B
:20CFC000C0070000000F000000FE3F0000F83F0000FC3F00001F000080070000E003000043
:20CFE000F00000007C0000001E0000000E0000000200000000000000000000000000000097
:20D00000000000000000000000000000000000000000000000000000110000000000003CC3
:20D02000000E003E000E003F000E803B000EC039000EF038000E7838000E3C38000E1E38AD
:20D04000000E0738008E033800CE013800EE0038007E0038003E0038001E0038000000000B
:20D060000000000000000000000000000000000000000000000000000000000000000000B0
:20D080000000000000000000000700000000FEFFFF0FFEFFFF0FFEFFFF0F0E00000E0E003E
:20D0A000000E0E00000E000000000000000000000000000000000000000000000000000046
:20D0C000000000000000000000000000000000000000000000000000000000000000000050
:20D0E000000000000000000000000000000000000000000000000000000008060000003EE4
:20D10000000000F8030000C01F000000FC010000E00F0000003E00000030000000000000DB
:20D120000000000000000000000000000000000000000000000000000000000000000000EF
:20D140000000000000000000000000000000000000000000000000000000000000000000CF
:20D160000000000000000000000000060E00000E0E00000E0E00000EFEFFFF0FFEFFFF0F3F
:20D18000FEFFFF0F0000000000000000000000000000000000000000000000000000000084
:20D1A00000000000000000000000000000000000000000000000000000000000000000006F
:20D1C000000000000000000000000000000000000000000000000000000000000E00000041
:20D1E0000000080000000E000080070000C0010000F00000003C0000000E0000003C00005B
:20D200000070000000C001000080070000000E000000080000000000000000000000000040
:20D220000000000000000000000000000000000000000000000000000000000000000000EE
:20D2400000000000000000000000000000180000000C0000000C0000000C0000000C000086
:20D26000000C0000000C0000000C0000000C0000000C0000000C0000000C0000000C00004E
:20D28000000C0000000C0000000C0000000C0000000C0000000C0000000C0000000C00002E
:20D2A000000C0000000C0000000C0000000C00000000000000000000000000000000060038
:20D2C00000000002000000060000000E0000001E0000001800000000000000000000000002
:20D2E00000000000000000000000000000000000000000000000000000000000000000002E
:20D3000000000000000000000000000000000000000000000000000000000000000000000D
:20D320000000000000000000000000000000000F00000000000C0F00008E1F00008F3F0048
:20D3400000C3390080C1300080C1300080C1300080C110008061180080630C0080FF1F00A7
:20D3600000FF3F0000FE3F0000002000000000000000000000000000000000000000000012
:20D3800000000000000000000000000000000000000000000000000000000000000000008D
:20D3A0000E00000000FEFF3F00FEFF3F00FEFF3F0000070C0000031800800130008001301B
:20D3C00000800130008003380000071C0000FF1F0000FE0F0000F803000000000000000098
:20D3E00000000000000000000000000000000000000000000000000000000000000000002D
:20D4000000000000000000000000000000000000000D0000000000F8030000FE0F0000FFF8
:20D420001F0000071C008003380080013000800130008001300080033800000F1E00000EE6
:20D440000E00000C06000000000000000000000000000000000000000000000000000000AC
:20D460000000000000000000000000000000000000000000000000000000000000000000AC
:20D4800000000E0000000000F8030000FE0F0000FF1F0000071C0080033800800130008049
:20D4A000013000800130000003180000070C00FEFF3F00FEFF3F00FEFF3F000000000000A8
:20D4C00000000000000000000000000000000000000000000000000000000000000000004C
:20D4E000000000000000000000000000000000000000000E0000000000F8030000FE0F0016
:20D5000000FF1F0000671C00806338008061300080613000806130008063380000673C005E
:20D52000007F1E00007E0E0000780600000000000000000000000000000000000000000044
:20D540000000000000000000000000000000000000000000000000000000000000000000CB
:20D5600000000000098001000080010000F8FF3F00FCFF3F00FEFF3F0086010000860100E6
:20D580000086010000060000000000000000000000000000000000000000000000000000FE
:20D5A00000000000000000000000000000000000000000000000000000000000000000006B
:20D5C0000000000000000000000000000000000000000000000E0000000000F8830100FEC3
:20D5E0008F0700FF9F0700071C0E8003380C8001300C8001300C8001300C0003180E000692
:20D600001C0780FFFF0780FFFF0380FFFF0000000000000000000000000000000000000063
:20D620000000000000000000000000000000000000000000000000000000000000000000EA
:20D640000000000000000E00000000FEFF3F00FEFF3F00FEFF3F000006000000030000807F
:20D660000100008001000080010000800100008003000000FF3F0000FF3F0000FE3F0000EA
:20D6800000000000000000000000000000000000000000000000000000000000000000008A
:20D6A000000000000000000000000000000000000000000000000004000000008EFF3F009A
:20D6C0008EFF3F008EFF3F00000000000000000000000000000000000000000000000000B2
:20D6E00000000000000000000000000000000000000000000000000000000000000000002A
:20D70000000000000000000000000000000000000000000000000000000000000000000009
:20D720000000000000000000040000000C8EFFFF0F8EFFFF078EFFFF03000000000000001C
:20D740000000000000000000000000000000000000000000000000000000000000000000C9
:20D760000000000000000000000000000000000000000000000000000000000000000000A9
:20D78000000000000000000000000000000000000000000000000000000F00000000FEFF7D
:20D7A0003F00FEFF3F00FEFF3F0000E00000007000000078000000FC000000CE0300008F8E
:20D7C000070000070F0080031E008001380080003000000020000000000000000000000002
:20D7E000000000000000000000000000000000000000000000000000000000000000000029
:20D80000000000000000000000000400000000FEFF3F00FEFF3F00FEFF3F00000000000050
:20D820000000000000000000000000000000000000000000000000000000000000000000E8
:20D840000000000000000000000000000000000000000000000000000000000000000000C8
:20D86000000000000000000000000000000000000000000000000000000000160000000092
:20D8800080FF3F0080FF3F0080FF3F000006000000030000800100008001000080010000C2
:20D8A0008003000080FF3F0000FF3F0000FE3F0000060000000300008001000080010000A1
:20D8C000800100008003000080FF3F0000FF3F0000FE3F000000000000000000000000000B
:20D8E0000000000000000000000000000E0000000080FF3F0080FF3F0080FF3F00000600DA
:20D900000000030000800100008001000080010000800100008003000000FF3F0000FF3F01
:20D920000000FE3F00000000000000000000000000000000000000000000000000000000AA
:20D9400000000000000000000000000000000000000000000000000000000000000E0000B9
:20D96000000000F8030000FE0F0000FF1F0000071C008003380080013000800130008001C0
:20D9800030008003380000071C0000FF1F0000FE0F0000F803000000000000000000000053
:20D9A000000000000000000000000000000000000000000000000000000000000000000067
:20D9C00000000000000000000000000000000E0000000080FFFF0F80FFFF0F80FFFF0F0092
:20D9E0000E1C00000318008001300080013000800130008003380000071C0000FF1F0000D3
:20DA0000FE0F0000F8030000000000000000000000000000000000000000000000000000FE
:20DA2000000000000000000000000000000000000000000000000000000000000000000ED8
:20DA40000000000000F8030000FE0F0000FF1F0000071C0080033800800130008001300060
:20DA60008001300000031800000E1C0080FFFF0F80FFFF0F80FFFF0F000000000000000009
:20DA8000000000000000000000000000000000000000000000000000000000000000000086
:20DAA000000000000000000000000000000000000A0000000080FF3F0080FF3F0080FF3F22
:20DAC0000000060000000300008001000080010000800300000001000000000000000000B7
:20DAE000000000000000000000000000000000000000000000000000000000000000000026
:20DB0000000000000000000000000000000000000000000000000000000000000000000005
:20DB2000000D00000000001E0600003F1E00007F1E008073380080F1300080E1300080E1FC
:20DB4000310080C3310000CF390000CF1F00008C1F0000000F000000000000000000000070
:20DB60000000000000000000000000000000000000000000000000000000000000000000A5
:20DB8000000000000000000000000000000000000000078001000080010000F8FF1F00F86E
:20DBA000FF3F00FCFF3F00800130008001300000000000000000000000000000000000008B
:20DBC000000000000000000000000000000000000000000000000000000000000000000045
:20DBE000000000000000000000000000000000000000000000000000000000000000000025
:20DC00000000000E0000000080FF070080FF1F0080FF1F000000380000003000000030009C
:20DC200000003000000030000000180000000C0080FF3F0080FF3F0080FF3F000000000026
:20DC40000000000000000000000000000000000000000000000000000000000000000000C4
:20DC600000000000000000000000000000000000000000000F8000000080070000803F00CF
:20DC80000000FF000000F8070000E03F0000003F000000380000003F0000C03F0000F807B3
:20DCA0000000FF0000803F000080070000800000000000000000000000000000000000009F
:20DCC000000000000000000000000000000000000000000000000000000000000000000044
:20DCE0000000000000140000000080030000807F000080FF070000FC3F0000803F0000000E
:20DD0000380000C03F0000FC0700807F000080030000807F000000FC070000C03F00000046
:20DD2000380000C03F0000FC3F0080FF0700803F00008003000000000000000000000000A9
:20DD4000000000000000000000000000000000000000000000000E800020008001300080E4
:20DD6000033800000F1E00001E0F0000FC070000F0010000F0010000FC0700001E0F0000F9
:20DD80000F1E0080033800800130008000200000000000000000000000000000000000004A
:20DDA000000000000000000000000000000000000000000000000000000000000000000063
:20DDC000000000000000000F800100008007000C801F000C00FE000C00F8030E00E08F07EC
:20DDE0000080FF030000FC0100007F0000E00F0000F80300007F0000801F00008007000096
:20DE0000800000000000000000000000000000000000000000000000000000000000000082
:20DE20000000000000000000000000000000000000000000000000000E00000000000030A4
:20DE40000080013C0080013E0080013F008081330080C1310080E1300080793000803D3039
:20DE600000801F3000800730008003300080013000000000000000000000000000000000B8
:20DE8000000000000000000000000000000000000000000000000000000000000000000082
:20DEA00000000000000000000014000000000000000000000000000000000000000000004E
:20DEC0000000000000000000000000000000000000000000000000000000000000000060E2
:20DEE000000000F80000F09FFF00F807FE010C00000306000006020000040000000000007D
:20DF00000000000000000000000000000000000000000000000000000000050000000000FC
:20DF200000000000000000FEFFFF0FFEFFFF0F0000000000000000000000000000000000CB
:20DF40000000000000000000000000000000000000000000000000000000000000000000C1
:20DF60000000000000000000000000000000000000000000000000000000000000000000A1
:20DF80000000000000000000000000050C000003F80FFE01F09FFF0000F800000060000081
:20DFA000000000000000000000000000000000000000000000000000000000000000000061
:20DFC000000000000000000000000000000000000000000000000000000000000000000041
:20DFE000000000000000000000000000000000000000000000000000000000000F00000012
:20E000000000380000001C0000001C0000001C0000001C0000001C0000001C0000003800E8
:20E02000000038000000380000003800000038000000380000001C000000000000000000AC
:20E040000000000000000000000000000000000000000000000000000000000000000000C0
:20E0600000000000000000000000000000010000000000000000000000000000000000009F
:20E08000000000000000000000000000000000000000000000000000000000000000000080
:20E0A000000000000000000000000000000000000000000000000000000000000000000060
:20E0C000000000000000000000000000000000000000000000000000000000000000DA1F47
:20E0E0003707100000000000000000000000000000000000000000000000000000000000D2
:20E100000000000000000000000000000000000000000000000000000000000000000000FF
:20E120000000000000000000000000000000000000000000000000000000000000000000DF
:20E140000000000000000000000000000000000000000000000000000000000000000000BF
:20E1600000000000000000000000000000000000000000000000000000000000000000009F
:20E1800000000000000000000000000000000000000000000000000000000000000000007F
:20E1A00000000000000000000000000000000000000000000000000000000000150000004A
:20E1C00000000000000000000000000000000000000000000000000000000000000000003F
:20E1E00000000000000000000000000000000000000000000000000000000000000000001F
:20E200000000000000000000000000000000E0000000000000F80300C0FF3F00F80300C06A
:20E22000FFFF3FFC0700C0FFFF3FFC0700C0FFFF3FFC0700C0FFFF3FFC0700C0FF0300F8E4
:20E24000030000000000F0010000000000400000000000000000000000000000000000008A
:20E2600000000000000000000000000000000000000000000000000000000000000000009E
:20E28000000000000000000000000000000000000000000000001B00000000000000000063
:20E2A0000000000000000000000000000000000000000000000000000000C03F000000005F
:20E2C00000C0FF3F00000000C0FFFF01000000C0FFFF01000000C0FFFF01000000C0FFFF45
:20E2E00001000000C0FF0F00000000C0070000000000000000000000000000000000000088
:20E3000000000000000000000000000000000000000000000000000000000000C03F0000FE
:20E32000000000C0FF3F00000000C0FFFF01000000C0FFFF01000000C0FFFF01000000C0E2
:20E34000FFFF01000000C0FF0F00000000C007000000000000000000000000000000000029
:20E36000000000000000000000000000000000001C00000000000000000000000000000081
:20E3800000000000000000000000000000000000F800000000001FF800000000001FF80057
:20E3A000000000001FF8C0030000001FF8FF03000000FFFFFF030000E0FFFFFF030000FF8B
:20E3C000FFFF07000000FFFFFB00000000FF1FF800000000031FF800000000001FF80000F8
:20E3E0000000001FF800000000001FF8E0030000001FF8FF03000000FFFFFF030000F0FF04
:20E40000FFFF030000FFFFFF07000000FFFFFB00000000FF1FF800000000031FF8000000CE
:20E4200000001FF800000000001FF800000000001F0000000000000000000000000000008F
:20E44000000000000000000000001B000000000000000000000000000000000000000000A1
:20E460000000000000000000000000080000000007001E000000E01F003F000000F03F0002
:20E480003F000000F87F007E000000FCFF007E000000FCFF017C000000FCFC01FC00000062
:20E4A0007EF803FC0000003EF003F80000FC3FF003F8FF00FC3FE007F8FF00FC3FE007F866
:20E4C000FF00FC3FC00FF8FF00003EC00FF80000003EC01FFC0000007E801F7C0000007C09
:20E4E000807F7F000000FC00FF7F000000F801FF3F000000F800FE1F0000007000FC0F005D
:20E5000000002000F8070000000000000000000000000000000000000000000000000000DC
:20E52000000000001F0000000000000000C0070020000000F03F0030000000FCFF00780003
:20E540000000FEFF01FC000000FEFF017E0000000FE0033F0000000780830F000000078074
:20E56000C3070000000780E3030000000FC0FB010000001FE07300000000FEFF2100000009
:20E5800000FCFF0000000000FC7F0000000000F03F800F0000000003E07F0000000000F8ED
:20E5A000FF0100000000FCFF0300000008FCFF030000003E1EC0070000001F0E0007000000
:20E5C000800F0E00070000C0070E00070000F0031E80070000F8013EC0070000FC00FCFF2E
:20E5E0000300007E00F8FF0100003C00F8FF0000001800E07F0000001000000600001F00C3
:20E6000000000000000000000000000000000000E01F0000000000F07F0000000000FCFF91
:20E620000000008001FEFF010000F81FFFFF030000FC7FFFFF030000FEFF3FF0030000FF99
:20E64000FF0FE0070000FFFF0FE00700801FF01FC00700800FF07FC00700800FF8FFC0074A
:20E6600000800FF8FEC10700801F7CFCC3070080FF7FF0E7030000FF3FE0EF030000FF1F66
:20E68000C0FF030000FE0780FF010000F80380FF010000000000FF0000000000C0FF0000FA
:20E6A000000000F0FF0000000000FEFF0100000080FFFF0100000080FFF10300000080FFFC
:20E6C000E003000000801FE0070000008007C00300000080004000001400000000000000B3
:20E6E00000000000000000000000000000000000000000000000000000000000000000001A
:20E700000000000000000000000000000000000000000000000000000000000000000000F9
:20E7200000000000000000000000000000C03F0000000000C0FF3F00000000C0FFFF01001D
:20E740000000C0FFFF01000000C0FFFF01000000C0FFFF01000000C0FF0F00000000C007E7
:20E76000000000000000000000000000000000000000000000000000000000000000000099
:20E78000000000000000000000000000000000000000000000000000000000000000000079
:20E7A000000000000000000000000000000000000000190000000000000000000000000040
:20E7C000000000000000000000000000000000000000000000000000000000000000000039
:20E7E000000000000000000000000000000000000000000000000000000000807F0000001A
:20E800000000FCFF0F00000080FFFF7F000000E0FFFFFF010000F8FFFFFF070000FCFFFF1D
:20E82000FF0F0000FE0700F81F0080FF0000C07F00C03F000000FF00E00F000000FC01F016
:20E8400007000000F803F803000000F007F001000000E003700000000080032000000000DD
:20E86000000100000000000000000000000000000000000000000000000000000000000097
:20E88000000000000000000000000000160000000000000000000000000000000000000062
:20E8A0000000000000000000000000000000000000000000000000000000000000006000F8
:20E8C0000000008001F000000000C003F801000000E007F803000000F007F007000000F843
:20E8E00003E01F000000FE01C07F000080FF0000FF0100E03F0000FE0F00FC1F0000FCFF17
:20E90000FFFF0F0000F0FFFFFF030000C0FFFFFF00000000FFFF3F00000000F8FF07000002
:20E920000000000C00000000000000000000000000000000000000000000000000000000CB
:20E940000000000000000000000000000000000000000000000000000000000000000000B7
:20E960000000000000001C000000000000000000000000000000000000000000000000007B
:20E980000000000000300000000000007800000000000078000000000000F0000400000063
:20E9A00000F0000F00000000F0811F00000000F0E10F00000000E0FB0700000000E0FF0126
:20E9C00000000000E0FF00000000F0FF7F00000000F0FF3F00000000F0FF3F00000000F09E
:20E9E000FF7F0000000000E0FF0000000000E0FF0300000000E0F30700000000F0E10F001E
:20EA0000000000F0811F00000000F0000E00000000F0000400000000780000000000007884
:20EA20000000000000002000000000000000000000000000000000000000000000000000B6
:20EA40001C000000000000000000000000000000000000000000000000000000000000C0DA
:20EA6000070000000000C0070000000000C0070000000000C0070000000000C00700000073
:20EA80000000C0070000000000C0070000000000C0070000000000C0070000000000C00793
:20EAA00000000000F0FFFF1F000000F0FFFF1F000000F0FFFF1F000000F0FFFF1F00000022
:20EAC00000C0070000000000C0070000000000C0070000000000C0070000000000C0070053
:20EAE00000000000C0070000000000C0070000000000C0070000000000C0070000000000FA
:20EB0000C00700000000000000000000000000000000000000000000000016000000000018
:20EB20000000000000000000000000000000000000000000000000000000000000000000D5
:20EB40000000000000000000000000000000000000000000000000000000000000000000B5
:20EB600000000000000000020000000078001F00000000FE000F00000000FE800F00000062
:20EB800000FFC10F00000000FFE10700000000FFF90300000000FFFF0300000000FFFF01C4
:20EBA00000000000FE7F0000000000FC3F0000000000F007000000000000000000000000A6
:20EBC000000000000000000000000000000000000000000000000000000000000000000035
:20EBE00000000000000000000000000000000000000000001C0000000000000000000000F9
:20EC000000000000000000000000000000000000000000C0070000000000C0070000000066
:20EC200000C0070000000000C0070000000000C0070000000000C0070000000000C00700F1
:20EC400000000000C0070000000000C0070000000000C0070000000000C007000000000098
:20EC6000C0070000000000C0070000000000C0070000000000C0070000000000C0070000B1
:20EC8000000000C0070000000000C0070000000000C0070000000000C0070000000000C098
:20ECA000070000000000C0070000000000C0070000000000C00700000000000000000000F8
:20ECC00000000000000000000000000000001500000000000000000000000000000000001F
:20ECE000000000000000000000000000000000000000000000000000000000000000000014
:20ED00000000000000000000000000000000000000000000000000000000000000000000F3
:20ED2000FC010000000000FE030000000000FE030000000000FF070000000000FF070000C8
:20ED4000000000FF070000000000FF070000000000FE030000000000FE030000000000F8AD
:20ED6000000000000000000000000000000000000000000000000000000000000000000093
:20ED8000000000000000000000000000000000000000000000000000000000000000000073
:20EDA00000000000000000001B000000000000000000000000000000000000000000000038
:20EDC000000000000000000000000000000000000000030000000000E0030000000000FC51
:20EDE000030000000000FF0300000000E0FF0300000000FCFF0000000000FF3F00000000F3
:20EE0000E0FF0700000000FCFF0000000000FF3F00000000E0FF0700000000F8FF000000F6
:20EE20000000FF3F00000000E0FF0700000000F8FF0000000000FF3F00000000E0FF070093
:20EE4000000000F0FF0100000000F03F0000000000F0070000000000F0010000000000307B
:20EE6000000000000000000000000000000000000000000000000000000000000000000092
:20EE800000001C0000000000000000000000000000000000000000000000C00F0000000087
:20EEA00000FEFF03000000C0FFFF0F000000E0FFFF3F000000F0FFFF7F000000F8FFFFFF06
:20EEC000000000FC0780FF010000FE0000FC0300007E0000F00300003F8007E00700001F75
:20EEE000C00FC00700001FE01FC00700001FE01FC00700001FE01FC00700001FE01FC007E8
:20EF000000003FC00FE00700003F0003E00300007E0000F0030000FE0100FC030000FC0F5D
:20EF200080FF010000F8FFFFFF000000F0FFFF7F000000E0FFFF3F00000080FFFF0F000045
:20EF40000000FCFF0100000000000000000000000000000000000000000000001C00000099
:20EF6000000000000000000000000000000000000000000000000000000000000000000091
:20EF800000000000E0030000000000E00300007C0000E00300007C0000E00300007C000071
:20EFA000E00300007C0000E00300007C0000E00300007E0000E00300007E0000E0030000EE
:20EFC000FFFFFFFF030000FFFFFFFF030000FFFFFFFF030000FFFFFFFF030000FFFFFFFF39
:20EFE000030000FFFFFFFF030000000000E0030000000000E0030000000000E00300000066
:20F000000000E0030000000000E0030000000000E0030000000000E0030000000000E00381
:20F02000000000000000000000000000000000000000000000001C000000000000000000B4
:20F040000000000000000000000000000020000080030000700000C0030000F80000E003FF
:20F060000000FC0100F0030000FC0000F80300007E0000FC0300003E0000FE0300003E00AF
:20F0800000FF0300001F0000FF0300001F0080FF0300001F00C0EF0300001F00E0E70300F2
:20F0A000001F00F0E30300001F00FCE10300003F00FEE10300003F00FFE00300007EC07F5D
:20F0C000E0030000FEFF1FE0030000FCFF0FE0030000FCFF07E0030000F8FF03E00300009F
:20F0E000F0FF00E0030000C03F00E0030000000000E0030000000000E00300000000000096
:20F10000000000000000000000000000000000001C000000000000000000000000000000D3
:20F120000000000000000000000060000000100000F0000000780000FC010000FC0000F806
:20F14000010000FC0000F00300007E0000F00300003E0000E00300003EC007E00700001F22
:20F16000C007C00700001FC007C00700001FC007C00700001FC007C00700001FC007C0074D
:20F1800000001FE00FC00700001FE00FC00700003FF00FE00700007EF01FE0030000FEFF33
:20F1A0003EF0030000FEFF7EFC030000FC7FFEFF010000FC3FFCFF010000F83FF8FF0000C6
:20F1C00000F00FF87F0000008003E03F0000000000800F0000000000000000000000000088
:20F1E000000000000000000000001D0000000000000000000000000000000000F001000001
:20F20000000000F8010000000000FE010000000000FF010000000080FF0100000000E0FF97
:20F220000100000000F0FF0100000000F8F30100000000FEF10100000000FFF00100000011
:20F24000803FF001000000E01FF001000000F007F001000000F803F001000000FE01F0014A
:20F260000000007F00F0010000001F00F001000000FFFFFFFF030000FFFFFFFF030000FF11
:20F28000FFFFFF030000FFFFFFFF030000FFFFFFFF0300000000F0010000000000F001008E
:20F2A00000000000F0010000000000F0010000000000F0010000000000000000000000007B
:20F2C000000000001C000000000000000000000000000000000000000000000000006000B2
:20F2E0000000000000F0000000008001FC000000FFFF03F8010000FFFF03F0030000FFFFB5
:20F3000007F0030000FFFF03E0030000FFFF03E0070000FFE001C00700001FE001C00700B9
:20F32000001FF001C00700001FF001C00700001FF001C00700001FF001C00700001FF00161
:20F34000E00700001FF003E00700001FF003F00300001FE007F80300001FE01FFC030000AA
:20F360001FE0FFFF0100001FC0FFFF0000001F80FF7F0000001F00FF3F0000000000FE1F1B
:20F380000000000000F80300000000000000000000000000000000000000000000001D0055
:20F3A0000000000000000000000000000000000000000000000000000000000000F8FF0155
:20F3C00000000000FFFF0F000000C0FFFF3F000000E0FFFF7F000000F0FFFFFF000000F8E1
:20F3E0007FFEFF010000FC071FFC010000FC010FF00300007E8007E00300003EC007E0079E
:20F4000000003FC003C00700001FE003C00700001FE003C00700001FE003C00700001FE0C9
:20F4200003C00700001FE003E00700001FE007E00300003FE00FF00300003EC01FFC0300F3
:20F44000007EC0FFFF010000FE80FFFF0000007C00FFFF0000003800FE3F0000000800FC00
:20F460001F0000000000C001000000000000000000000000000000001C0000000000000090
:20F480000000000000000000000000000000001F0000000000001F0000000000001F00000F
:20F4A000000000001F0000000000001F0000000000001F0000000000001F000000000000D0
:20F4C0001F0000000000001F0000E00300001F0080FF0300001F00F8FF0300001F00FEFF35
:20F4E0000300001F80FFFF0300001FE0FFFF0300001FF8FF3F0000001FFE3F000000001F99
:20F50000FF03000000009FFF0000000000FF1F0000000000FF0F0000000000FF030000001D
:20F520000000FF0000000000007F0000000000003F0000000000001F0000000000000000EF
:20F540000000000000000000000000000000000000001C000000000000000000000000008F
:20F56000000000000000000000000000070000000000C03F0000008007F07F000000F01F80
:20F58000F8FF000000F87FF8FF010000FC7FFCFF010000FCFF3EF8030000FEFF1FF003004B
:20F5A000007EF00FE00700003FE007E00700001FC007C00700001FC007C00700001F800FD2
:20F5C000C00700001F800FC00700001F000FC00700001F001FC00700003F801FE007000030
:20F5E0007EC03FE0070000FEF07FF0030000FEFFFDFC030000FCFFFCFF010000F87FF8FFE9
:20F60000010000F03FF8FF000000C00FF07F0000000000C03F000000000000000000000086
:20F620000000000000000000000000001C00000000000000000000000000000000000000AE
:20F64000000000003F0000000000C0FF00C0000000F0FF03E0010000F8FF07F8010000FC26
:20F66000FF07F0030000FCFF0FE0030000FEC00FE00300007E801FC00700003F801FC0076B
:20F6800000001F001FC00700001F001FC00700001F001FC00700001F001FC00700001F0037
:20F6A0001FE00700001F000FE00700003F800FF00300007E8007F8030000FEC007FC0100AC
:20F6C00000FCE103FF010000FCFFFDFF000000F8FFFF7F000000F0FFFF3F000000C0FFFFF3
:20F6E0000F00000000FFFF0300000000F87F00000000000000000000000000000000000083
:20F700000000000000001500000000000000000000000000000000000000000000000000D4
:20F720000000000000000000000000000000000000000000000000000000000000000000C9
:20F74000000000000000000000000000000000000000000000007F00FC01000080FF00FEB0
:20F7600003000080FF00FE030000C0FF01FF070000C0FF01FF070000C0FF01FF070000C0F4
:20F78000FF01FF07000080FF00FE03000080FF00FE030000003E00F800000000000000002D
:20F7A000000000000000000000000000000000000000000000000000000000000000000049
:20F7C000000000000000000000000000000000000000000000000000000000000000000029
:20F7E0001600000000000000000000000000000000000000000000000000000000000000F3
:20F800000000000000000000000000000000000000000000000000000000000000000000E8
:20F82000000000000000000000000000000200007F0078001F0080FF00FE000F0080FF00A5
:20F84000FE800F00C0FF01FFC10F00C0FF01FFE10700C0FF01FFF90300C0FF01FFFF030069
:20F8600080FF00FFFF010080FF00FE7F0000003E00FC3F0000000000F0070000000000009E
:20F88000000000000000000000000000000000000000000000000000000000000000000068
:20F8A00000000000000000000000000000000000000000000000000000001A00000000002E
:20F8C000000000000000000000000000000000000000000000000000000000000000000028
:20F8E00000000000000000C0070000000000E00F0000000000E00F0000000000F01F000054
:20F90000000000F83F0000000000F83E0000000000FC7E00000000007EFC00000000003E48
:20F92000F800000000003FF801000000801FF003000000800FE003000000C007C007000005
:20F9400000E007C00F000000E003800F000000F001001F000000F001001F000000F8000067
:20F960003E0000007C00007C0000007E0000FC0000000000000000000000000000000000D7
:20F9800000000000000000000000000000000000000000001C00000000000000000000004B
:20F9A000000000000000000000000000000000000000001FF001000000001FF00100000027
:20F9C000001FF001000000001FF001000000001FF001000000001FF001000000001FF001D7
:20F9E000000000001FF001000000001FF001000000001FF001000000001FF00100000000C7
:20FA00001FF001000000001FF001000000001FF001000000001FF001000000001FF0010096
:20FA20000000001FF001000000001FF001000000001FF001000000001FF001000000001F67
:20FA4000F001000000001FF001000000001FF001000000001FF00100000000000000000085
:20FA600000000000000000000000000000001A00000000000000000000000000000000006C
:20FA8000000000000000000000000000000000000000003E0000F80000007C00007C000038
:20FAA000007C00007C000000F800003E000000F001001F000000F003801F000000E0038013
:20FAC0000F000000C007C007000000C00FE007000000800FE003000000001FF00100000051
:20FAE000003FF801000000003EF800000000007EFC0000000000FC7E0000000000F83F006D
:20FB000000000000F83F0000000000F01F0000000000E00F0000000000E00F0000000000C1
:20FB2000C007000000000000000000000000000000000000000000000000000000000000FE
:20FB400000000000000000001A00000000000000000000000000000000000000000000008B
:20FB60000000000000000000000000000000000000000000040000000000000E0000000073
:20FB800000003F0000000000801F0000000000800F0000000000800F0000F00100C00700B1
:20FBA0003CF80300C007003FFC0700C007803FFC0700C007C03FFC0700C007E03FFC0700CA
:20FBC000C007F05FF80300C00FF803F80300801FFE01E0000080FF7F0000000080FF3F0015
:20FBE00000000000FF1F0000000000FE0F0000000000FC070000000000F0010000000000E6
:20FC00000000000000000000000000000000000000000000000000000000000000000000E4
:20FC200000001D0000000000000000000000000000000080FF0300000000F8FF3F000000EF
:20FC400000FEFFFF01000080FFFFFF070000E0FFC7FF0F0000F01F00E01F0000F8030080E6
:20FC60003F0000FC0100007E00007C000000FC00003E004000F800003E00F807F001001E90
:20FC800000FE0FE001001F00FF1FE003000F00FF1FC003000F800F3FC003000F80073EC032
:20FCA00003000FC0073EC003000FC0033EC003000FC0033EC003001FC0031EC003003EE0E3
:20FCC000011FE001007EE0010FE00100FCE18107F00100F8FFFF0FF00000F0FFFF1FC000BC
:20FCE00000C0FFFF1F00000000FFFF1F000000000000000000000000000000001F000000EB
:20FD0000000000000000000000020000000000C0030000000000FC030000000080FF03009D
:20FD2000000000F0FF0300000000FEFF03000000C0FFFF01000000F8FF3F00000000FFFFDE
:20FD400007000000E0FFFF01000000FEFFFF01000080FFFFF001000080FF0FF00100008052
:20FD6000FF01F0010000801F00F0010000803F00F001000080FF03F001000080FF3FF00130
:20FD8000000080FFFFF301000000FCFFFF01000000E0FFFF0100000000FFFF0F000000000A
:20FDA000F8FFFF0000000080FFFF0300000000FCFF0300000000E0FF030000000000FF03EA
:20FDC0000000000000F8030000000000C00300000000000002001D00000000000000000046
:20FDE000000000000000000000000000000000000000000000000000000080FFFFFFFF0384
:20FE00000080FFFFFFFF030080FFFFFFFF030080FFFFFFFF030080FFFFFFFF030080FFFF68
:20FE2000FFFF0300800FE003E00300800FE003E00300800FE003E00300800FE003E003006D
:20FE4000800FE003E00300800FE003E00300800FE003E00300800FF003E00300801FF007A8
:20FE6000F00300003FF807F0030000FFFF07F8010000FFFF1FFC010000FE3FFFFF0100000A
:20FE8000FE3FFFFF000000FC1FFE7F000000F807FE7F0000000000FC1F0000000000F00FF9
:20FEA000000000000000000000000000000000001E00000000000000000000000000000024
:20FEC0000000000000000000E01F0000000000FEFF0100000080FFFF07000000E0FFFF1FA3
:20FEE000000000F0FFFF3F000000F8FFFF7F000000FCFFFCFF000000FE0780FF010000FEE7
:20FF00000100FE0100007F0000F80300003F0000F00300001F0000E00300801F0000E007AD
:20FF200000800F0000C00700800F0000C00700800F0000C00700800F0000C00700800F00DA
:20FF400000C00700800F0000C00700801F0000E00700001F0000E00300003F0000F00300CA
:20FF6000007E0000F80300003E0000F80100001C0000F0000000080000600000000000005D
:20FF8000400000000000000000001D00000000000000000000000000000000000000000004
:20FFA0000000000000000080FFFFFFFF030080FFFFFFFF030080FFFFFFFF030080FFFFFF47
:20FFC000FF030080FFFFFFFF030080FFFFFFFF0300800F0000E00300800F0000E0030080BD
:20FFE0000F0000E00300800F0000E00300800F0000E00300800F0000E00300801F0000F02A
:020000040001F9
:200000000300801F0000F00300001F0000F80100003F0000F80100007F0000FC010000FE81
:200020000100FF000000FE0FE0FF000000FCFFFF7F000000F8FFFF3F000000F0FFFF1F0019
:200040000000E0FFFF0F00000080FFFF0300000000FC7F00000000000000000000000000B7
:20006000000000001C00000000000000000000000000000000000000000000000000000064
:2000800000000000000000000000000000000080FFFFFFFF030080FFFFFFFF030080FFFFE4
:2000A000FFFF030080FFFFFFFF030080FFFFFFFF030080FFFFFFFF0300800FE003E003006D
:2000C000800FE003E00300800FE003E00300800FE003E00300800FE003E00300800FE0035A
:2000E000E00300800FE003E00300800FE003E00300800FE003E00300800FE003E003008049
:200100000FE003E00300800FE003E00300800FE003E00300800F0000E00300800F0000E07F
:200120000300800F0000E003000000000000000000000000000000000000000000001C002E
:2001400000000000000000000000000000000000000000000000000000000000000000009F
:2001600000000000000000000080FFFFFFFF030080FFFFFFFF030080FFFFFFFF030080FF83
:20018000FFFFFF030080FFFFFFFF030080FFFFFFFF030080FFFFFFFF0300800FC00700008C
:2001A00000800FC007000000800FC007000000800FC007000000800FC007000000800FC098
:2001C00007000000800FC007000000800FC007000000800FC007000000800FC007000000C0
:2001E000800FC007000000800FC007000000800FC007000000800F0000000000800F0000DF
:200200000000000000000000000000000000000000000000000000001D00000000000000C1
:2002200000000000000000000000000000000000FCFF0000000000FFFF07000000C0FFFF00
:200240000F000000F0FFFF3F000000F8FFFF7F000000FCFFFFFF000000FC0FC0FF01000029
:20026000FE0100FE010000FF0000F80300003F0000F00300003F0000E00300801F0000E0B3
:200280000700800F0000C00700800F0000C00700800F001FC00700800F001FC00700800F32
:2002A000001FC00700800F001FC00700801F001FE00700001F001FE00300003F00FFFF03DD
:2002C00000007F00FFFF0300003E00FFFF0100001C00FFFF0100000800FFFF000000000040
:2002E000FF7F000000000000000000000000000000001C0000000000000000000000000064
:2003000000000000000000000000000000000080FFFFFFFF030080FFFFFFFF030080FFFF61
:20032000FFFF030080FFFFFFFF030080FFFFFFFF030080FFFFFFFF03000000E0030000005C
:200340000000E0030000000000E0030000000000E0030000000000E0030000000000E0032E
:200360000000000000E0030000000000E0030000000000E0030000000000E00300000000F1
:2003800000E0030000000000E00300000080FFFFFFFF030080FFFFFFFF030080FFFFFFFF1D
:2003A000030080FFFFFFFF030080FFFFFFFF030080FFFFFFFF0300000000000000000000BD
:2003C0000000000000000000000000001B0000000000000000000000000000000000000002
:2003E000000000000000000000800F0000E00300800F0000E00300800F0000E00300800F18
:200400000000E00300800F0000E00300800F0000E00300800F0000E00300800F0000E00331
:2004200000800F0000E0030080FFFFFFFF030080FFFFFFFF030080FFFFFFFF030080FFFF4F
:20044000FFFF030080FFFFFFFF030080FFFFFFFF0300800F0000E00300800F0000E00300B9
:20046000800F0000E00300800F0000E00300800F0000E00300800F0000E00300800F000025
:20048000E00300800F0000E003000000000000000000000000000000000000000000000007
:2004A0000000000000001B0000000000000000000000000000000000000000000000000021
:2004C0000000000000000060000000000000F0000000000000F80000800F0000FC010080C8
:2004E0000F0000F80300800F0000F00300800F0000E00300800F0000E00700800F0000C039
:200500000700800F0000C00700800F0000C00700800F0000C00700800F0000C00700800FED
:200520000000E00700800F0000E00700800F0000F00300800F0000FF030080FFFFFFFF01CE
:200540000080FFFFFFFF010080FFFFFFFF000080FFFFFF7F000080FFFFFF1F000080FFFF8C
:20056000FF0300000000000000000000000000000000000000000000000000000000000079
:200580001F0000000000000000000000000000000000000000000000000000000080FFFFBE
:2005A000FFFF030080FFFFFFFF030080FFFFFFFF030080FFFFFFFF030080FFFFFFFF03003E
:2005C00080FFFFFFFF030080FFFFFFFF03000000C07F0000000000E01F0000000000F80FD8
:2005E0000000000000FC070000000000FE030000000000FF0700000000C0FF1F0000000013
:20060000E0FF7F00000000F0EFFF01000000FC87FF07000000FE03FE1F000000FF01FC7F7B
:200620000000807F00F0FF0100803F00C0FF0300801F0000FF030080070000FC03008003A0
:200640000000F8030080010000E0030080000000800300000000000002001D000000000019
:2006600000000000000000000000000000000000000000000000000000000000000000007A
:20068000000000000080FFFFFFFF030080FFFFFFFF030080FFFFFFFF030080FFFFFFFF035E
:2006A0000080FFFFFFFF030080FFFFFFFF030000000000E0030000000000E0030000000076
:2006C00000E0030000000000E0030000000000E0030000000000E0030000000000E00300AB
:2006E00000000000E0030000000000E0030000000000E0030000000000E00300000000006E
:20070000E0030000000000E0030000000000E0030000000000E0030000000000E00300006A
:20072000000000E0030000000000000000000000000000001C0000000000000000000000BA
:20074000000000000000000000000000000000000080FFFFFFFF030080FFFFFFFF0300801B
:20076000FFFFFFFF030080FFFFFFFF0300803FF8FFFF030080FF030000000000FF1F0000A3
:20078000000000F8FF0000000000C0FF070000000000FC3F0000000000E0FF010000000081
:2007A00000FE010000000000FF0100000000E0FF0000000000FE1F00000000C0FF0300007C
:2007C0000000F87F0000000080FF0F0000000080FF0000000000809FFFFFFF030080FFFFF8
:2007E000FFFF030080FFFFFFFF030080FFFFFFFF030080FFFFFFFF0300000000000000007B
:2008000000000000000000000000000000001C0000000000000000000000000000000000BC
:20082000000000000000000000000080FFFFFFFF030080FFFFFFFF030080FFFFFFFF03003B
:2008400080FFFFFFFF030080FFFFFFFF030080FFE0FFFF030000FF030000000000FC0F002D
:2008600000000000F07F0000000000C0FF010000000000FF070000000000FC1F0000000028
:2008800000F07F000000000080FF010000000000FE070000000000F81F0000000000E0FF6E
:2008A000000000000080FF030080FFFF3FFC030080FFFFFFFF030080FFFFFFFF030080FF7D
:2008C000FFFFFF030080FFFFFFFF030080FFFFFFFF0300000000000000000000000000001A
:2008E00000000000000000001E00000000000000000000000000000000E01F0000000000DB
:20090000FEFF01000000C0FFFF0F000000E0FFFF1F000000F8FFFF7F000000FCFFFFFF00A1
:200920000000FEFFFFFF010000FE0300FF010000FF0000FC0300003F0000F00300801F00EB
:2009400000E00700801F0000E00700800F0000C00700800F0000C00700800F0000C0070028
:20096000800F0000C00700801F0000E00700801F0000E00700003F0000F0030000FF0000E4
:20098000FC030000FE0780FF010000FEFFFFFF000000FCFFFFFF000000F8FFFF3F000000AA
:2009A000E0FFFF1F00000080FFFF0700000000FEFF000000000000030000000000000000B5
:2009C00000001D0000000000000000000000000000000000000000000000000000000000FA
:2009E00000000000000080FFFFFFFF030080FFFFFFFF030080FFFFFFFF030080FFFFFFFFFE
:200A0000030080FFFFFFFF030080FFFFFFFF0300800F001F000000800F001F000000800FEA
:200A2000001F000000800F001F000000800F001F000000800F001F000000800F001F0000DF
:200A400000800F001F000000800F801F000000801F801F000000001FC00F000000003FE06F
:200A60000F00000000FFFF0F00000000FEFF0700000000FEFF0300000000FCFF0300000058
:200A800000F8FF0000000000E07F0000000000000000000000000000000000001E000000E2
:200AA00000000000000000000000000000E00F0000000000FFFF01000000C0FFFF07000083
:200AC00000F0FFFF1F000000F8FFFF3F000000FCFFFF7F000000FEFFFFFF000000FE0180E1
:200AE000FF0100007F0000FC0100003F0000F80300801F0000F00300800F0000E0070080B8
:200B00000F0000E01F00800F0000E07F00800F0000E0FF00800F0000E0FF00801F0000F06E
:200B2000FF01001F0000F0FF03003F0000FCF10300FF0000FEE10300FE07C0FFE00700FCED
:200B4000FFFFFFC00700FCFFFF7FC00700F0FFFF3FC00700E0FFFF0FC0070080FFFF03C0A8
:200B6000070000FC7F00E00700000000000003000000000000001E000000000000000000EB
:200B80000000000000000000000000000000000000000080FFFFFFFF030080FFFFFFFF0357
:200BA0000080FFFFFFFF030080FFFFFFFF030080FFFFFFFF030080FFFFFFFF030080FFFFBB
:200BC000FFFF0300800F800F000000800F800F000000800F800F000000800F800F0000009C
:200BE000800F800F000000800F801F000000800F807F000000800F80FF010000801FC0FFAE
:200C0000070000801FC0FF1F0000003FE0FF7F0000007FF8F7FF010000FFFFC3FF03000082
:200C2000FEFF03FF030000FCFF01FC030000FCFF00F8030000F07F00E0030000C00F008020
:200C4000030000000000000200000000000000001D00000000000000000000000000000072
:200C6000000000000000000000004000000000000060000000E01F00F8000000F83F00FCAA
:200C8000010000FC7F00F8010000FEFF00F8030000FEFF01F0030000FFFF01E00300003FD5
:200CA000FC03E00700001FF803E00700801FF007C00700800FF007C00700800FE00FC0075E
:200CC00000800FE00FC00700800FC00FC00700800FC01FC00700800F801FE00700801F8041
:200CE0003FE00300001F807FF00300003F00FFFC0300003F00FFFF0100007E00FEFF0100CA
:200D0000003E00FCFF0000001C00F87F0000000800F03F0000000000C00700000000000009
:200D2000000000000000000000001E0000000000000000000000000000800F000000000006
:200D4000800F0000000000800F0000000000800F0000000000800F0000000000800F0000C8
:200D6000000000800F0000000000800F0000000000800F0000000000800F000000000080B7
:200D80000F000000000080FFFFFFFF030080FFFFFFFF030080FFFFFFFF030080FFFFFFFF4B
:200DA000030080FFFFFFFF030080FFFFFFFF0300800F0000000000800F0000000000800F85
:200DC0000000000000800F0000000000800F0000000000800F0000000000800F00000000D7
:200DE00000800F0000000000800F0000000000800F0000000000800F0000000000000000B7
:200E0000000000001C000000000000000000000000000000000000000000000000000000B6
:200E20000080FFFFFF07000080FFFFFF1F000080FFFFFF7F000080FFFFFFFF000080FFFF9C
:200E4000FFFF010080FFFFFFFF010000000000FC030000000000F0030000000000E007003D
:200E600000000000C0070000000000C0070000000000C0070000000000C007000000000056
:200E8000C0070000000000C0070000000000E0070000000000F0030000000000FC0300806B
:200EA000FFFFFFFF010080FFFFFFFF010080FFFFFFFF000080FFFFFF7F000080FFFFFF1FA4
:200EC000000080FFFFFF0300000000000000000000000000000000000000000000001E0074
:200EE0000000000000008000000000000080030000000000803F000000000080FF010000B0
:200F0000000080FF0F0000000080FF7F0000000080FFFF0300000000FEFF3F00000000E0A8
:200F2000FFFF0100000000FFFF0F00000000F0FF7F0000000000FFFF0300000000F0FF0344
:200F40000000000000FF030000000000F8030000000000F0030000000000FF03000000009F
:200F6000F0FF0300000000FFFF03000000F0FF7F00000000FFFF0F000000E0FFFF00000025
:200F800000FEFF1F00000080FFFF0300000080FF7F0000000080FF070000000080FF0000B1
:200FA000000000801F000000000080030000000000000000000000001F8000000000000070
:200FC000807F000000000080FF3F0000000080FFFF1F00000080FFFFFF0F000080FFFFFFAE
:200FE000FF030080FFFFFFFF03000000FEFFFF0300000000F0FF030000000000F803000084
:20100000000080FF0300000000F8FF0300000080FF7F00000000F8FF0700000000FF3F001A
:2010200000000000FF010000000000FF030000000000FF7F0000000000FEFF07000000002C
:20104000E0FF7F0000000000FEFF0300000000C0FF030000000000FC030000000000FE0370
:20106000000000F0FFFF030000FFFFFFFF030080FFFFFFFF030080FFFFFF0F000080FFFFF7
:201080001F00000080FF1F00000000803F00000000001E00000000000000000000000000B6
:2010A00000000000000002008001000080030080030000E00300800F0000F00300803F0083
:2010C00000FC030080FF0000FF030080FF03C0FF030080FF07E0FF000000FE1FF83F000093
:2010E00000F87FFE0F000000E0FFFF0300000080FFFF0000000000FE3F0000000000F80FC9
:201100000000000000F03F0000000000FCFF0000000080FFFF03000000E0FFFF070000003F
:20112000F87FFC1F000000FE1FF87F000080FF07E0FF010080FF0180FF030080FF0000FEA4
:201140000300803F0000FC0300800F0000F0030080030000C0030080000000000300000083
:201160000000000200000000000000001E000000000000008000000000000080010000004E
:20118000000080070000000000801F0000000000807F000000000080FF010000000080FF2B
:2011A000070000000000FF1F0000000000FC7F0000000000E0FF010000000080FF07000029
:2011C000000000FE1F0000000000F8FFFF03000000E0FFFF0300000000FFFF030000000017
:2011E000FFFF03000000E0FFFF03000000F8FFFF03000000FE1F0000000080FF0700000071
:2012000000F0FF0100000000FC7F0000000000FF1F0000000080FF070000000080FF01003F
:20122000000000807F0000000000801F000000000080070000000000800100000000000008
:201240000000000000001D0000000000000000000000000000000000000000000000000071
:20126000C0030000000000E00300800F0000F80300800F0000FC0300800F0000FF0300809F
:201280000F0080FF0300800F00E0FF0300800F00F0FF0300800F00FCEF0300800F00FEE3DE
:2012A0000300800F80FFE10300800FC07FE00300800FF03FE00300800FF80FE00300800FDF
:2012C000FE07E00300800FFF03E0030080CFFF00E0030080EF7F00E0030080FF1F00E0032F
:2012E0000080FF0F00E0030080FF0300E0030080FF0100E00300807F0000E00300803F0014
:2013000000E00300800F0000E0030080070000E0030000000000000000000000000000000E
:201320001A0000000000000000000000000000000000000000000000000000000000000093
:2013400000000000000000000000000000000000000000000000000000000000000000008D
:201360000000000000000000000000000000E0FFFFFFFFFF03E0FFFFFFFFFF03E0FFFFFFD4
:20138000FFFF03E0FFFFFFFFFF03E0FFFFFFFFFF03E0000000008003E0000000008003E0EA
:2013A000000000008003E0000000008003E0000000008003E0000000008003E000000000A1
:2013C0008003E0000000008003E0000000008003E000000000800300000000000000000061
:2013E00000000000000000000000000000000000000000000000000000001B0000000000D2
:2014000000000000000000000000000000000000000000000000000000000000000030009C
:201420000000000000F0010000000000F00F0000000000F03F0000000000F0FF010000009D
:2014400000C0FF0F0000000000FF3F0000000000F8FF0100000000C0FF0F0000000000FFBB
:201460003F0000000000F8FF0100000000C0FF070000000000FF3F0000000000F8FF010039
:20148000000000C0FF070000000000FF3F0000000000F8FF0100000000E0FF03000000006E
:2014A00000FF030000000000F8030000000000E00300000000000003000000000000000049
:2014C0000000000000000000000000000000000000000000150000000000000000000000F7
:2014E000000000000000000000000000000000000000000000000000E0000000008003E0A9
:20150000000000008003E0000000008003E0000000008003E0000000008003E0000000003F
:201520008003E0000000008003E0000000008003E0000000008003E0000000008003E000BC
:201540000000008003E0FFFFFFFFFF03E0FFFFFFFFFF03E0FFFFFFFFFF03E0FFFFFFFFFF93
:2015600003E0FFFFFFFFFF030000000000000000000000000000000000000000000000008A
:2015800000000000000000000000000000000000000000000000000000000000000000004B
:2015A00000000000000000000000000000001B000000000000000000000000000000000010
:2015C000000000000000000000000000000000000000000000040000000000000700000000
:2015E0000000E0070000000000FC070000000000FF0700000000E0FF0700000000F8FF001E
:2016000000000000FF1F00000000C0FF0300000000C07F0000000000C01F0000000000C00C
:201620001F0000000000C0FF0000000000C0FF070000000000FE3F0000000000F8FF0000D2
:20164000000000C0FF070000000000FF070000000000F8070000000000C0070000000000F8
:2016600000070000000000000400000000000000000000000000000000000000000000005F
:2016800000000000000000001D00000000000000000000000000000000000000000000002D
:2016A000000000E0030000000000E0030000000000E0030000000000E0030000000000E0BE
:2016C000030000000000E0030000000000E0030000000000E0030000000000E0030000007B
:2016E0000000E0030000000000E0030000000000E0030000000000E0030000000000E0037B
:201700000000000000E0030000000000E0030000000000E0030000000000E003000000003D
:2017200000E0030000000000E0030000000000E0030000000000E0030000000000E003003A
:2017400000000000E0030000000000E0030000000000E003000000000000000000000000E0
:20176000000014000000000000000000000000000000000000000000000000000000000055
:20178000000000000000000000000000000000000000000000000000000000000000000049
:2017A0000000080000000000001800000000000038000000000000F8000000000000F801E0
:2017C0000000000000F8030000000000F0070000000000E0070000000000800700000000A9
:2017E0000000060000000000000400000000000000000000000000000000000000000000DF
:201800000000000000000000000000000000000000000000000000000000000000000000C8
:20182000000000000000000000000000000000000000000000000000000000001C0000008C
:2018400000000000000000000000000000000000000000000000000000000000003F000049
:2018600000000CC0FF000000003CE0FF010000007EF0FF030000003EF0FF030000003FF8AA
:20188000FF070000001FF8E0070000001F78E0070000800F7CC0070000800F3CC007000062
:2018A000800F3CC0070000800F3CC0070000800F3CC0030000800F1EE0030000800F1EE059
:2018C000010000801F1EF0010000803F1EF800000000FF1E7C00000000FFFFFF00000000EE
:2018E000FEFFFF03000000FEFFFF03000000F8FFFF03000000F0FFFF0300000080FFFF037F
:20190000000000000000000000000000000000000000000000001D000000000000000000AA
:2019200000000000000000000000000000000000000000E0FFFFFFFF0300E0FFFFFFFF03E9
:2019400000E0FFFFFFFF0300E0FFFFFFFF0300E0FFFFFFFF0300E0FFFFFFFF0000E03FFCF3
:20196000FFFF000000003E00F0010000003E00E0030000001F00E0030000000F00C0030045
:2019800000800F00C0070000800F00C0070000800F00C0070000800F00C0070000801F0050
:2019A000E0070000801F00F0070000807F00F803000000FF83FF03000000FFFFFF0100002E
:2019C00000FEFFFF00000000FCFF7F00000000F8FF3F00000000E0FF0F0000000000FF016D
:2019E000000000000000000000000000000000001D000000000000000000000000000000CA
:201A000000000000000000000000000000000000FE0300000000C0FF0F00000000E0FF3FD9
:201A200000000000F8FF7F00000000FCFFFF00000000FCFFFF01000000FE03FF010000003A
:201A4000FE00FC030000007F00F8030000003F00F0030000801F00E0070000801F00E007D1
:201A60000000800F00C0070000800F00C0070000800F00C0070000800F00C0070000800F7F
:201A800000C0070000800F00C0070000801F00E0030000001F00E0030000003F00F0030073
:201AA00000003E00F8010000001E00F0010000000C00E00000000000008000000000000074
:201AC000000000000000000000001B000000000000000000000000000000000000000000EB
:201AE000000000FF0700000000E0FF1F00000000F0FF7F00000000F8FFFF00000000FCFF83
:201B0000FF01000000FEFFFF03000000FF03FE030000007F00F8030000803F00E0070000A3
:201B2000801F00E0070000800F00C0070000800F00C0070000800F00C0070000800F00C0CE
:201B4000070000800F00C0030000001F00E0030000001E00F0010000003E00F80000E0FF06
:201B6000FDFFFF0000E0FFFFFFFF0300E0FFFFFFFF0300E0FFFFFFFF0300E0FFFFFFFF03EE
:201B800000E0FFFFFFFF030000000000000000000000000000000000000000000000000066
:201BA000000000001D000000000000000000000000000000000000000000000000FC00000C
:201BC00000000080FF0700000000E0FF1F00000000F0FF3F00000000F8FF7F00000000FCE1
:201BE000FFFF00000000FEFFFF010000007F7CFC010000003F7CF8030000001F7CF00300AE
:201C000000801F7CE0070000800F7CE0070000800F7CC0070000800F7CC0070000800F7C21
:201C2000C0070000800F7CC0070000800F7CC0070000001F7CC0070000003F7CC007000055
:201C4000007F7CE003000000FE7FE003000000FC7FF001000000F87FF001000000F07FC043
:201C600001000000C07F8000000000007E00000000000000000000000000000000001F0007
:201C8000000000000000000000000000000000000000000000000000000000000000000044
:201CA000000000001F0000000000001F0000000000001F0000000000001F000000000000A8
:201CC0001F0000000000001F0000000000001F0000000000F8FFFFFF030000FEFFFFFF03B1
:201CE0000080FFFFFFFF0300C0FFFFFFFF0300C0FFFFFFFF0300E0FFFFFFFF0300E00F1FFA
:201D000000000000F0031F00000000F0031F00000000F0011F00000000F0011F000000007F
:201D2000F0011F00000000F0011F00000000F0011F00000000F0011F00000000F0011F0053
:201D4000000000E0030000000000E0030000000000600000000000001E000000000000003F
:201D600000000000000000000000000000000000000000C0010000000000F0070000F01F9C
:201D80007CF80F0000F83FFEFD0F0000FC7FFFFF1F0000FEFFFFDF1F0000FFFFFF0F1F00C2
:201DA00000FFF8E3073F00003FF0C1073E00801FE0C3073E00800FC0C3073E00800FC0C3DE
:201DC000073E00800FC0C3073E00800FC0C3073E00800FC0C3073E00001FE0C3073E0000B2
:201DE0003FF0C1073E0000FFFFC1071F0000FFFFC1071F0000FFFFC0071F0000FF7FC08F33
:201E00001F0000DF3FC0FF0F00001F0780FF0F00001F0080FF0700001F0080FF0300001F9E
:201E20000000FF0100001F00007C00000000000000001C00000000000000000000000000EB
:201E4000000000000000000000000000000000E0FFFFFFFF0300E0FFFFFFFF0300E0FFFFE6
:201E6000FFFF0300E0FFFFFFFF0300E0FFFFFFFF0300E0FFFFFFFF0300E03FF8FFFF0300AC
:201E800000007C0000000000003E0000000000001E0000000000001F0000000000000F003C
:201EA00000000000800F0000000000800F0000000000800F0000000000800F0000000000E6
:201EC000801F0000000000807F000000000080FFFFFF03000000FFFFFF03000000FFFFFFE7
:201EE00003000000FEFFFF03000000FCFFFF03000000E0FFFF030000000000000000000002
:201F00000000000000000000000000001700000000000000000000000000000000000000AA
:201F200000000000000000000000001F0000000000001F0000000000001F00000000000044
:201F40001F0000000000001F0000000000001F0000000000001F0000000000001F000000E6
:201F60000000001F0000000000001F00000000E0011F00000000F0031F00000000F807FF13
:201F8000FFFF0300F807FFFFFF0300F807FFFFFF0300F807FFFFFF0300F807FFFFFF030044
:201FA000F003FFFFFF0300C00000000000000000000000000000000000000000000000006E
:201FC000000000000000000000000000000000000000000000000000000000000000000001
:201FE0000000000000001700000000000000000000000000000000000000000000000000CA
:2020000000000E00001F0000800F00001F0000800F00001F0000801F00001F0000001F005A
:20202000001F0000001F00001F0000001F00001F0000001F00001F0000001F00001F000089
:20204000001F00001F0000801FE0011F0000C01FF0031F0000F00FF807FFFFFFFF0FF807AA
:20206000FFFFFFFF07F807FFFFFFFF07F807FFFFFFFF03F807FFFFFFFF00F003FFFFFF1F53
:2020800000C000000000000000000000000000000000000000000000000000000000000080
:2020A000000000000000000000000000000000000000000000000000000000000000000020
:2020C0001F00000000000000000000000000000000000000000000000000000000000000E1
:2020E00000000000E0FFFFFFFF0300E0FFFFFFFF0300E0FFFFFFFF0300E0FFFFFFFF030064
:20210000E0FFFFFFFF0300E0FFFFFFFF0300000000F0070000000000F8030000000000FC13
:20212000010000000000FE0000000000007F0000000000807F0000000000C0FF0100000062
:2021400000F0FF0300000000F8FF0F00000000FCF31F00000000FEE13F00000000FF80FFDD
:20216000000000003F00FF010000001F00FE030000000F00F8030000000700F003000000FC
:202180000300C003000000010080030000000100000300000000000002001D0000000000D2
:2021A0000000000000000000000000000000000000000000000000E0030000000000E00359
:2021C0000000000000E0030000000000E0030000000000E0030000000000E0030000000073
:2021E00000E0030000000000E0030000000000E0FFFFFF1F0000E0FFFFFF7F0000E0FFFFE3
:20220000FFFF0100E0FFFFFFFF0100E0FFFFFFFF0300E0FFFFFFFF030000000000F007002D
:2022200000000000E0070000000000C0070000000000C0070000000000C007000000000062
:20224000C0070000000000C0070000000000C0030000000000E0030000000000C003000087
:2022600000000000020000000000000000000000000000001E00000000000000000000003E
:20228000000000000000000000000000FFFFFF03000000FFFFFF03000000FFFFFF0300003E
:2022A00000FFFFFF03000000FCFFFF03000000FC0000000000003E0000000000000F0000D8
:2022C000000000800F0000000000800F0000000000801F000000000080FFFFFF0300008041
:2022E000FFFFFF03000000FFFFFF03000000FEFFFF03000000F8FFFF030000003C000000AA
:202300000000001F0000000000000F0000000000800F0000000000801F000000000080FFE2
:20232000FFFF03000080FFFFFF03000080FFFFFF03000000FFFFFF03000000FEFFFF03009D
:202340000000F0FFFF0300000000000000001C000000000000000000000000000000000070
:2023600000000000000000000000000000FFFFFF03000000FFFFFF03000000FFFFFF03005D
:202380000000FFFFFF03000000FFFFFF03000000FEFFFF03000000F8FFFF030000007C00C9
:2023A00000000000003E0000000000001E0000000000001F0000000000000F000000000093
:2023C000800F0000000000800F0000000000800F0000000000800F0000000000801F000022
:2023E000000000807F000000000080FFFFFF03000000FFFFFF03000000FFFFFF030000005E
:20240000FEFFFF03000000FCFFFF03000000E0FFFF030000000000000000000000000000DF
:2024200000000000000000001D00000000000000000000000000000000000000000000007F
:2024400000FF0300000000C0FF0F00000000F0FF3F00000000F8FF7F00000000FCFFFF000E
:20246000000000FEFFFF01000000FE03FF010000007F00F8030000003F00F0030000801F13
:2024800000E0070000800F00C0070000800F00C0070000800F00C0070000800F00C00700FD
:2024A00000800F00C0070000801F00E0070000001F00E0070000003F00F0030000007F0089
:2024C000F803000000FE87FF01000000FEFFFF01000000FCFFFF00000000F8FF7F0000000F
:2024E00000F0FF3F00000000C0FF0F0000000000FE010000000000000000000000000000E1
:2025000000001D00000000000000000000000000000000000000000000000000000000009E
:2025200000FFFFFFFF0F0000FFFFFFFF0F0000FFFFFFFF0F0000FFFFFFFF0F0000FFFFFF72
:20254000FF0F0000FEFFFFFF0F0000FCFFFFF00F00007E00F0010000003E00E003000000DA
:202560001F00E0030000000F00C0030000800F00C0070000800F00C0070000800F00C00785
:202580000000800F00C0070000801F00E0070000801F00F0070000807F00F803000000FFD0
:2025A00083FF03000000FFFFFF01000000FEFFFF00000000FCFF7F00000000F8FF3F0000EC
:2025C0000000E0FF0F0000000000FF01000000000000000000000000000000001B000000F2
:2025E000000000000000000000000000000000000000000000FF0700000000E0FF1F0000D7
:202600000000F0FF7F00000000F8FFFF00000000FCFFFF01000000FEFFFF03000000FF035A
:20262000FE030000007F00F8030000803F00E0070000801F00E0070000800F00C00700009D
:20264000800F00C0070000800F00C0070000800F00C0070000800F00C0030000001F00E027
:20266000030000001F00F0010000003E00F800000000FCFFFFFE0F0000FEFFFFFF0F000000
:20268000FFFFFFFF0F0000FFFFFFFF0F0000FFFFFFFF0F0000FFFFFFFF0F0000000000000E
:2026A000000000000000000000000000000000000000000000001D000000000000000000FD
:2026C0000000000000000000000000000000000000000000000000000000000000000000FA
:2026E00000000000000000000000FFFFFF03000000FFFFFF03000000FFFFFF03000000FFDB
:20270000FFFF03000000FFFFFF03000000C0FFFF03000000E0030000000000F8000000001C
:2027200000007C0000000000003E0000000000003E0000000000001F0000000000001F0063
:2027400000000000800F0000000000800F0000000000800F0000000000800F00000000003D
:20276000800F0000000000800F0000000000801F0000000000801F000000000000010000FC
:20278000000000000000000000000000000000001C0000000000000000000000000000001D
:2027A00000000000000000000000400000000000006000000000F001F000000000FC07F89D
:2027C00001000000FE0FF001000000FE0FF003000000FF1FE003000000FF1FE003000000F8
:2027E0001F3FE0030000801F3EC0070000800F3EC0070000800F7CC0070000800F7CC007BC
:202800000000800F7CC0070000800FFCC0070000800FF8C0070000800FF8C0070000001FD9
:20282000F8E1070000001FF0E3030000003FF0FF030000007EE0FF030000003EE0FF010014
:2028400000001CC0FF000000000C807F0000000000003F0000000000000000000000000053
:20286000000000000000000000001D0000000000000000000000000000000000000000003B
:2028800000001F0000000000001F0000000000001F0000000000001F0000000000001F009D
:2028A00000000000001F0000000000001F0000000000C0FFFF0F000000FEFFFF7F00000092
:2028C000FEFFFFFF000000FEFFFFFF010000FEFFFFFF030000FEFFFFFF030000001F00F8EE
:2028E000030000001F00F0070000001F00E0070000001F00C0070000001F00C007000000ED
:202900001F00C0070000001F00C0070000001F00C0070000001F00C0070000001F00C0033D
:202920000000001F00E0030000001F00E00300000000008003000000000000000000000010
:20294000000000001B0000000000000000000000000000000000000000000000000000005C
:20296000000000FFFF3F00000000FFFFFF00000000FFFFFF01000000FFFFFF03000000FF20
:20298000FFFF03000000FFFFFF070000000000F0070000000000E0070000000000C007008D
:2029A00000000000C0070000000000C0070000000000C0070000000000C0030000000000FF
:2029C000E0030000000000E0010000000000F00000000000007C00000000FFFF3F0000008A
:2029E00000FFFFFF03000000FFFFFF03000000FFFFFF03000000FFFFFF03000000FFFFFFDA
:202A00000300000000000000000000000000000000000000000000000000000000001E0095
:202A200000000000000000000000000000000001000000000000070000000000003F00004F
:202A400000000000FF000000000000FF070000000000FF1F0000000000FFFF000000000055
:202A6000F8FF0300000000C0FF1F0000000000FF7F0000000000F8FF0300000000C0FF0344
:202A80000000000000FF030000000000F0030000000000F0030000000000FE03000000004D
:202AA000C0FF0300000000F8FF0300000000FE7F00000000C0FF1F00000000F8FF03000005
:202AC0000000FEFF0000000000FF1F0000000000FF070000000000FF0000000000001F00B7
:202AE0000000000000070000000000000100000000000000000000001F00000100000000AE
:202B000000003F000000000000FF070000000000FFFF0000000000FFFF3F00000000FFFF37
:202B2000FF03000000FEFFFF03000000C0FFFF0300000000F0FF030000000000F8030000E6
:202B4000000000FC0300000000E0FF0300000000FEFF03000000F0FF1F00000000F8FF008F
:202B600000000000F8010000000000F8070000000000F8FF0000000000F0FF1F0000000058
:202B800000FFFF0300000000F0FF030000000000FE030000000000F00300000000E0FF036C
:202BA00000000000FFFF03000000FCFFFF03000000FFFFFF03000000FFFF1F00000000FFFB
:202BC000FF0000000000FF0700000000001F000000001D00000000000000000000000000B4
:202BE0000000000000000000000001000002000000030080030000000700C0030000000F73
:202C000000E0030000003F00F8030000007F00FC03000000FF01FF01000000FE83FF000099
:202C20000000FCEF3F00000000F0FF1F00000000E0FF070000000080FF030000000000FFF5
:202C4000000000000000FE030000000080FF0700000000C0FF1F00000000F0FF3F000000E1
:202C600000FCCF7F00000000FE03FF01000000FF01FE030000007F00FC030000003F00F05B
:202C8000030000000F00E0030000000700C00300000001000003000000000000020000006F
:202CA0000000000000000000000000001E00000000000000000000000000000000010000F5
:202CC00000000000070000000000001F0000001E0000FF0000001F0000FF0300001F000071
:202CE000FF0F00001F0000FE3F00001F0000F8FF00001F0000C0FF07801F000000FF1FC0F2
:202D00000F000000FC7FE00F000000E0FFF90700000080FFFF0300000000FCFF01000000DE
:202D200000E0FF0000000000FC3F0000000080FF0F00000000F0FF0300000000FE7F00007C
:202D4000000080FF1F00000000F0FF0300000000FEFF0000000000FF1F0000000000FF07C2
:202D60000000000000FF0000000000003F000000000000070000000000000100000000000D
:202D80000000000000001C0000000000000000000000000000000000000000000000000017
:202DA00000000000000000C0030000000000E0030000001F00F0030000001F00FC0300003D
:202DC000001F00FE030000001F00FF030000001F80FF030000001FC0FF030000001FE0FF32
:202DE000030000001FF0EF030000001FF8E7030000001FFEE1030000001FFFE003000000CC
:202E00009F7FE003000000DF3FE003000000FF1FE003000000FF0FE003000000FF07E003D5
:202E2000000000FF03E003000000FF00E0030000007F00E0030000003F00E0030000001F28
:202E400000E0030000000F00E003000000000000000000000000000000000000000000009D
:202E600017000000000000000000000000000000000000000000000000000000000000003B
:202E8000000000000000000000000000000000000000000000000000000000000000000032
:202EA00000FC000000000000FF030000000080FF070000000080870700000000C0030F00AE
:202EC000000000C0010E00000000C0010E00000000C0010E00000000C0010E00000000C0F6
:202EE000030F00000000808F070000000000FF030000000000FF030000000000FC000000AA
:202F00000000000000000000000000000000000000000000000000000000000000000000B1
:202F200000000000000000000000000000000000000000000000000000001200000000007F
:202F4000000000000000000000000000000000000000000000000000000000000000000071
:202F6000000000000000000000000000000000000000000000000000000000000000000051
:202F80000000000000000000000000000000000000000000000000000000000000FCFFFF37
:202FA000FFFFFF7FFCFFFFFFFFFF7FFCFFFFFFFFFF7FFCFFFFFFFFFF7F0000000000000033
:202FC0000000000000000000000000000000000000000000000000000000000000000000F1
:202FE0000000000000000000000000000000000000000000000000000000000000000000D1
:2030000000000000000000000000000000000000000000001E000000000000000000000092
:2030200000000000000000000000000000000000000000FFFFFFFF0F0000FFFFFFFF0F007A
:2030400000FFFFFFFF0F0000FFFFFFFF0F0000FFFFFFFF0F0000FFFFFFE00F00000000F86B
:20306000010000000000F0030000000000E0030000000000E0030000000000E003000000B3
:203080000000E0030000000000E0030000000000F0010000000000F0010000000000FC008C
:2030A00000000000007E00000000FFFF1F00000000FFFFFF00000000FFFFFF01000000FF7B
:2030C000FFFF03000000FFFFFF07000000FFFFFF070000000000C0070000000000C0070059
:2030E00000000000C00700000000000000001C0000000000000000000000000000000000ED
:2031000000000000000000080000000000000E0000000000800F0000000000C01F0000002B
:203120000000E00F0000000000E0070000000000F0030000000000F0010000000000F001E4
:203140000000000000F0010000000000F0030000000000E0030000000000E00700000000C1
:2031600000C00F0000000000800F0000000000801F0000000000001F0000000000001F0014
:2031800000000000001F0000000000801F0000000000C00F0000000000F00F0000000000A3
:2031A000F0070000000000E0010000000000E0000000000000000000000000000000000057
:2031C00000000000000000001F0000F803E003000080FF3FE0030000E0FFFFE0030000F0A0
:2031E000FFFFE3030000F8FFFFE7030000FCFFFFEF030000FEFFFFFF030000FF01C0FF035F
:2032000000007F0000FF0300803F0000FC0300801F0000F80300800F0000F00300C00F0084
:2032200000E00300C0070000000000C0070000000000C0070000000000C00700000000008F
:20324000C0070000000000C0070000000000C00F0000E00300800F0000F00300801F00000D
:20326000F80300803F0000FC0300007F0000FF030000FF03E0FF030000FEFFFFFF03000032
:20328000FCFFFFEF030000F8FFFFE7030000F0FFFFE3030000C0FFFFE003000000FF1FE0EF
:2032A00003000808080000000000000000000000000030787830300030006C6C6C000000FF
:2032C00000006C6CFE6CFE6C6C00183E603C067C18000063660C183363001C361C3B6E664A
:2032E0003B0030306000000000000C18303030180C0030180C0C0C18300000663CFF3C6604
:203300000000003030FC3030000000000000001818300000007E00000000000000000018FB
:20332000180003060C18306040003E63636B63633E001838581818187E003C66061C30663D
:203340007E003C66061C06663C000E1E36667F060F007E607C0606663C001C30607C66662B
:203360003C007E66060C181818003C66663C66663C003C66663E060C3800001818000018AF
:20338000180000181800001818300C18306030180C0000007E00007E000030180C060C1803
:2033A00030003C66060C180018003E636F696F603E00183C66667E6666007E33333E333381
:2033C0007E001E33606060331E007C36333333367C007F31343C34317F007F31343C343028
:2033E00078001E33606067331F006666667E666666003C18181818183C000F0606066666CC
:203400003C007333363C363373007830303031337F0063777F7F6B63630063737B6F6763FE
:2034200063003E63636363633E007E33333E303078003C6666666E3C0E007E33333E363313
:2034400073003C6630180C663C007E5A181818183C006666666666667E0066666666663CD1
:2034600018006363636B7F7763006363361C1C3663006666663C18183C007F63460C193320
:203480007F003C30303030303C006030180C060301003C0C0C0C0C0C3C00081C3663000016
:2034A000000000000000000000FF18180C000000000000003C063E663B0070303E33333339
:2034C0006E0000003C6660663C000E063E6666663B0000003C667E603C001C363078303005
:2034E000780000003B66663E067C7030363B333373001800381818183C0006000606066651
:20350000663C703033363C3673003818181818183C000000667F7F6B630000007C6666664F
:20352000660000003C6666663C0000006E33333E307800003B66663E060F00006E3B33305B
:20354000780000003E603C067C0008183E18181A0C000000666666663B0000006666663CA2
:2035600018000000636B7F7F3600000063361C36630000006666663E067C00007E4C1832DD
:203580007E000E18187018180E000C0C0C000C0C0C007018180E181870003B6E0000000082
:2035A00000001C36361C000000000000636C61696D2072657175697265732061206E616DF4
:2035C0006520746F20626520676976656E20696E2074686520696E7374616E74696F61743D
:2035E0006F72206F66207468652054657874446973706C617920696E7374616E6365210D56
:203600000A00190C0C02070000000000000000000000000000000000000000000000000264
:2036200000007F0100000000000000000000000000000000000000000307000000070000F9
:203640000000000000000000000000000000000000072400A4017C00A7017C0027002400AF
:2036600000000000000000000000060000CE001101FF031101E2000000000000000000006E
:203680000000000A00000E0011001101CE003800E60011011001E00000000000080000E018
:2036A000001E0111012901C600A0000001000000000000000002000007000000000000003F
:2036C0000000000000000000000000000000040000F80006030104000000000000000000E0
:2036E000000000000000000301040603F800000000000000000000000000000000000000C1
:203700000502000A0007000A0002000000000000000000000000000000060000100010005F
:203720007C00100010000000000000000000000000000200000007000000000000000000E4
:20374000000000000000000000000003200020002000000000000000000000000000000006
:203760000000000002000000010000000000000000000000000000000000000000038001C2
:203780007C000300000000000000000000000000000000000000060000FE000101010101A1
:2037A00001FE0000000000000000000000000006000004000200FF010000000000000000FE
:2037C000000000000000000006000002018101410131010E010000000000000000000000DB
:2037E000000600008200010111011101EE000000000000000000000000000600006000586F
:20380000004600FF0140000000000000000000000000000600009C000B0109010901F1006F
:20382000000000000000000000000000060000FE00110109010901F200000000000000006C
:2038400000000000000600000100C101390007000100000000000000000000000000060058
:2038600000EE00110111011101EE000000000000000000000000000600009E00210121014E
:203880001101FE000000000000000000000000000200000401000000000000000000000011
:2038A0000000000000000000000200004007000000000000000000000000000000000000BF
:2038C000000006000010002800280044004400000000000000000000000000064800480064
:2038E0004800480048004800000000000000000000000000060000440044002800280010BA
:203900000000000000000000000000000006000006000100610111000E0000000000000019
:203920000000000000000C0000F0010C02E204120909090909F10919090205860478020729
:20394000800170002E0021002E007000800100000000000000000000070000FF01110111DE
:203960000111011101FE00000000000000000000000800007C008200010101010101820096
:2039800044000000000000000000080000FF01010101010101010182007C000000000000D5
:2039A000000000070000FF011101110111011101110100000000000000000000060000FFA1
:2039C0000111001100110001000000000000000000000000000800007C00820001010101A8
:2039E0001101920074000000000000000000080000FF0110001000100010001000FF010057
:203A000000000000000000020000FF010000000000000000000000000000000000000000A4
:203A200005C000000100010001FF000000000000000000000000000000080000FF01200097
:203A4000100028004400820001010000000000000000070000FF010001000100010001005B
:203A60000100000000000000000000080000FF0106007800800178000600FF0100000000C0
:203A800000000000080000FF0102000C00100060008000FF01000000000000000008000018
:203AA0007C00820001010101010182007C000000000000000000070000FF011100110011CA
:203AC0000011000E00000000000000000000000800007C00820001014101410182007C013C
:203AE0000000000000000000080000FF011100110011003100D1000E01000000000000007A
:203B000000070000CE001101110111011101E6000000000000000000000007010001000198
:203B200000FF01010001000100000000000000000000000800007F00800000010001000178
:203B400080007F0000000000000000000703001C006000800160001C0003000000000000E0
:203B600000000000000B07007800800170000E0001000E00700080017C0003000000070135
:203B800001C600280010002800C60001010000000000000000000007010006000800F0012F
:203BA000080006000100000000000000000000000700018101610111010D010301010100E4
:203BC000000000000000000000030000FF07010400000000000000000000000000000000D7
:203BE00000000303007C008001000000000000000000000000000000000000020104FF07B5
:203C0000000000000000000000000000000000000000000005180006000100060018000062
:203C2000000000000000000000000000000700040004000400040004000400040000000061
:203C4000000000000000030000010002000000000000000000000000000000000000000658
:203C60000000C80024012401A400F801000000000000000000000000060000FF0188000403
:203C8000010401F800000000000000000000000000050000F8000401040188000000000097
:203CA00000000000000000000000060000F800040104010801FF01000000000000000000F3
:203CC000000000060000F800240124012401B800000000000000000000000000040400FEB9
:203CE000010500010000000000000000000000000000000000060000F8040405040588041D
:203D0000FC03000000000000000000000000060000FF01080004000400F801000000000095
:203D200000000000000000020000FD01000000000000000000000000000000000000000083
:203D4000020004FD030000000000000000000000000000000000000000060000FF01200037
:203D60003000C8000401000000000000000000000000020000FF0100000000000000000044
:203D800000000000000000000000000A0000FC01080004000400F801080004000400F8010A
:203DA00000000000060000FC01080004000400F801000000000000000000000000060000F1
:203DC000F800040104010401F800000000000000000000000000060000FC0788000401044A
:203DE00001F800000000000000000000000000060000F800040104018800FC070000000037
:203E00000000000000000000040000FC010800040000000000000000000000000000000095
:203E2000000600009800240124012401C800000000000000000000000000030400FF0104A2
:203E400001000000000000000000000000000000000000060000FC00000100010001FC015F
:203E6000000000000000000000000000050C007000800170000C00000000000000000000C4
:203E80000000000000090C007000800170000C007000800170000C0000000000000005042A
:203EA00001D8002000D80004010000000000000000000000000000050C00700480037000B4
:203EC0000C000000000000000000000000000000050401C40124011C0104010000000000C0
:203EE000000000000000000000032000DE03010400000000000000000000000000000000B9
:203F00000000020000FF070000000000000000000000000000000000000000040000010490
:203F2000DE03200000000000000000000000000000000000070000200010001000200020F9
:203F400000100000000000000000000000080000FE0102010201020102010201FE0100003C
:203F60000000000000002F737464696E002F7374646F7574002F737464657272000000005B
:203F800000C0092000C009400200000002C0092000C00040010000000AC009200080094085
:203FA000010000000FC00920000001400100000019C0092000C009400300000040C009208F
:203FC000000001400200000048C0092000800940020000009CC0092000C009400300000011
:203FE000FFFFFFFFFFFFFFFF0000000001C0092000C009400200000003C0092000C00040E8
:20400000010000000BC00920008009400100000010C0092000000140010000001AC00920A3
:2040200000C009400300000041C00920000001400200000049C0092000800940020000000A
:204040009DC0092000C0094003000000FFFFFFFFFFFFFFFF0000000007C0092000000340A3
:20406000020000000FC00920008008400200000034C0092000800840030000003FC009206C
:204080000000034002000000FFFFFFFFFFFFFFFF0000000009C009200000034002000000AC
:2040A0000DC00920000003400200000012C00920008008400200000038C009200080084017
:2040C00003000000FFFFFFFFFFFFFFFF0000000008C0092000000340020000000CC00920BA
:2040E000000003400200000011C00920008008400200000037C009200080084003000000CC
:20410000FFFFFFFFFFFFFFFF0000000006C0092000000340020000000BC00920000003403C
:204120000200000010C00920008008400200000035C009200080084003000000FFFFFFFFD5
:20414000FFFFFFFF0000000030313233343536373839414243444546403058003031323333
:204160003435363738396162636465664030780004000008000000000000000200010000AC
:204180001000000000000000000000001F1D1F1E1F1E1F1F1E1F1E1F303132333435363705
:2041A000383961626364656678700030313233343536373839414243444546585000000007
:2041C00002400000000000A00000000005400000000000C8000000000C4000000000409CC8
:2041E00000000000194000000020BCBE0000000034400000BFC91B8E00000004B54000002E
:20420000504BCFD06607E2CF010000006C4100003E8251AADFEEA73401000000D942000019
:20422000DCB5A0E23A301F97FFFFFFFFB4450000FD25A0C8E9A3C14FFFFFFFFFFF3F0000F6
:204240000000008000000000FF3F000000000080000000000000000000000000FB6E0000B7
:20426000F36E0000CB6E0000236F0000F76E000000000000AF6E0000000000000000000090
:204280002D2E00008D2E0000077200000772000007720000932D0000CF2D00001F2E000094
:2042A000252E0000292E0000FCFFFFFF00000000000000000000000000000000000000005B
:2042C000FB6E0000F36E0000CB6E0000236F0000F76E000000000000AF6E000000000000C7
:2042E000000000002D2E00008D2E0000E11400001B15000009150000932D0000EB130000A7
:204300001F2E0000252E0000292E00000772000007720000077200008B130000A7130000E3
:204320001D1400005714000093140000FCFFFFFF0000000000000000000000000000000041
:2043400000000000FB6E0000F36E0000CB6E0000236F0000F76E000000000000AF6E000046
:204360003771000000000000D92300008D2E000019240000C3230000AD230000932D00002B
:20438000332200005D210000252E0000292E0000531900003319000043190000092B000058
:2043A000A71300001D1400005714000093140000FCFFFFFF00000000000000000000000007
:2043C0000000000000000000A96D000000000000000000000772000007720000077200005C
:2043E000077200000772000007720000D56C0000116D000000000000000000000000000093
:20440000696D000000000000077200000000000000000000A96D0000000000000000000037
:20442000FB6E0000F36E0000CB6E0000236F0000F76E000000000000AF6E0000816F000075
:20444000000000000772000007720000FCFFFFFF0000000000000000000000000000000071
:2044600000000000DB6F000000000000BF6F00000000000000000000417000000000000013
:20448000000000000000000007720000077200000772000007720000077200000772000046
:2044A000D56C00009170000000000000FCFFFFFF00000000000000000000000084470100F5
:2044C000C80000100C0200000001000058480100D4020010300400005C0100007801000064
:2044E00043000000F8FFFFFF380000005400000099000000C9000000400100004301000011
:20450000460100004C01000055010000040000000A000000040000000A0000005E01000036
:2045200053756E004D6F6E00547565005765640054687500467269005361740053756E64B9
:204540006179000000004D6F6E64617900000000547565736461790000005765646E6573D4
:204560006461790054687572736461790000467269646179000000005361747572646179FD
:20458000004A616E00466562004D617200417072004D6179004A756E004A756C0041756716
:2045A00000536570004F6374004E6F7600446563004A616E756172790000004665627275A0
:2045C00061727900004D617263680000000000417072696C00000000004D61790000000085
:2045E0000000004A756E650000000000004A756C790000000000004175677573740000000C
:204600000053657074656D626572004F63746F6265720000004E6F76656D626572000044A3
:204620006563656D62657200414D00504D0025782025580025642025622025590025483ACD
:20464000254D3A25530025493A254D3A25532025700000001001000043000000F8FFFFFF6C
:20466000004040404040404040404141414141404040404040404040404040404040404075
:2046800040050202020202020202020202020202022020202020202020202002020202026D
:2046A00002029090909090901010101010101010101010101010101010101010020202024E
:2046C0000202888888888888080808080808080808080808080808080808080802020202FE
:2046E00040000000000000000000000000000000000000000000000000000000000000007A
:20470000000000000000000000000000000000000000000000000000000000000000000099
:20472000000000000000000000000000000000000000000000000000000000000000000079
:20474000000000000000000000000000000000000000000000000000000000000000000059
:20476000000000001C00000043000000F8FFFFFF0C0000000E0000000F0000002E0000008E
:2047800013CBFEFF0118B20C32065A01040174180F2057616974696E672053796E63200163
:2047A000112E205265616412100964636620646174612F20436865636B131F5061726974AD
:2047C0007924280F4C617374204D696E757465204F6B36480D5369676E616C206572726F44
:2047E0007248690111100A4C65617020596561721D1F1C1F1E0239056132033202720529F8
:2048000010290C320132045A0620290C512A10B53132303240325032603270328032903294
:20482000A032B032C032D032E042F019562A805A19522A8056196E2A8072195E2A806219A1
:184840007A2A807E19762A807A1A0708190429766BD8B8A30135000052
:00000001FF
